ARM Linker, RVCT2.2 [Build 616]

================================================================================

Image Symbol Table

    Local Symbols

    Symbol Name                              Value     Ov Type        Size  Object(Section)

    ../../unhosted.s                         0x00000000   Number         0  switch8.o ABSOLUTE
    M:\\epoc32\\build\\euser\\c_e18a23aea4fd210f\\edll_lib\\armv5\\udeb\\uc_dll_.cpp 0x00000000   Number         0  uc_dll_.o ABSOLUTE
    M:\\sf\\os\\kernelhwsrv\\kernel\\eka\\compsupp\\rvct\\ucppinit.cpp 0x00000000   Number         0  ucppinit.o ABSOLUTE
    M:\epoc32\build\euser\c_e18a23aea4fd210f\edll_lib\armv5\udeb\uc_dll_.cpp 0x00000000   Number         0  uc_dll_.o ABSOLUTE
    M:\sf\mw\uiaccelerator\uiacceltk\hitchcock\goommonitor\src\goomIdletimerule.cpp 0x00000000   Number         0  goomIdletimerule.o ABSOLUTE
    M:\sf\mw\uiaccelerator\uiacceltk\hitchcock\goommonitor\src\goomaction.cpp 0x00000000   Number         0  goomaction.o ABSOLUTE
    M:\sf\mw\uiaccelerator\uiacceltk\hitchcock\goommonitor\src\goomactionconfig.cpp 0x00000000   Number         0  goomactionconfig.o ABSOLUTE
    M:\sf\mw\uiaccelerator\uiacceltk\hitchcock\goommonitor\src\goomactionlist.cpp 0x00000000   Number         0  goomactionlist.o ABSOLUTE
    M:\sf\mw\uiaccelerator\uiacceltk\hitchcock\goommonitor\src\goomactionref.cpp 0x00000000   Number         0  goomactionref.o ABSOLUTE
    M:\sf\mw\uiaccelerator\uiacceltk\hitchcock\goommonitor\src\goomappclosetimer.cpp 0x00000000   Number         0  goomappclosetimer.o ABSOLUTE
    M:\sf\mw\uiaccelerator\uiacceltk\hitchcock\goommonitor\src\goomappclosewatcher.cpp 0x00000000   Number         0  goomappclosewatcher.o ABSOLUTE
    M:\sf\mw\uiaccelerator\uiacceltk\hitchcock\goommonitor\src\goomapplicationconfig.cpp 0x00000000   Number         0  goomapplicationconfig.o ABSOLUTE
    M:\sf\mw\uiaccelerator\uiacceltk\hitchcock\goommonitor\src\goomcloseapp.cpp 0x00000000   Number         0  goomcloseapp.o ABSOLUTE
    M:\sf\mw\uiaccelerator\uiacceltk\hitchcock\goommonitor\src\goomcloseappconfig.cpp 0x00000000   Number         0  goomcloseappconfig.o ABSOLUTE
    M:\sf\mw\uiaccelerator\uiacceltk\hitchcock\goommonitor\src\goomconfig.cpp 0x00000000   Number         0  goomconfig.o ABSOLUTE
    M:\sf\mw\uiaccelerator\uiacceltk\hitchcock\goommonitor\src\goomconfigparser.cpp 0x00000000   Number         0  goomconfigparser.o ABSOLUTE
    M:\sf\mw\uiaccelerator\uiacceltk\hitchcock\goommonitor\src\goomforegroundrule.cpp 0x00000000   Number         0  goomforegroundrule.o ABSOLUTE
    M:\sf\mw\uiaccelerator\uiacceltk\hitchcock\goommonitor\src\goomglobalconfig.cpp 0x00000000   Number         0  goomglobalconfig.o ABSOLUTE
    M:\sf\mw\uiaccelerator\uiacceltk\hitchcock\goommonitor\src\goomlog.cpp 0x00000000   Number         0  goomlog.o ABSOLUTE
    M:\sf\mw\uiaccelerator\uiacceltk\hitchcock\goommonitor\src\goommemorymonitor.cpp 0x00000000   Number         0  goommemorymonitor.o ABSOLUTE
    M:\sf\mw\uiaccelerator\uiacceltk\hitchcock\goommonitor\src\goommemorymonitorserver.cpp 0x00000000   Number         0  goommemorymonitorserver.o ABSOLUTE
    M:\sf\mw\uiaccelerator\uiacceltk\hitchcock\goommonitor\src\goommemorymonitorsession.cpp 0x00000000   Number         0  goommemorymonitorsession.o ABSOLUTE
    M:\sf\mw\uiaccelerator\uiacceltk\hitchcock\goommonitor\src\goommonitor.cpp 0x00000000   Number         0  goommonitor.o ABSOLUTE
    M:\sf\mw\uiaccelerator\uiacceltk\hitchcock\goommonitor\src\goommonitorplugin.cpp 0x00000000   Number         0  goommonitorplugin.o ABSOLUTE
    M:\sf\mw\uiaccelerator\uiacceltk\hitchcock\goommonitor\src\goommonitorsession.cpp 0x00000000   Number         0  goommonitorsession.o ABSOLUTE
    M:\sf\mw\uiaccelerator\uiacceltk\hitchcock\goommonitor\src\goompanic.cpp 0x00000000   Number         0  goompanic.o ABSOLUTE
    M:\sf\mw\uiaccelerator\uiacceltk\hitchcock\goommonitor\src\goompluginwaiter.cpp 0x00000000   Number         0  goompluginwaiter.o ABSOLUTE
    M:\sf\mw\uiaccelerator\uiacceltk\hitchcock\goommonitor\src\goomrunplugin.cpp 0x00000000   Number         0  goomrunplugin.o ABSOLUTE
    M:\sf\mw\uiaccelerator\uiacceltk\hitchcock\goommonitor\src\goomrunpluginconfig.cpp 0x00000000   Number         0  goomrunpluginconfig.o ABSOLUTE
    M:\sf\mw\uiaccelerator\uiacceltk\hitchcock\goommonitor\src\goomwindowgrouplist.cpp 0x00000000   Number         0  goomwindowgrouplist.o ABSOLUTE
    M:\sf\mw\uiaccelerator\uiacceltk\hitchcock\goommonitor\src\goomwserveventreceiver.cpp 0x00000000   Number         0  goomwserveventreceiver.o ABSOLUTE
    M:\sf\os\kernelhwsrv\kernel\eka\compsupp\rvct\dllexp.cpp 0x00000000   Number         0  dllexp.o ABSOLUTE
    M:\sf\os\kernelhwsrv\kernel\eka\compsupp\rvct\ucppinit.cpp 0x00000000   Number         0  ucppinit.o ABSOLUTE
    M:\sf\os\kernelhwsrv\kernel\eka\euser\epoc\arm\uc_dll.cpp 0x00000000   Number         0  uc_dll.o ABSOLUTE
    M:\sf\os\kernelhwsrv\kernel\eka\euser\epoc\up_dll_tls.cpp 0x00000000   Number         0  up_dll_tls.o ABSOLUTE
    .emb_text                                0x00008000   Section       40  uc_dll_.o(.emb_text)
    Symbian$$eit_base                        0x00008014   Data           4  uc_dll_.o(.emb_text)
    Symbian$$eit_limit                       0x00008018   Data           4  uc_dll_.o(.emb_text)
    Symbian$$code_seg_base                   0x0000801c   Data           4  uc_dll_.o(.emb_text)
    Symbian$$code_seg_limit                  0x00008020   Data           4  uc_dll_.o(.emb_text)
    Symbian$$reserved                        0x00008024   Data           4  uc_dll_.o(.emb_text)
    .emb_text                                0x00008028   Section       52  ucppinit.o(.emb_text)
    loop                                     0x0000803c   ARM Code       0  ucppinit.o(.emb_text)
    ret                                      0x00008044   ARM Code       0  ucppinit.o(.emb_text)
    base                                     0x00008054   Data           0  ucppinit.o(.emb_text)
    limit                                    0x00008058   Data           0  ucppinit.o(.emb_text)
    Panic(const TDesC8&, int)                0x000086bd   Thumb Code    64  goomIdletimerule.o(.text)
    .text                                    0x000086bc   Section      348  goomIdletimerule.o(.text)
    Panic(const TDesC8&, int)                0x00008819   Thumb Code    64  goomaction.o(.text)
    .text                                    0x00008818   Section      220  goomaction.o(.text)
    Panic(const TDesC8&, int)                0x000088f5   Thumb Code    64  goomactionconfig.o(.text)
    .text                                    0x000088f4   Section      432  goomactionconfig.o(.text)
    Panic(const TDesC8&, int)                0x00008aa5   Thumb Code    64  goomactionlist.o(.text)
    .text                                    0x00008aa4   Section     2978  goomactionlist.o(.text)
    .text                                    0x00009646   Section       86  goomactionref.o(.text)
    Panic(const TDesC8&, int)                0x0000969d   Thumb Code    64  goomappclosetimer.o(.text)
    .text                                    0x0000969c   Section      232  goomappclosetimer.o(.text)
    Panic(const TDesC8&, int)                0x00009785   Thumb Code    64  goomappclosewatcher.o(.text)
    .text                                    0x00009784   Section      476  goomappclosewatcher.o(.text)
    Panic(const TDesC8&, int)                0x00009961   Thumb Code    64  goomapplicationconfig.o(.text)
    .text                                    0x00009960   Section      348  goomapplicationconfig.o(.text)
    Panic(const TDesC8&, int)                0x00009abd   Thumb Code    64  goomcloseapp.o(.text)
    .text                                    0x00009abc   Section      636  goomcloseapp.o(.text)
    Panic(const TDesC8&, int)                0x00009d39   Thumb Code    64  goomcloseappconfig.o(.text)
    .text                                    0x00009d38   Section      252  goomcloseappconfig.o(.text)
    Panic(const TDesC8&, int)                0x00009e35   Thumb Code    64  goomconfig.o(.text)
    .text                                    0x00009e34   Section      900  goomconfig.o(.text)
    Panic(const TDesC8&, int)                0x0000a1b9   Thumb Code    64  goomconfigparser.o(.text)
    .text                                    0x0000a1b8   Section     4330  goomconfigparser.o(.text)
    Panic(const TDesC8&, int)                0x0000b2a5   Thumb Code    64  goomforegroundrule.o(.text)
    .text                                    0x0000b2a4   Section      228  goomforegroundrule.o(.text)
    Panic(const TDesC8&, int)                0x0000b389   Thumb Code    64  goomglobalconfig.o(.text)
    .text                                    0x0000b388   Section      144  goomglobalconfig.o(.text)
    .text                                    0x0000b418   Section     1408  goomlog.o(.text)
    Panic(const TDesC8&, int)                0x0000b999   Thumb Code    64  goommemorymonitor.o(.text)
    .text                                    0x0000b998   Section     2944  goommemorymonitor.o(.text)
    Panic(const TDesC8&, int)                0x0000c519   Thumb Code    64  goommemorymonitorserver.o(.text)
    .text                                    0x0000c518   Section      584  goommemorymonitorserver.o(.text)
    Panic(const TDesC8&, int)                0x0000c761   Thumb Code    64  goommemorymonitorsession.o(.text)
    .text                                    0x0000c760   Section     1132  goommemorymonitorsession.o(.text)
    Panic(const TDesC8&, int)                0x0000cbcd   Thumb Code    64  goommonitor.o(.text)
    .text                                    0x0000cbcc   Section      664  goommonitor.o(.text)
    Panic(const TDesC8&, int)                0x0000ce65   Thumb Code    64  goommonitorplugin.o(.text)
    .text                                    0x0000ce64   Section      680  goommonitorplugin.o(.text)
    Panic(const TDesC8&, int)                0x0000d10d   Thumb Code    64  goommonitorsession.o(.text)
    .text                                    0x0000d10c   Section     1176  goommonitorsession.o(.text)
    .text                                    0x0000d5a4   Section       52  goompanic.o(.text)
    Panic(const TDesC8&, int)                0x0000d5d9   Thumb Code    64  goompluginwaiter.o(.text)
    .text                                    0x0000d5d8   Section      292  goompluginwaiter.o(.text)
    Panic(const TDesC8&, int)                0x0000d6fd   Thumb Code    64  goomrunplugin.o(.text)
    .text                                    0x0000d6fc   Section      532  goomrunplugin.o(.text)
    Panic(const TDesC8&, int)                0x0000d911   Thumb Code    64  goomrunpluginconfig.o(.text)
    .text                                    0x0000d910   Section      296  goomrunpluginconfig.o(.text)
    Panic(const TDesC8&, int)                0x0000da39   Thumb Code    64  goomwindowgrouplist.o(.text)
    .text                                    0x0000da38   Section     3388  goomwindowgrouplist.o(.text)
    Panic(const TDesC8&, int)                0x0000e775   Thumb Code    64  goomwserveventreceiver.o(.text)
    .text                                    0x0000e774   Section      572  goomwserveventreceiver.o(.text)
    .text                                    0x0000e9b0   Section       24  switch8.o(.text)
    .text                                    0x0000e9c8   Section       80  uc_dll.o(.text)
    .text                                    0x0000ea18   Section       44  up_dll_tls.o(.text)
    .text                                    0x0000ea44   Section        4  dllexp.o(.text)
    .text.clean                              0x0000ea48   Section       40  goomIdletimerule.o(.text.clean)
    .text.clean                              0x0000ea70   Section       30  goomaction.o(.text.clean)
    .text.clean                              0x0000ea8e   Section       46  goomactionconfig.o(.text.clean)
    .text.clean                              0x0000eabc   Section      116  goomactionlist.o(.text.clean)
    .text.clean                              0x0000eb30   Section       36  goomappclosetimer.o(.text.clean)
    .text.clean                              0x0000eb54   Section       62  goomappclosewatcher.o(.text.clean)
    .text.clean                              0x0000eb92   Section       46  goomapplicationconfig.o(.text.clean)
    .text.clean                              0x0000ebc0   Section       86  goomcloseapp.o(.text.clean)
    .text.clean                              0x0000ec16   Section       30  goomcloseappconfig.o(.text.clean)
    .text.clean                              0x0000ec34   Section      108  goomconfig.o(.text.clean)
    .text.clean                              0x0000eca0   Section       28  goomconfigparser.o(.text.clean)
    .text.clean                              0x0000ecbc   Section       20  goomforegroundrule.o(.text.clean)
    .text.clean                              0x0000ecd0   Section       16  goomglobalconfig.o(.text.clean)
    .text.clean                              0x0000ece0   Section       28  goomlog.o(.text.clean)
    .text.clean                              0x0000ecfc   Section      206  goommemorymonitor.o(.text.clean)
    .text.clean                              0x0000edca   Section       70  goommemorymonitorserver.o(.text.clean)
    .text.clean                              0x0000ee10   Section       76  goommemorymonitorsession.o(.text.clean)
    .text.clean                              0x0000ee5c   Section       48  goommonitor.o(.text.clean)
    .text.clean                              0x0000ee8c   Section       56  goommonitorplugin.o(.text.clean)
    .text.clean                              0x0000eec4   Section      120  goommonitorsession.o(.text.clean)
    .text.clean                              0x0000ef3c   Section       46  goompluginwaiter.o(.text.clean)
    .text.clean                              0x0000ef6a   Section       66  goomrunplugin.o(.text.clean)
    .text.clean                              0x0000efac   Section       40  goomrunpluginconfig.o(.text.clean)
    .text.clean                              0x0000efd4   Section      172  goomwindowgrouplist.o(.text.clean)
    .text.clean                              0x0000f080   Section       72  goomwserveventreceiver.o(.text.clean)
    i._ZN11CGOomConfigC1Ev                   0x0000f0c8   Section      180  goomconfig.o(i._ZN11CGOomConfigC1Ev)
    i._ZN11CGOomConfigC1Ev.clean             0x0000f17c   Section       20  goomconfig.o(i._ZN11CGOomConfigC1Ev.clean)
    i._ZN12CleanupStack3PopEPv               0x0000f190   Section       16  goomconfigparser.o(i._ZN12CleanupStack3PopEPv)
    i._ZN13CGOomCloseApp9IsRunningEv         0x0000f1a0   Section        6  goomcloseapp.o(i._ZN13CGOomCloseApp9IsRunningEv)
    i._ZN14CGOomRunPlugin9IsRunningEv        0x0000f1a6   Section       12  goomrunplugin.o(i._ZN14CGOomRunPlugin9IsRunningEv)
    i._ZN14CMemoryMonitor21NeedToPostponeMemGoodEv 0x0000f1b2   Section       16  goommemorymonitor.o(i._ZN14CMemoryMonitor21NeedToPostponeMemGoodEv)
    i._ZN14CMemoryMonitor27SessionInCriticalAllocationEi 0x0000f1c2   Section       48  goommemorymonitorsession.o(i._ZN14CMemoryMonitor27SessionInCriticalAllocationEi)
    i._ZN15CGOomActionList8ClientIdEv        0x0000f1f2   Section        8  goomactionlist.o(i._ZN15CGOomActionList8ClientIdEv)
    i._ZN15CGOomPluginListI18CGOomMonitorPluginED0Ev 0x0000f1fa   Section       22  goomactionlist.o(i._ZN15CGOomPluginListI18CGOomMonitorPluginED0Ev)
    i._ZN16CSimpleSchedulerD0Ev              0x0000f210   Section       24  goommonitor.o(i._ZN16CSimpleSchedulerD0Ev)
    i._ZN16CSimpleSchedulerD1Ev              0x0000f228   Section       14  goommonitor.o(i._ZN16CSimpleSchedulerD1Ev)
    i._ZN17CGOomConfigParserD0Ev             0x0000f236   Section       24  goomconfigparser.o(i._ZN17CGOomConfigParserD0Ev)
    i._ZN17CGOomConfigParserD1Ev             0x0000f24e   Section       14  goomconfigparser.o(i._ZN17CGOomConfigParserD1Ev)
    i._ZN17CGOomPluginWaiterD0Ev             0x0000f25c   Section       24  goompluginwaiter.o(i._ZN17CGOomPluginWaiterD0Ev)
    i._ZN17CGOomPluginWaiterD1Ev             0x0000f274   Section       14  goompluginwaiter.o(i._ZN17CGOomPluginWaiterD1Ev)
    i._ZN18CGOomAppCloseTimerD0Ev            0x0000f282   Section       24  goomappclosetimer.o(i._ZN18CGOomAppCloseTimerD0Ev)
    i._ZN18CGOomAppCloseTimerD1Ev            0x0000f29a   Section       14  goomappclosetimer.o(i._ZN18CGOomAppCloseTimerD1Ev)
    i._ZN19CGOomForegroundRuleD0Ev           0x0000f2a8   Section       24  goomforegroundrule.o(i._ZN19CGOomForegroundRuleD0Ev)
    i._ZN19CGOomForegroundRuleD1Ev           0x0000f2c0   Section       14  goomforegroundrule.o(i._ZN19CGOomForegroundRuleD1Ev)
    i._ZN21CAppGOomMonitorPluginD0Ev         0x0000f2ce   Section       24  goommonitorplugin.o(i._ZN21CAppGOomMonitorPluginD0Ev)
    i._ZN21CAppGOomMonitorPluginD1Ev         0x0000f2e6   Section       14  goommonitorplugin.o(i._ZN21CAppGOomMonitorPluginD1Ev)
    i._ZN21CGoomThresholdCrossed10ThreadNameEv 0x0000f2f4   Section       36  goommemorymonitor.o(i._ZN21CGoomThresholdCrossed10ThreadNameEv)
    i._ZN21CGoomThresholdCrossed12SetThresholdEi 0x0000f318   Section       44  goommemorymonitor.o(i._ZN21CGoomThresholdCrossed12SetThresholdEi)
    i._ZN21CGoomThresholdCrossed12SetThresholdEi.clean 0x0000f344   Section       10  goommemorymonitor.o(i._ZN21CGoomThresholdCrossed12SetThresholdEi.clean)
    i._ZN21CGoomThresholdCrossed15ResetThresholdsEv 0x0000f350   Section       48  goommemorymonitor.o(i._ZN21CGoomThresholdCrossed15ResetThresholdsEv)
    i._ZN21CGoomThresholdCrossed15ResetThresholdsEv.clean 0x0000f380   Section       10  goommemorymonitor.o(i._ZN21CGoomThresholdCrossed15ResetThresholdsEv.clean)
    i._ZN21CGoomThresholdCrossed18StartRequestEventsEv 0x0000f38c   Section      324  goommemorymonitor.o(i._ZN21CGoomThresholdCrossed18StartRequestEventsEv)
    i._ZN21CGoomThresholdCrossed18StartRequestEventsEv.clean 0x0000f4d0   Section       10  goommemorymonitor.o(i._ZN21CGoomThresholdCrossed18StartRequestEventsEv.clean)
    i._ZN21CGoomThresholdCrossed20RequestNotificationsEi 0x0000f4dc   Section       96  goommemorymonitor.o(i._ZN21CGoomThresholdCrossed20RequestNotificationsEi)
    i._ZN21CGoomThresholdCrossed20RequestNotificationsEi.clean 0x0000f53c   Section       10  goommemorymonitor.o(i._ZN21CGoomThresholdCrossed20RequestNotificationsEi.clean)
    i._ZN21CGoomThresholdCrossed4RunLEv      0x0000f548   Section      124  goommemorymonitor.o(i._ZN21CGoomThresholdCrossed4RunLEv)
    i._ZN21CGoomThresholdCrossed4RunLEv.clean 0x0000f5c4   Section       14  goommemorymonitor.o(i._ZN21CGoomThresholdCrossed4RunLEv.clean)
    i._ZN21CGoomThresholdCrossed4StopEv      0x0000f5d2   Section       30  goommemorymonitor.o(i._ZN21CGoomThresholdCrossed4StopEv)
    i._ZN21CGoomThresholdCrossed7TriggerEi   0x0000f5f0   Section      172  goommemorymonitor.o(i._ZN21CGoomThresholdCrossed7TriggerEi)
    i._ZN21CGoomThresholdCrossed7TriggerEi.clean 0x0000f69c   Section       10  goommemorymonitor.o(i._ZN21CGoomThresholdCrossed7TriggerEi.clean)
    i._ZN21CGoomThresholdCrossed8ContinueEv  0x0000f6a6   Section       24  goommemorymonitor.o(i._ZN21CGoomThresholdCrossed8ContinueEv)
    i._ZN21CGoomThresholdCrossed8DoCancelEv  0x0000f6c0   Section       40  goommemorymonitor.o(i._ZN21CGoomThresholdCrossed8DoCancelEv)
    i._ZN21CGoomThresholdCrossed8DoCancelEv.clean 0x0000f6e8   Section       10  goommemorymonitor.o(i._ZN21CGoomThresholdCrossed8DoCancelEv.clean)
    i._ZN21CGoomThresholdCrossedC1ER14CMemoryMonitorji 0x0000f6f4   Section      240  goommemorymonitor.o(i._ZN21CGoomThresholdCrossedC1ER14CMemoryMonitorji)
    i._ZN21CGoomThresholdCrossedC1ER14CMemoryMonitorji.clean 0x0000f7e4   Section       16  goommemorymonitor.o(i._ZN21CGoomThresholdCrossedC1ER14CMemoryMonitorji.clean)
    i._ZN21CGoomThresholdCrossedD0Ev         0x0000f7f4   Section       22  goommemorymonitor.o(i._ZN21CGoomThresholdCrossedD0Ev)
    i._ZN21CGoomThresholdCrossedD1Ev         0x0000f80c   Section      100  goommemorymonitor.o(i._ZN21CGoomThresholdCrossedD1Ev)
    i._ZN21CGoomThresholdCrossedD1Ev.clean   0x0000f870   Section       26  goommemorymonitor.o(i._ZN21CGoomThresholdCrossedD1Ev.clean)
    i._ZN5CBasenwEj                          0x0000f88a   Section       16  goommonitor.o(i._ZN5CBasenwEj)
    i._ZN5TLex8C1ERK6TDesC8                  0x0000f89a   Section       30  goomconfigparser.o(i._ZN5TLex8C1ERK6TDesC8)
    i._ZN8TFuncLog7CleanupEPv                0x0000f8b8   Section       44  goomIdletimerule.o(i._ZN8TFuncLog7CleanupEPv)
    i._ZN8TFuncLogC1EPKc                     0x0000f8e4   Section      244  goomIdletimerule.o(i._ZN8TFuncLogC1EPKc)
    i._ZN8TFuncLogD1Ev                       0x0000f9d8   Section       40  goomconfigparser.o(i._ZN8TFuncLogD1Ev)
    i._ZNK12RMessagePtr26IsNullEv            0x0000fa00   Section       16  goommemorymonitorsession.o(i._ZNK12RMessagePtr26IsNullEv)
    i._ZNK12RSessionBase11SendReceiveEiRK8TIpcArgs 0x0000fa10   Section       20  goommonitorsession.o(i._ZNK12RSessionBase11SendReceiveEiRK8TIpcArgs)
    i._ZNK16CSimpleScheduler5ErrorEi         0x0000fa24   Section        2  goommonitor.o(i._ZNK16CSimpleScheduler5ErrorEi)
    i._ZNK17CGOomIdleTimeRule8PriorityEv     0x0000fa26   Section        6  goomIdletimerule.o(i._ZNK17CGOomIdleTimeRule8PriorityEv)
    i._ZNK19CGOomForegroundRule8PriorityEv   0x0000fa2c   Section        6  goomforegroundrule.o(i._ZNK19CGOomForegroundRule8PriorityEv)
    i._ZNK20CGOomWindowGroupList5CountEv     0x0000fa32   Section       14  goomactionlist.o(i._ZNK20CGOomWindowGroupList5CountEv)
    i._ZNK6TDesC8eqERKS_                     0x0000fa40   Section       26  goomconfigparser.o(i._ZNK6TDesC8eqERKS_)
    i._ZThn4_N15CGOomActionList8ClientIdEv   0x0000fa5a   Section       12  goomactionlist.o(i._ZThn4_N15CGOomActionList8ClientIdEv)
    i._ZThn4_NK17CGOomIdleTimeRule8PriorityEv 0x0000fa66   Section        8  goomIdletimerule.o(i._ZThn4_NK17CGOomIdleTimeRule8PriorityEv)
    i._ZThn4_NK19CGOomForegroundRule8PriorityEv 0x0000fa6e   Section        8  goomforegroundrule.o(i._ZThn4_NK19CGOomForegroundRule8PriorityEv)
    i._ZdlPvS_                               0x0000fa76   Section        2  goomconfigparser.o(i._ZdlPvS_)
    i._ZnwjPv                                0x0000fa78   Section        6  goomIdletimerule.o(i._ZnwjPv)
    t._ZN12CleanupCloseI13RPointerArrayI26CImplementationInformationEE5CloseEPv 0x0000fa7e   Section       14  goomactionlist.o(t._ZN12CleanupCloseI13RPointerArrayI26CImplementationInformationEE5CloseEPv)
    t._ZN12CleanupCloseI5RFileE5CloseEPv     0x0000fa8c   Section       12  goomconfigparser.o(t._ZN12CleanupCloseI5RFileE5CloseEPv)
    t._ZN13RPointerArrayI13CGOomCloseAppE15ResetAndDestroyEv 0x0000fa98   Section       64  goomactionlist.o(t._ZN13RPointerArrayI13CGOomCloseAppE15ResetAndDestroyEv)
    t._ZN13RPointerArrayI14CGOomRunPluginE15ResetAndDestroyEv 0x0000fad8   Section       64  goomactionlist.o(t._ZN13RPointerArrayI14CGOomRunPluginE15ResetAndDestroyEv)
    t._ZN13RPointerArrayI15MGOomRuleConfigE15ResetAndDestroyEv 0x0000fb18   Section       54  goomactionconfig.o(t._ZN13RPointerArrayI15MGOomRuleConfigE15ResetAndDestroyEv)
    t._ZN15CGOomPluginListI18CGOomMonitorPluginE10ConstructLEi 0x0000fb50   Section      208  goomactionlist.o(t._ZN15CGOomPluginListI18CGOomMonitorPluginE10ConstructLEi)
    t._ZN15CGOomPluginListI18CGOomMonitorPluginE10ConstructLEi.clean 0x0000fc20   Section       10  goomactionlist.o(t._ZN15CGOomPluginListI18CGOomMonitorPluginE10ConstructLEi.clean)
    t._ZN15CGOomPluginListI18CGOomMonitorPluginE3UidEi 0x0000fc2a   Section       18  goomactionlist.o(t._ZN15CGOomPluginListI18CGOomMonitorPluginE3UidEi)
    t._ZN15CGOomPluginListI18CGOomMonitorPluginE4NewLEi 0x0000fc3c   Section       76  goomactionlist.o(t._ZN15CGOomPluginListI18CGOomMonitorPluginE4NewLEi)
    t._ZN15CGOomPluginListI18CGOomMonitorPluginE4NewLEi.clean 0x0000fc88   Section       10  goomactionlist.o(t._ZN15CGOomPluginListI18CGOomMonitorPluginE4NewLEi.clean)
    t._ZN15CGOomPluginListI18CGOomMonitorPluginE5CountEv 0x0000fc92   Section       14  goomactionlist.o(t._ZN15CGOomPluginListI18CGOomMonitorPluginE5CountEv)
    t._ZN15CGOomPluginListI18CGOomMonitorPluginE7TPluginC1Ev 0x0000fca0   Section       36  goomactionlist.o(t._ZN15CGOomPluginListI18CGOomMonitorPluginE7TPluginC1Ev)
    t._ZN15CGOomPluginListI18CGOomMonitorPluginEC1Ev 0x0000fcc4   Section       60  goomactionlist.o(t._ZN15CGOomPluginListI18CGOomMonitorPluginEC1Ev)
    t._ZN15CGOomPluginListI18CGOomMonitorPluginEC1Ev.clean 0x0000fd00   Section       10  goomactionlist.o(t._ZN15CGOomPluginListI18CGOomMonitorPluginEC1Ev.clean)
    t._ZN15CGOomPluginListI18CGOomMonitorPluginED1Ev 0x0000fd0c   Section       96  goomactionlist.o(t._ZN15CGOomPluginListI18CGOomMonitorPluginED1Ev)
    t._ZN15CGOomPluginListI18CGOomMonitorPluginED1Ev.clean 0x0000fd6c   Section       16  goomactionlist.o(t._ZN15CGOomPluginListI18CGOomMonitorPluginED1Ev.clean)
    t._ZN6RArrayI10TActionRefEixEi           0x0000fd7c   Section       16  goomactionlist.o(t._ZN6RArrayI10TActionRefEixEi)
    t._ZN6RArrayIN10RWsSession21TWindowGroupChainInfoEE8ReserveLEi 0x0000fd8c   Section       22  goomlog.o(t._ZN6RArrayIN10RWsSession21TWindowGroupChainInfoEE8ReserveLEi)
    t._ZN6RArrayIN10RWsSession21TWindowGroupChainInfoEEC1Ev 0x0000fda2   Section       16  goomwindowgrouplist.o(t._ZN6RArrayIN10RWsSession21TWindowGroupChainInfoEEC1Ev)
    t._ZN6RArrayIN10RWsSession21TWindowGroupChainInfoEEixEi 0x0000fdb2   Section       16  goomlog.o(t._ZN6RArrayIN10RWsSession21TWindowGroupChainInfoEEixEi)
    t._ZN6RArrayIN15CGOomPluginListI18CGOomMonitorPluginE7TPluginEEixEi 0x0000fdc2   Section       16  goomactionlist.o(t._ZN6RArrayIN15CGOomPluginListI18CGOomMonitorPluginE7TPluginEEixEi)
    t._ZN8RHashMapIiN20CGOomWindowGroupList26TGOomWindowGroupPropertiesEE4FindERKi 0x0000fdd2   Section       28  goomwindowgrouplist.o(t._ZN8RHashMapIiN20CGOomWindowGroupList26TGOomWindowGroupPropertiesEE4FindERKi)
    t._ZN8RHashMapIlP20CGOomRunPluginConfigE4FindERKl 0x0000fdee   Section       28  goomconfig.o(t._ZN8RHashMapIlP20CGOomRunPluginConfigE4FindERKl)
    t._ZN8RHashMapIlP22CGOomApplicationConfigE4FindERKl 0x0000fe0a   Section       28  goomconfig.o(t._ZN8RHashMapIlP22CGOomApplicationConfigE4FindERKl)
    t._ZN8RHashMapIlP22CGOomApplicationConfigE7InsertLERKlRKS1_ 0x0000fe26   Section       34  goomconfig.o(t._ZN8RHashMapIlP22CGOomApplicationConfigE7InsertLERKlRKS1_)
    t._ZNK6RArrayI10TActionRefE5CountEv      0x0000fe48   Section       12  goomactionlist.o(t._ZNK6RArrayI10TActionRefE5CountEv)
    t._ZNK6RArrayIN10RWsSession21TWindowGroupChainInfoEE5CountEv 0x0000fe54   Section       12  goomwindowgrouplist.o(t._ZNK6RArrayIN10RWsSession21TWindowGroupChainInfoEE5CountEv)
    .extab._ZN17CGOomIdleTimeRuleC1E20TTimeIntervalSecondsi 0x0000fe60   Data           0  goomIdletimerule.o(.ARM.extab)
    .extab._ZN17CGOomIdleTimeRule4NewLE20TTimeIntervalSecondsi 0x0000fe70   Data           0  goomIdletimerule.o(.ARM.extab)
    .extab._ZNK17CGOomIdleTimeRule16RuleIsApplicableERK20CGOomWindowGroupListi 0x0000fe80   Data           0  goomIdletimerule.o(.ARM.extab)
    .extab._ZN17CGOomIdleTimeRuleD1Ev        0x0000fe90   Data           0  goomIdletimerule.o(.ARM.extab)
    .extab._ZN11CGOomActionD2Ev              0x0000fea0   Data           0  goomaction.o(.ARM.extab)
    .extab._ZN11CGOomAction11MemoryFreedEi   0x0000feb0   Data           0  goomaction.o(.ARM.extab)
    .extab._ZN11CGOomActionC2ER19MGOomActionObserver 0x0000fec0   Data           0  goomaction.o(.ARM.extab)
    .extab._ZN17CGOomActionConfig8AddRuleLEP15MGOomRuleConfig 0x0000fed0   Data           0  goomactionconfig.o(.ARM.extab)
    .extab._ZN17CGOomActionConfigD1Ev        0x0000fee0   Data           0  goomactionconfig.o(.ARM.extab)
    .extab._ZNK17CGOomActionConfig8PriorityERK20CGOomWindowGroupListi 0x0000ff00   Data           0  goomactionconfig.o(.ARM.extab)
    .extab._ZN17CGOomActionConfigC1El        0x0000ff10   Data           0  goomactionconfig.o(.ARM.extab)
    .extab._ZN15CGOomActionList10ConstructLER11CGOomConfig 0x0000ff20   Data           0  goomactionlist.o(.ARM.extab)
    .extab._ZN15CGOomActionListC1ER14CMemoryMonitorR20CMemoryMonitorServerR10RWsSession 0x0000ff30   Data           0  goomactionlist.o(.ARM.extab)
    .extab._ZN15CGOomActionList4NewLER14CMemoryMonitorR20CMemoryMonitorServerR10RWsSessionR11CGOomConfig 0x0000ff40   Data           0  goomactionlist.o(.ARM.extab)
    .extab._ZN15CGOomActionListD1Ev          0x0000ff50   Data           0  goomactionlist.o(.ARM.extab)
    .extab._ZN15CGOomActionList17ComparePrioritiesERK10TActionRefS2_ 0x0000ff70   Data           0  goomactionlist.o(.ARM.extab)
    .extab._ZN15CGOomActionList16BuildActionListLER20CGOomWindowGroupListR11CGOomConfig 0x0000ffd0   Data           0  goomactionlist.o(.ARM.extab)
    .extab._ZN15CGOomActionList10MemoryGoodEv 0x0000ffe8   Data           0  goomactionlist.o(.ARM.extab)
    .extab._ZN15CGOomActionList21FreeMemoryAboveTargetERi 0x0000fff8   Data           0  goomactionlist.o(.ARM.extab)
    .extab._ZN15CGOomActionList10FreeMemoryEi 0x00010008   Data           0  goomactionlist.o(.ARM.extab)
    .extab._ZN15CGOomActionList13AppNotExitingEi 0x00010028   Data           0  goomactionlist.o(.ARM.extab)
    .extab._ZN15CGOomActionList12StateChangedEv 0x00010038   Data           0  goomactionlist.o(.ARM.extab)
    .extab._ZN15CGOomPluginListI18CGOomMonitorPluginE10ConstructLEi 0x00010048   Data           0  goomactionlist.o(.ARM.extab)
    .extab._ZN15CGOomPluginListI18CGOomMonitorPluginEC1Ev 0x00010058   Data           0  goomactionlist.o(.ARM.extab)
    .extab._ZN15CGOomPluginListI18CGOomMonitorPluginE4NewLEi 0x00010068   Data           0  goomactionlist.o(.ARM.extab)
    .extab._ZN15CGOomPluginListI18CGOomMonitorPluginED1Ev 0x00010078   Data           0  goomactionlist.o(.ARM.extab)
    .extab._ZN18CGOomAppCloseTimerC1ER13CGOomCloseApp 0x00010098   Data           0  goomappclosetimer.o(.ARM.extab)
    .extab._ZN18CGOomAppCloseTimer4NewLER13CGOomCloseApp 0x000100b8   Data           0  goomappclosetimer.o(.ARM.extab)
    .extab._ZN18CGOomAppCloseTimer4RunLEv    0x000100c8   Data           0  goomappclosetimer.o(.ARM.extab)
    .extab._ZN20CGOomAppCloseWatcherC1ER13CGOomCloseApp 0x000100d8   Data           0  goomappclosewatcher.o(.ARM.extab)
    .extab._ZN20CGOomAppCloseWatcherD1Ev     0x000100f8   Data           0  goomappclosewatcher.o(.ARM.extab)
    .extab._ZN20CGOomAppCloseWatcher5StartERK8TApaTask 0x00010118   Data           0  goomappclosewatcher.o(.ARM.extab)
    .extab._ZN20CGOomAppCloseWatcher8DoCancelEv 0x00010128   Data           0  goomappclosewatcher.o(.ARM.extab)
    .extab._ZN20CGOomAppCloseWatcher4RunLEv  0x00010138   Data           0  goomappclosewatcher.o(.ARM.extab)
    .extab._ZN22CGOomApplicationConfigC1Ej   0x00010148   Data           0  goomapplicationconfig.o(.ARM.extab)
    .extab._ZN22CGOomApplicationConfig4NewLEj 0x00010158   Data           0  goomapplicationconfig.o(.ARM.extab)
    .extab._ZN22CGOomApplicationConfig8AddRuleLEP15MGOomRuleConfig 0x00010168   Data           0  goomapplicationconfig.o(.ARM.extab)
    .extab._ZN22CGOomApplicationConfigD1Ev   0x00010178   Data           0  goomapplicationconfig.o(.ARM.extab)
    .extab._ZN13CGOomCloseApp10ConstructLEv  0x00010198   Data           0  goomcloseapp.o(.ARM.extab)
    .extab._ZN13CGOomCloseAppC1ER19MGOomActionObserverR10RWsSession 0x000101a8   Data           0  goomcloseapp.o(.ARM.extab)
    .extab._ZN13CGOomCloseApp4NewLER19MGOomActionObserverR10RWsSession 0x000101b8   Data           0  goomcloseapp.o(.ARM.extab)
    .extab._ZN13CGOomCloseApp10FreeMemoryEi  0x000101c8   Data           0  goomcloseapp.o(.ARM.extab)
    .extab._ZN13CGOomCloseAppD1Ev            0x000101d8   Data           0  goomcloseapp.o(.ARM.extab)
    .extab._ZN13CGOomCloseApp13CloseAppEventEv 0x000101f8   Data           0  goomcloseapp.o(.ARM.extab)
    .extab._ZN13CGOomCloseApp11ReconfigureERK10TActionRef 0x00010208   Data           0  goomcloseapp.o(.ARM.extab)
    .extab._ZN13CGOomCloseApp8KillTaskEv     0x00010218   Data           0  goomcloseapp.o(.ARM.extab)
    .extab._ZN19CGOomCloseAppConfigC1El      0x00010228   Data           0  goomcloseappconfig.o(.ARM.extab)
    .extab._ZN19CGOomCloseAppConfig4NewLEl   0x00010238   Data           0  goomcloseappconfig.o(.ARM.extab)
    .extab._ZN19CGOomCloseAppConfigD1Ev      0x00010248   Data           0  goomcloseappconfig.o(.ARM.extab)
    .extab._ZN11CGOomConfig4NewLEv           0x00010258   Data           0  goomconfig.o(.ARM.extab)
    .extab._ZN11CGOomConfig18SetAppCloseConfigLEP19CGOomCloseAppConfig 0x00010268   Data           0  goomconfig.o(.ARM.extab)
    .extab._ZN11CGOomConfig16AddPluginConfigLEP20CGOomRunPluginConfig 0x00010278   Data           0  goomconfig.o(.ARM.extab)
    .extab._ZN11CGOomConfig19AddApplicationRuleLEjP15MGOomRuleConfig 0x00010288   Data           0  goomconfig.o(.ARM.extab)
    .extab._ZN11CGOomConfig14AddPluginRuleLEjP15MGOomRuleConfig 0x00010298   Data           0  goomconfig.o(.ARM.extab)
    .extab._ZN11CGOomConfig21AddApplicationConfigLEP22CGOomApplicationConfig 0x000102a8   Data           0  goomconfig.o(.ARM.extab)
    .extab._ZN11CGOomConfig20GetApplicationConfigEl 0x000102b8   Data           0  goomconfig.o(.ARM.extab)
    .extab._ZN11CGOomConfig15GetPluginConfigEl 0x000102c8   Data           0  goomconfig.o(.ARM.extab)
    .extab._ZN11CGOomConfigD1Ev              0x000102d8   Data           0  goomconfig.o(.ARM.extab)
    .extab._ZN11CGOomConfigC1Ev              0x00010300   Data           0  goomconfig.o(.ARM.extab)
    .extab._ZN17CGOomConfigParser6ParseLEv   0x00010318   Data           0  goomconfigparser.o(.ARM.extab)
    .extab._ZN17CGOomConfigParser25GetValueFromAttributeListERK6RArrayIN3Xml10RAttributeEERK6TDesC8R6TPtrC8 0x0001032c   Data           0  goomconfigparser.o(.ARM.extab)
    .extab._ZN19CGOomForegroundRuleC1Eii     0x0001033c   Data           0  goomforegroundrule.o(.ARM.extab)
    .extab._ZNK19CGOomForegroundRule16RuleIsApplicableERK20CGOomWindowGroupListi 0x0001034c   Data           0  goomforegroundrule.o(.ARM.extab)
    .extab._ZN17CGOomGlobalConfigD1Ev        0x0001035c   Data           0  goomglobalconfig.o(.ARM.extab)
    .extab._ZN11CGOomLoggerC1ER10RWsSessionR3RFs 0x0001037c   Data           0  goomlog.o(.ARM.extab)
    .extab._ZN11CGOomLogger17LogApplicationIdsEv 0x0001038c   Data           0  goomlog.o(.ARM.extab)
    .extab._ZN11CGOomLoggerD1Ev              0x000103c0   Data           0  goomlog.o(.ARM.extab)
    .extab._Z29CreateThresholdCrossedThreadLR14CMemoryMonitorji 0x000103d0   Data           0  goommemorymonitor.o(.ARM.extab)
    .extab._ZN14CMemoryMonitor13GetFreeMemoryEv 0x000103e0   Data           0  goommemorymonitor.o(.ARM.extab)
    .extab._ZN14CMemoryMonitor17RefreshThresholdsEi 0x00010400   Data           0  goommemorymonitor.o(.ARM.extab)
    .extab._ZN14CMemoryMonitor10ConstructLEv 0x00010488   Data           0  goommemorymonitor.o(.ARM.extab)
    .extab._ZN14CMemoryMonitorC1Ev           0x00010498   Data           0  goommemorymonitor.o(.ARM.extab)
    .extab._ZN14CMemoryMonitor4NewLEv        0x000104b8   Data           0  goommemorymonitor.o(.ARM.extab)
    .extab._ZN14CMemoryMonitorD1Ev           0x000104c8   Data           0  goommemorymonitor.o(.ARM.extab)
    .extab._ZN14CMemoryMonitor33FreeGraphicsMemoryAboveThresholdLERi 0x000104e8   Data           0  goommemorymonitor.o(.ARM.extab)
    .extab._ZN14CMemoryMonitor17StartFreeSomeRamLEii 0x000104f8   Data           0  goommemorymonitor.o(.ARM.extab)
    .extab._ZN14CMemoryMonitor17StartFreeSomeRamLEi 0x00010510   Data           0  goommemorymonitor.o(.ARM.extab)
    .extab._ZN14CMemoryMonitor24FreeMemThresholdCrossedLEii 0x00010520   Data           0  goommemorymonitor.o(.ARM.extab)
    .extab._ZN14CMemoryMonitor13AppNotExitingEi 0x00010530   Data           0  goommemorymonitor.o(.ARM.extab)
    .extab._ZN14CMemoryMonitor16FreeOptionalRamLEiii 0x00010540   Data           0  goommemorymonitor.o(.ARM.extab)
    .extab._ZN14CMemoryMonitor18RequestFreeMemoryLEii 0x00010550   Data           0  goommemorymonitor.o(.ARM.extab)
    .extab._ZN14CMemoryMonitor22HandleFocusedWgChangeLEi 0x00010560   Data           0  goommemorymonitor.o(.ARM.extab)
    .extab._ZN14CMemoryMonitor15SetPriorityBusyEi 0x00010578   Data           0  goommemorymonitor.o(.ARM.extab)
    .extab._ZN14CMemoryMonitor17SetPriorityNormalEi 0x00010588   Data           0  goommemorymonitor.o(.ARM.extab)
    .extab._ZN14CMemoryMonitor21DoPostponedMemoryGoodEv 0x00010598   Data           0  goommemorymonitor.o(.ARM.extab)
    .extab._ZN21CGoomThresholdCrossed15ResetThresholdsEv 0x000105a8   Data           0  goommemorymonitor.o(.ARM.extab)
    .extab._ZN21CGoomThresholdCrossed7TriggerEi 0x000105b8   Data           0  goommemorymonitor.o(.ARM.extab)
    .extab._ZN21CGoomThresholdCrossed18StartRequestEventsEv 0x000105c8   Data           0  goommemorymonitor.o(.ARM.extab)
    .extab._ZN21CGoomThresholdCrossed20RequestNotificationsEi 0x000105e0   Data           0  goommemorymonitor.o(.ARM.extab)
    .extab._ZN21CGoomThresholdCrossed12SetThresholdEi 0x000105f0   Data           0  goommemorymonitor.o(.ARM.extab)
    .extab._ZN21CGoomThresholdCrossedD1Ev    0x00010600   Data           0  goommemorymonitor.o(.ARM.extab)
    .extab._ZN21CGoomThresholdCrossedC1ER14CMemoryMonitorji 0x00010628   Data           0  goommemorymonitor.o(.ARM.extab)
    .extab._ZN21CGoomThresholdCrossed4RunLEv 0x00010648   Data           0  goommemorymonitor.o(.ARM.extab)
    .extab._ZN21CGoomThresholdCrossed8DoCancelEv 0x00010688   Data           0  goommemorymonitor.o(.ARM.extab)
    .extab._ZN20CMemoryMonitorServer10ConstructLEv 0x00010698   Data           0  goommemorymonitorserver.o(.ARM.extab)
    .extab._ZN20CMemoryMonitorServerC1ER14CMemoryMonitor 0x000106a8   Data           0  goommemorymonitorserver.o(.ARM.extab)
    .extab._ZN20CMemoryMonitorServer4NewLER14CMemoryMonitor 0x000106b8   Data           0  goommemorymonitorserver.o(.ARM.extab)
    .extab._ZN20CMemoryMonitorServerD1Ev     0x000106c8   Data           0  goommemorymonitorserver.o(.ARM.extab)
    .extab._ZN20CMemoryMonitorServer17CloseAppsFinishedEii 0x000106d8   Data           0  goommemorymonitorserver.o(.ARM.extab)
    .extab._ZNK20CMemoryMonitorServer11NewSessionLERK8TVersionRK9RMessage2 0x000106e8   Data           0  goommemorymonitorserver.o(.ARM.extab)
    .extab._ZN20CMemoryMonitorServer8RunErrorEi 0x000106f8   Data           0  goommemorymonitorserver.o(.ARM.extab)
    .extab._ZN21CMemoryMonitorSessionC1Ev    0x00010708   Data           0  goommemorymonitorsession.o(.ARM.extab)
    .extab._ZN21CMemoryMonitorSession17CloseAppsFinishedEii 0x00010718   Data           0  goommemorymonitorsession.o(.ARM.extab)
    .extab._ZN21CMemoryMonitorSessionD1Ev    0x00010728   Data           0  goommemorymonitorsession.o(.ARM.extab)
    .extab._ZN21CMemoryMonitorSession7MonitorEv 0x00010748   Data           0  goommemorymonitorsession.o(.ARM.extab)
    .extab._ZN21CMemoryMonitorSession8ServiceLERK9RMessage2 0x00010758   Data           0  goommemorymonitorsession.o(.ARM.extab)
    .extab._Z25GOOMWatcherThreadFunctionPv   0x00010810   Data           0  goommonitor.o(.ARM.extab)
    .extab._Z24CreateGOOMWatcherThreadLv     0x00010868   Data           0  goommonitor.o(.ARM.extab)
    .extab._Z11PanicClientRK12RMessagePtr223TGOomMonitorClientPanic 0x00010878   Data           0  goommonitor.o(.ARM.extab)
    .extab._ZN5CBasenwEj                     0x00010888   Data           0  goommonitor.o(.ARM.extab)
    .extab._Z20SetGMemoryMonitorTlsP14CMemoryMonitor 0x00010898   Data           0  goommonitorplugin.o(.ARM.extab)
    .extab._Z16MemoryMonitorTlsv             0x000108a8   Data           0  goommonitorplugin.o(.ARM.extab)
    .extab._Z22GOomMonitorPluginPanic23TGOomMonitorPluginPanic 0x000108b8   Data           0  goommonitorplugin.o(.ARM.extab)
    .extab._ZN22CGOomMonitorPluginBaseC2Ev   0x000108c8   Data           0  goommonitorplugin.o(.ARM.extab)
    .extab._ZN22CGOomMonitorPluginBaseD2Ev   0x000108e8   Data           0  goommonitorplugin.o(.ARM.extab)
    .extab._ZN19RGOomMonitorSession7ConnectEv 0x000108f8   Data           0  goommonitorsession.o(.ARM.extab)
    .extab._ZN19RGOomMonitorSession17RequestFreeMemoryEi 0x00010908   Data           0  goommonitorsession.o(.ARM.extab)
    .extab._ZN19RGOomMonitorSession17RequestFreeMemoryEiR14TRequestStatus 0x00010918   Data           0  goommonitorsession.o(.ARM.extab)
    .extab._ZN19RGOomMonitorSession18RequestOptionalRamEiiiRi 0x00010928   Data           0  goommonitorsession.o(.ARM.extab)
    .extab._ZN19RGOomMonitorSession18RequestOptionalRamEiiiR14TRequestStatus 0x00010938   Data           0  goommonitorsession.o(.ARM.extab)
    .extab._ZN19RGOomMonitorSession23CancelRequestFreeMemoryEv 0x00010948   Data           0  goommonitorsession.o(.ARM.extab)
    .extab._ZN19RGOomMonitorSession19ThisAppIsNotExitingEi 0x00010958   Data           0  goommonitorsession.o(.ARM.extab)
    .extab._ZN19RGOomMonitorSession15SetGOomPriorityENS_13TGOomPriorityE 0x00010968   Data           0  goommonitorsession.o(.ARM.extab)
    .extab._ZN19RGOomMonitorSession23ApplicationAboutToStartERK4TUid 0x00010980   Data           0  goommonitorsession.o(.ARM.extab)
    .extab._ZN19RGOomMonitorSession22UsesAbsoluteMemTargetsEi 0x00010990   Data           0  goommonitorsession.o(.ARM.extab)
    .extab._ZN19RGOomMonitorSession7ConnectER14TRequestStatus 0x000109a0   Data           0  goommonitorsession.o(.ARM.extab)
    .extab._ZN19RGOomMonitorSession15AppAboutToStartER14TRequestStatusRK4TUid 0x000109b0   Data           0  goommonitorsession.o(.ARM.extab)
    .extab._ZN17CGOomPluginWaiterC1EiR14CGOomRunPlugin 0x000109c0   Data           0  goompluginwaiter.o(.ARM.extab)
    .extab._ZN17CGOomPluginWaiter4NewLEiR14CGOomRunPlugin 0x000109e0   Data           0  goompluginwaiter.o(.ARM.extab)
    .extab._ZN17CGOomPluginWaiter5StartEv    0x000109f0   Data           0  goompluginwaiter.o(.ARM.extab)
    .extab._ZN17CGOomPluginWaiter4RunLEv     0x00010a00   Data           0  goompluginwaiter.o(.ARM.extab)
    .extab._ZN14CGOomRunPlugin10ConstructLER20CGOomRunPluginConfig 0x00010a10   Data           0  goomrunplugin.o(.ARM.extab)
    .extab._ZN14CGOomRunPluginC1EjR20CGOomRunPluginConfigR19MGOomActionObserverR18CGOomMonitorPlugin 0x00010a20   Data           0  goomrunplugin.o(.ARM.extab)
    .extab._ZN14CGOomRunPlugin4NewLEjR20CGOomRunPluginConfigR19MGOomActionObserverR18CGOomMonitorPlugin 0x00010a30   Data           0  goomrunplugin.o(.ARM.extab)
    .extab._ZN14CGOomRunPluginD1Ev           0x00010a40   Data           0  goomrunplugin.o(.ARM.extab)
    .extab._ZN14CGOomRunPlugin10FreeMemoryEi 0x00010a60   Data           0  goomrunplugin.o(.ARM.extab)
    .extab._ZN14CGOomRunPlugin10MemoryGoodEv 0x00010a70   Data           0  goomrunplugin.o(.ARM.extab)
    .extab._ZN20CGOomRunPluginConfigC1Ej15TGOomPluginType 0x00010a80   Data           0  goomrunpluginconfig.o(.ARM.extab)
    .extab._ZN20CGOomRunPluginConfig4NewLEj15TGOomPluginType 0x00010a90   Data           0  goomrunpluginconfig.o(.ARM.extab)
    .extab._ZN20CGOomRunPluginConfig23CalculatePluginPriorityERK20CGOomWindowGroupList 0x00010aa0   Data           0  goomrunpluginconfig.o(.ARM.extab)
    .extab._ZN20CGOomRunPluginConfigD1Ev     0x00010ab0   Data           0  goomrunpluginconfig.o(.ARM.extab)
    .extab._ZN20CGOomWindowGroupList10ConstructLEv 0x00010ac0   Data           0  goomwindowgrouplist.o(.ARM.extab)
    .extab._ZN20CGOomWindowGroupListC1ER10RWsSession 0x00010ad0   Data           0  goomwindowgrouplist.o(.ARM.extab)
    .extab._ZN20CGOomWindowGroupList4NewLER10RWsSession 0x00010ae0   Data           0  goomwindowgrouplist.o(.ARM.extab)
    .extab._ZNK20CGOomWindowGroupList5AppIdEii 0x00010af0   Data           0  goomwindowgrouplist.o(.ARM.extab)
    .extab._ZN20CGOomWindowGroupList33RemovePropertiesForClosedWindowsLEv 0x00010b08   Data           0  goomwindowgrouplist.o(.ARM.extab)
    .extab._ZN20CGOomWindowGroupList23CollapseWindowGroupTreeEv 0x00010b18   Data           0  goomwindowgrouplist.o(.ARM.extab)
    .extab._ZN20CGOomWindowGroupList8RefreshLEv 0x00010b28   Data           0  goomwindowgrouplist.o(.ARM.extab)
    .extab._ZN20CGOomWindowGroupList7RefreshEv 0x00010b50   Data           0  goomwindowgrouplist.o(.ARM.extab)
    .extab._ZNK20CGOomWindowGroupList8IdleTimeEi 0x00010b90   Data           0  goomwindowgrouplist.o(.ARM.extab)
    .extab._ZN20CGOomWindowGroupListD1Ev     0x00010ba0   Data           0  goomwindowgrouplist.o(.ARM.extab)
    .extab._ZN20CGOomWindowGroupList15SetPriorityBusyEi 0x00010bc0   Data           0  goomwindowgrouplist.o(.ARM.extab)
    .extab._ZN20CGOomWindowGroupList17SetPriorityNormalEi 0x00010c08   Data           0  goomwindowgrouplist.o(.ARM.extab)
    .extab._ZN20CGOomWindowGroupList15SetPriorityHighEi 0x00010c50   Data           0  goomwindowgrouplist.o(.ARM.extab)
    .extab._ZN20CGOomWindowGroupList21IsDynamicHighPriorityEi 0x00010c98   Data           0  goomwindowgrouplist.o(.ARM.extab)
    .extab._ZNK20CGOomWindowGroupList17GetIndexFromAppIdEj 0x00010cb0   Data           0  goomwindowgrouplist.o(.ARM.extab)
    .extab._ZN19CWservEventReceiverC1ER14CMemoryMonitorR10RWsSession 0x00010cc0   Data           0  goomwserveventreceiver.o(.ARM.extab)
    .extab._ZN19CWservEventReceiverD1Ev      0x00010ce0   Data           0  goomwserveventreceiver.o(.ARM.extab)
    .extab._ZN19CWservEventReceiver5QueueEv  0x00010d00   Data           0  goomwserveventreceiver.o(.ARM.extab)
    .extab._ZN19CWservEventReceiver10ConstructLEv 0x00010d10   Data           0  goomwserveventreceiver.o(.ARM.extab)
    .extab._ZN19CWservEventReceiver8DoCancelEv 0x00010d20   Data           0  goomwserveventreceiver.o(.ARM.extab)
    .extab._ZN19CWservEventReceiver4RunLEv   0x00010d30   Data           0  goomwserveventreceiver.o(.ARM.extab)
    .constdata$1                             0x00010d40   Data           0  goomIdletimerule.o(.constdata)
    KFuncNameTerminator                      0x00010d40   Data           8  goomIdletimerule.o(.constdata)
    .constdata                               0x00010d40   Section      383  goomIdletimerule.o(.constdata)
    KFuncLeavePatternL                       0x00010d48   Data           8  goomIdletimerule.o(.constdata)
    __PRETTY_FUNCTION__@_ZN17CGOomIdleTimeRule4NewLE20TTimeIntervalSecondsi_0 0x00010d50   Data          77  goomIdletimerule.o(.constdata)
    _ZZNK17CGOomIdleTimeRule16RuleIsApplicableERK20CGOomWindowGroupListiE19__PRETTY_FUNCTION__@_ZNK17CGOomIdleTimeRule16RuleIsApplicableERK20CGOomWindowGroupListi_0 0x00010d9d   Data          88  goomIdletimerule.o(.constdata)
    __PRETTY_FUNCTION__@_ZN17CGOomIdleTimeRuleD1Ev_0 0x00010df5   Data          40  goomIdletimerule.o(.constdata)
    __PRETTY_FUNCTION__@_ZN17CGOomIdleTimeRuleC1E20TTimeIntervalSecondsi_0 0x00010e1d   Data          71  goomIdletimerule.o(.constdata)
    .constdata$1                             0x00010ec0   Data           0  goomaction.o(.constdata)
    KFuncNameTerminator                      0x00010ec0   Data           8  goomaction.o(.constdata)
    .constdata                               0x00010ec0   Section      227  goomaction.o(.constdata)
    KFuncLeavePatternL                       0x00010ec8   Data           8  goomaction.o(.constdata)
    __PRETTY_FUNCTION__@_ZN11CGOomActionD2Ev_0 0x00010ed0   Data          28  goomaction.o(.constdata)
    __PRETTY_FUNCTION__@_ZN11CGOomAction11MemoryFreedEi_0 0x00010eec   Data          42  goomaction.o(.constdata)
    __PRETTY_FUNCTION__@_ZN11CGOomActionC2ER19MGOomActionObserver_0 0x00010f16   Data          48  goomaction.o(.constdata)
    .constdata$1                             0x00010fa4   Data           0  goomactionconfig.o(.constdata)
    KFuncNameTerminator                      0x00010fa4   Data           8  goomactionconfig.o(.constdata)
    .constdata                               0x00010fa4   Section      371  goomactionconfig.o(.constdata)
    KFuncLeavePatternL                       0x00010fac   Data           8  goomactionconfig.o(.constdata)
    __PRETTY_FUNCTION__@_ZN17CGOomActionConfig8AddRuleLEP15MGOomRuleConfig_0 0x00010fb4   Data          52  goomactionconfig.o(.constdata)
    __PRETTY_FUNCTION__@_ZN17CGOomActionConfigD1Ev_0 0x00010fe8   Data          40  goomactionconfig.o(.constdata)
    __PRETTY_FUNCTION__@_ZNK17CGOomActionConfig8PriorityERK20CGOomWindowGroupListi_0 0x00011010   Data          89  goomactionconfig.o(.constdata)
    __PRETTY_FUNCTION__@_ZN17CGOomActionConfig10ConstructLEv_0 0x00011069   Data          37  goomactionconfig.o(.constdata)
    __PRETTY_FUNCTION__@_ZN17CGOomActionConfigC1El_0 0x0001108e   Data          43  goomactionconfig.o(.constdata)
    .constdata$1                             0x00011118   Data           0  goomactionlist.o(.constdata)
    KFuncNameTerminator                      0x00011118   Data           8  goomactionlist.o(.constdata)
    .constdata                               0x00011118   Section     3476  goomactionlist.o(.constdata)
    KFuncLeavePatternL                       0x00011120   Data           8  goomactionlist.o(.constdata)
    __PRETTY_FUNCTION__@_ZN15CGOomActionList4NewLER14CMemoryMonitorR20CMemoryMonitorServerR10RWsSessionR11CGOomConfig_0 0x00011128   Data         110  goomactionlist.o(.constdata)
    __PRETTY_FUNCTION__@_ZN15CGOomActionListD1Ev_0 0x00011196   Data          36  goomactionlist.o(.constdata)
    __PRETTY_FUNCTION__@_ZN15CGOomActionList16BuildActionListLER20CGOomWindowGroupListR11CGOomConfig_0 0x000111ba   Data          78  goomactionlist.o(.constdata)
    __PRETTY_FUNCTION__@_ZN15CGOomActionList10FreeMemoryEi_0 0x00011208   Data          45  goomactionlist.o(.constdata)
    __PRETTY_FUNCTION__@_ZN15CGOomActionList10MemoryGoodEv_0 0x00011235   Data          35  goomactionlist.o(.constdata)
    __PRETTY_FUNCTION__@_ZN15CGOomActionList21FreeMemoryAboveTargetERi_0 0x00011258   Data          57  goomactionlist.o(.constdata)
    __PRETTY_FUNCTION__@_ZN15CGOomActionList17ComparePrioritiesERK10TActionRefS2__0 0x00011291   Data          86  goomactionlist.o(.constdata)
    __PRETTY_FUNCTION__@_ZN15CGOomActionList13AppNotExitingEi_0 0x000112e7   Data          48  goomactionlist.o(.constdata)
    _ZZN15CGOomActionList12StateChangedEvE19__PRETTY_FUNCTION__@_ZN15CGOomActionList12StateChangedEv_0 0x00011317   Data          37  goomactionlist.o(.constdata)
    __PRETTY_FUNCTION__@_ZN15CGOomActionListC1ER14CMemoryMonitorR20CMemoryMonitorServerR10RWsSession_0 0x0001133c   Data          89  goomactionlist.o(.constdata)
    __PRETTY_FUNCTION__@_ZN15CGOomActionList10ConstructLER11CGOomConfig_0 0x00011395   Data          48  goomactionlist.o(.constdata)
    .constdata$1                             0x00011eac   Data           0  goomappclosetimer.o(.constdata)
    KFuncNameTerminator                      0x00011eac   Data           8  goomappclosetimer.o(.constdata)
    .constdata                               0x00011eac   Section      259  goomappclosetimer.o(.constdata)
    KFuncLeavePatternL                       0x00011eb4   Data           8  goomappclosetimer.o(.constdata)
    __PRETTY_FUNCTION__@_ZN18CGOomAppCloseTimer4NewLER13CGOomCloseApp_0 0x00011ebc   Data          62  goomappclosetimer.o(.constdata)
    __PRETTY_FUNCTION__@_ZN18CGOomAppCloseTimerC1ER13CGOomCloseApp_0 0x00011efa   Data          56  goomappclosetimer.o(.constdata)
    __PRETTY_FUNCTION__@_ZN18CGOomAppCloseTimer4RunLEv_0 0x00011f32   Data          32  goomappclosetimer.o(.constdata)
    .constdata$1                             0x00011fb0   Data           0  goomappclosewatcher.o(.constdata)
    KFuncNameTerminator                      0x00011fb0   Data           8  goomappclosewatcher.o(.constdata)
    .constdata                               0x00011fb0   Section      339  goomappclosewatcher.o(.constdata)
    KFuncLeavePatternL                       0x00011fb8   Data           8  goomappclosewatcher.o(.constdata)
    __PRETTY_FUNCTION__@_ZN20CGOomAppCloseWatcherC1ER13CGOomCloseApp_0 0x00011fc0   Data          60  goomappclosewatcher.o(.constdata)
    __PRETTY_FUNCTION__@_ZN20CGOomAppCloseWatcherD1Ev_0 0x00011ffc   Data          46  goomappclosewatcher.o(.constdata)
    __PRETTY_FUNCTION__@_ZN20CGOomAppCloseWatcher5StartERK8TApaTask_0 0x0001202a   Data          51  goomappclosewatcher.o(.constdata)
    __PRETTY_FUNCTION__@_ZN20CGOomAppCloseWatcher8DoCancelEv_0 0x0001205d   Data          38  goomappclosewatcher.o(.constdata)
    __PRETTY_FUNCTION__@_ZN20CGOomAppCloseWatcher4RunLEv_0 0x00012083   Data          34  goomappclosewatcher.o(.constdata)
    .constdata$1                             0x00012104   Data           0  goomapplicationconfig.o(.constdata)
    KFuncNameTerminator                      0x00012104   Data           8  goomapplicationconfig.o(.constdata)
    .constdata                               0x00012104   Section      387  goomapplicationconfig.o(.constdata)
    KFuncLeavePatternL                       0x0001210c   Data           8  goomapplicationconfig.o(.constdata)
    __PRETTY_FUNCTION__@_ZN22CGOomApplicationConfig4NewLEj_0 0x00012114   Data          67  goomapplicationconfig.o(.constdata)
    __PRETTY_FUNCTION__@_ZN22CGOomApplicationConfig8AddRuleLEP15MGOomRuleConfig_0 0x00012157   Data          57  goomapplicationconfig.o(.constdata)
    __PRETTY_FUNCTION__@_ZN22CGOomApplicationConfigD1Ev_0 0x00012190   Data          50  goomapplicationconfig.o(.constdata)
    __PRETTY_FUNCTION__@_ZN22CGOomApplicationConfig10ConstructLEv_0 0x000121c2   Data          42  goomapplicationconfig.o(.constdata)
    __PRETTY_FUNCTION__@_ZN22CGOomApplicationConfigC1Ej_0 0x000121ec   Data          61  goomapplicationconfig.o(.constdata)
    .constdata$1                             0x00012288   Data           0  goomcloseapp.o(.constdata)
    KFuncNameTerminator                      0x00012288   Data           8  goomcloseapp.o(.constdata)
    .constdata                               0x00012288   Section      636  goomcloseapp.o(.constdata)
    KFuncLeavePatternL                       0x00012290   Data           8  goomcloseapp.o(.constdata)
    __PRETTY_FUNCTION__@_ZN13CGOomCloseApp4NewLER19MGOomActionObserverR10RWsSession_0 0x00012298   Data          72  goomcloseapp.o(.constdata)
    __PRETTY_FUNCTION__@_ZN13CGOomCloseApp10FreeMemoryEi_0 0x000122e0   Data          43  goomcloseapp.o(.constdata)
    __PRETTY_FUNCTION__@_ZN13CGOomCloseAppD1Ev_0 0x0001230b   Data          32  goomcloseapp.o(.constdata)
    __PRETTY_FUNCTION__@_ZN13CGOomCloseApp13CloseAppEventEv_0 0x0001232b   Data          36  goomcloseapp.o(.constdata)
    __PRETTY_FUNCTION__@_ZN13CGOomCloseApp11ReconfigureERK10TActionRef_0 0x0001234f   Data          52  goomcloseapp.o(.constdata)
    __PRETTY_FUNCTION__@_ZN13CGOomCloseApp8KillTaskEv_0 0x00012383   Data          31  goomcloseapp.o(.constdata)
    __PRETTY_FUNCTION__@_ZN13CGOomCloseAppC1ER19MGOomActionObserverR10RWsSession_0 0x000123a2   Data          66  goomcloseapp.o(.constdata)
    __PRETTY_FUNCTION__@_ZN13CGOomCloseApp10ConstructLEv_0 0x000123e4   Data          33  goomcloseapp.o(.constdata)
    .constdata$1                             0x00012504   Data           0  goomcloseappconfig.o(.constdata)
    KFuncNameTerminator                      0x00012504   Data           8  goomcloseappconfig.o(.constdata)
    .constdata                               0x00012504   Section      251  goomcloseappconfig.o(.constdata)
    KFuncLeavePatternL                       0x0001250c   Data           8  goomcloseappconfig.o(.constdata)
    __PRETTY_FUNCTION__@_ZN19CGOomCloseAppConfig4NewLEl_0 0x00012514   Data          53  goomcloseappconfig.o(.constdata)
    __PRETTY_FUNCTION__@_ZN19CGOomCloseAppConfigD1Ev_0 0x00012549   Data          44  goomcloseappconfig.o(.constdata)
    __PRETTY_FUNCTION__@_ZN19CGOomCloseAppConfigC1El_0 0x00012575   Data          47  goomcloseappconfig.o(.constdata)
    .constdata$1                             0x00012600   Data           0  goomconfig.o(.constdata)
    KFuncNameTerminator                      0x00012600   Data           8  goomconfig.o(.constdata)
    .constdata                               0x00012600   Section      643  goomconfig.o(.constdata)
    KFuncLeavePatternL                       0x00012608   Data           8  goomconfig.o(.constdata)
    __PRETTY_FUNCTION__@_ZN11CGOomConfig4NewLEv_0 0x00012610   Data          33  goomconfig.o(.constdata)
    __PRETTY_FUNCTION__@_ZN11CGOomConfig18SetAppCloseConfigLEP19CGOomCloseAppConfig_0 0x00012631   Data          60  goomconfig.o(.constdata)
    __PRETTY_FUNCTION__@_ZN11CGOomConfig16AddPluginConfigLEP20CGOomRunPluginConfig_0 0x0001266d   Data          59  goomconfig.o(.constdata)
    __PRETTY_FUNCTION__@_ZN11CGOomConfig19AddApplicationRuleLEjP15MGOomRuleConfig_0 0x000126a8   Data          71  goomconfig.o(.constdata)
    __PRETTY_FUNCTION__@_ZN11CGOomConfig14AddPluginRuleLEjP15MGOomRuleConfig_0 0x000126ef   Data          66  goomconfig.o(.constdata)
    __PRETTY_FUNCTION__@_ZN11CGOomConfig21AddApplicationConfigLEP22CGOomApplicationConfig_0 0x00012731   Data          66  goomconfig.o(.constdata)
    __PRETTY_FUNCTION__@_ZN11CGOomConfig20GetApplicationConfigEl_0 0x00012773   Data          64  goomconfig.o(.constdata)
    __PRETTY_FUNCTION__@_ZN11CGOomConfig15GetPluginConfigEl_0 0x000127b3   Data          57  goomconfig.o(.constdata)
    __PRETTY_FUNCTION__@_ZN11CGOomConfigD1Ev_0 0x000127ec   Data          28  goomconfig.o(.constdata)
    __PRETTY_FUNCTION__@_ZN11CGOomConfig10ConstructLEv_0 0x00012808   Data          31  goomconfig.o(.constdata)
    .constdata$1                             0x00012884   Data           0  goomconfigparser.o(.constdata)
    KFuncNameTerminator                      0x00012884   Data           8  goomconfigparser.o(.constdata)
    .constdata                               0x00012884   Section     1420  goomconfigparser.o(.constdata)
    KFuncLeavePatternL                       0x0001288c   Data           8  goomconfigparser.o(.constdata)
    KXmlMimeType                             0x00012894   Data          16  goomconfigparser.o(.constdata)
    KGOomConfigFilePath                      0x000128a4   Data          72  goomconfigparser.o(.constdata)
    KRomDrive                                0x000128ec   Data           8  goomconfigparser.o(.constdata)
    KGOomConfigGOomConfig                    0x000128f4   Data          16  goomconfigparser.o(.constdata)
    KGOomConfigGlobalSettings                0x00012904   Data          20  goomconfigparser.o(.constdata)
    KGOomConfigForceCheckAtPriority          0x00012918   Data          16  goomconfigparser.o(.constdata)
    KGOomConfigAppSettings                   0x00012928   Data          28  goomconfigparser.o(.constdata)
    KGOomConfigApp                           0x00012944   Data           8  goomconfigparser.o(.constdata)
    KGOomConfigAppCloseSettings              0x0001294c   Data          24  goomconfigparser.o(.constdata)
    KGOomConfigCloseApp                      0x00012964   Data          16  goomconfigparser.o(.constdata)
    KGOomConfigAppCloseIdlePriority          0x00012974   Data          28  goomconfigparser.o(.constdata)
    KGOomConfigForegroundAppPriority         0x00012990   Data          28  goomconfigparser.o(.constdata)
    KGOomAttributeLowRamThreshold            0x000129ac   Data          24  goomconfigparser.o(.constdata)
    KGOomAttributeGoodRamThreshold           0x000129c4   Data          24  goomconfigparser.o(.constdata)
    KGOomAttributeMaxAppCloseBatch           0x000129dc   Data          24  goomconfigparser.o(.constdata)
    KGOomAttributeDefaultWaitAfterPlugin     0x000129f4   Data          32  goomconfigparser.o(.constdata)
    KGOomAttributeTargetFreeOnStartup        0x00012a14   Data          28  goomconfigparser.o(.constdata)
    KGOomAttributeSystemPluginSettings       0x00012a30   Data          28  goomconfigparser.o(.constdata)
    KGOomAttributeSystemPlugin               0x00012a4c   Data          20  goomconfigparser.o(.constdata)
    KGOomAttributeAppPluginSettings          0x00012a60   Data          24  goomconfigparser.o(.constdata)
    KGOomAttributeAppPlugin                  0x00012a78   Data          16  goomconfigparser.o(.constdata)
    KGOomAttributePluginIdlePriority         0x00012a88   Data          28  goomconfigparser.o(.constdata)
    KGOomAttributePluginForegroundAppPriority 0x00012aa4   Data          36  goomconfigparser.o(.constdata)
    KGOomAttibuteUid                         0x00012ac8   Data           8  goomconfigparser.o(.constdata)
    KGOomAttibuteSyncMode                    0x00012ad0   Data          16  goomconfigparser.o(.constdata)
    KGOomAttibutePriority                    0x00012ae0   Data          16  goomconfigparser.o(.constdata)
    KGOomAttibuteRamEstimate                 0x00012af0   Data          20  goomconfigparser.o(.constdata)
    KGOomConfigSyncModeContinue              0x00012b04   Data          16  goomconfigparser.o(.constdata)
    KGOomConfigSyncModeCheck                 0x00012b14   Data          12  goomconfigparser.o(.constdata)
    KGOomConfigSyncModeEstimate              0x00012b20   Data          16  goomconfigparser.o(.constdata)
    KGOomAttibuteIdleTime                    0x00012b30   Data          16  goomconfigparser.o(.constdata)
    KGOomAttibuteIdlePriority                0x00012b40   Data          16  goomconfigparser.o(.constdata)
    KGOomAttibuteNeverClose                  0x00012b50   Data          16  goomconfigparser.o(.constdata)
    KGOomAttributeTargetAppId                0x00012b60   Data          20  goomconfigparser.o(.constdata)
    KGOomAttributeWait                       0x00012b74   Data          12  goomconfigparser.o(.constdata)
    KGOomAttributeIfForegroundAppId          0x00012b80   Data          28  goomconfigparser.o(.constdata)
    KGOomConfigDefaultAppUid                 0x00012b9c   Data          16  goomconfigparser.o(.constdata)
    KGOomConfigDefaultPluginUid              0x00012bac   Data          20  goomconfigparser.o(.constdata)
    KGOomConfigTargetAppValue                0x00012bc0   Data          16  goomconfigparser.o(.constdata)
    KGOomConfigBusyAppUid                    0x00012bd0   Data          16  goomconfigparser.o(.constdata)
    KGOomConfigHighPriorityAppUid            0x00012be0   Data          24  goomconfigparser.o(.constdata)
    __PRETTY_FUNCTION__@_ZN17CGOomConfigParser6ParseLEv_0 0x00012bf8   Data          33  goomconfigparser.o(.constdata)
    _ZZN17CGOomConfigParser16OnStartDocumentLERKN3Xml19RDocumentParametersEiE19__PRETTY_FUNCTION__@_ZN17CGOomConfigParser16OnStartDocumentLERKN3Xml19RDocumentParametersEi_0 0x00012c19   Data          87  goomconfigparser.o(.constdata)
    _ZZN17CGOomConfigParser14OnEndDocumentLEiE19__PRETTY_FUNCTION__@_ZN17CGOomConfigParser14OnEndDocumentLEi_0 0x00012c70   Data          51  goomconfigparser.o(.constdata)
    .constdata$1                             0x00012e10   Data           0  goomforegroundrule.o(.constdata)
    KFuncNameTerminator                      0x00012e10   Data           8  goomforegroundrule.o(.constdata)
    .constdata                               0x00012e10   Section      263  goomforegroundrule.o(.constdata)
    KFuncLeavePatternL                       0x00012e18   Data           8  goomforegroundrule.o(.constdata)
    __PRETTY_FUNCTION__@_ZN19CGOomForegroundRuleC1Eii_0 0x00012e20   Data          65  goomforegroundrule.o(.constdata)
    _ZZNK19CGOomForegroundRule16RuleIsApplicableERK20CGOomWindowGroupListiE19__PRETTY_FUNCTION__@_ZNK19CGOomForegroundRule16RuleIsApplicableERK20CGOomWindowGroupListi_0 0x00012e61   Data          90  goomforegroundrule.o(.constdata)
    .constdata$1                             0x00012f18   Data           0  goomglobalconfig.o(.constdata)
    KFuncNameTerminator                      0x00012f18   Data           8  goomglobalconfig.o(.constdata)
    .constdata                               0x00012f18   Section      132  goomglobalconfig.o(.constdata)
    KFuncLeavePatternL                       0x00012f20   Data           8  goomglobalconfig.o(.constdata)
    __PRETTY_FUNCTION__@_ZN17CGOomGlobalConfigD1Ev_0 0x00012f28   Data          40  goomglobalconfig.o(.constdata)
    .constdata$1                             0x00012f9c   Data           0  goomlog.o(.constdata)
    KMemorySampleLoggingString               0x00012f9c   Data           8  goomlog.o(.constdata)
    .constdata                               0x00012f9c   Section      316  goomlog.o(.constdata)
    KMemorySampleLoggingSeparator            0x00012fa4   Data           8  goomlog.o(.constdata)
    KCrLf                                    0x00012fac   Data           8  goomlog.o(.constdata)
    KGOomLogCancel                           0x00012fb4   Data          80  goomlog.o(.constdata)
    KGOomLogFile                             0x00013004   Data          72  goomlog.o(.constdata)
    KGOomOldLogFile                          0x0001304c   Data          64  goomlog.o(.constdata)
    KTimeStampFormat                         0x0001308c   Data          36  goomlog.o(.constdata)
    KDummyWgName                             0x000130b0   Data          12  goomlog.o(.constdata)
    KUidPreamble                             0x000130bc   Data          16  goomlog.o(.constdata)
    KUidFormat                               0x000130cc   Data          12  goomlog.o(.constdata)
    .constdata$1                             0x000130d8   Data           0  goommemorymonitor.o(.constdata)
    KFuncNameTerminator                      0x000130d8   Data           8  goommemorymonitor.o(.constdata)
    .constdata                               0x000130d8   Section     4564  goommemorymonitor.o(.constdata)
    KFuncLeavePatternL                       0x000130e0   Data           8  goommemorymonitor.o(.constdata)
    KGoomAsyncWaitThreadName                 0x000130e8   Data          24  goommemorymonitor.o(.constdata)
    __PRETTY_FUNCTION__@_Z29CreateThresholdCrossedThreadLR14CMemoryMonitorji_0 0x00013100   Data          97  goommemorymonitor.o(.constdata)
    __PRETTY_FUNCTION__@_ZN14CMemoryMonitor4NewLEv_0 0x00013161   Data          39  goommemorymonitor.o(.constdata)
    __PRETTY_FUNCTION__@_ZN14CMemoryMonitorD1Ev_0 0x00013188   Data          34  goommemorymonitor.o(.constdata)
    __PRETTY_FUNCTION__@_ZN14CMemoryMonitor24FreeMemThresholdCrossedLEii_0 0x000131aa   Data          70  goommemorymonitor.o(.constdata)
    __PRETTY_FUNCTION__@_ZN14CMemoryMonitor13AppNotExitingEi_0 0x000131f0   Data          47  goommemorymonitor.o(.constdata)
    __PRETTY_FUNCTION__@_ZN14CMemoryMonitor17StartFreeSomeRamLEi_0 0x0001321f   Data          51  goommemorymonitor.o(.constdata)
    __PRETTY_FUNCTION__@_ZN14CMemoryMonitor16FreeOptionalRamLEiii_0 0x00013252   Data          67  goommemorymonitor.o(.constdata)
    __PRETTY_FUNCTION__@_ZN14CMemoryMonitor18RequestFreeMemoryLEii_0 0x00013295   Data          57  goommemorymonitor.o(.constdata)
    __PRETTY_FUNCTION__@_ZN14CMemoryMonitor22HandleFocusedWgChangeLEi_0 0x000132ce   Data          56  goommemorymonitor.o(.constdata)
    __PRETTY_FUNCTION__@_ZN14CMemoryMonitor15SetPriorityBusyEi_0 0x00013306   Data          49  goommemorymonitor.o(.constdata)
    __PRETTY_FUNCTION__@_ZN14CMemoryMonitor17SetPriorityNormalEi_0 0x00013337   Data          51  goommemorymonitor.o(.constdata)
    __PRETTY_FUNCTION__@_ZN14CMemoryMonitor12ResetTargetsEv_0 0x0001336a   Data          36  goommemorymonitor.o(.constdata)
    __PRETTY_FUNCTION__@_ZN14CMemoryMonitor13GetFreeMemoryEv_0 0x0001338e   Data          43  goommemorymonitor.o(.constdata)
    __PRETTY_FUNCTION__@_ZN14CMemoryMonitor21DoPostponedMemoryGoodEv_0 0x000133b9   Data          45  goommemorymonitor.o(.constdata)
    __PRETTY_FUNCTION__@_ZN14CMemoryMonitorC1Ev_0 0x000133e6   Data          33  goommemorymonitor.o(.constdata)
    __PRETTY_FUNCTION__@_ZN14CMemoryMonitor10ConstructLEv_0 0x00013407   Data          34  goommemorymonitor.o(.constdata)
    __PRETTY_FUNCTION__@_ZN14CMemoryMonitor33FreeGraphicsMemoryAboveThresholdLERi_0 0x00013429   Data          68  goommemorymonitor.o(.constdata)
    __PRETTY_FUNCTION__@_ZN14CMemoryMonitor17RefreshThresholdsEi_0 0x0001346d   Data          51  goommemorymonitor.o(.constdata)
    __PRETTY_FUNCTION__@_ZN14CMemoryMonitor17StartFreeSomeRamLEii_0 0x000134a0   Data          63  goommemorymonitor.o(.constdata)
    .constdata$1                             0x000142ac   Data           0  goommemorymonitorserver.o(.constdata)
    KGraphicsMemoryMonitorServerName         0x000142ac   Data          40  goommemorymonitorserver.o(.constdata)
    .constdata                               0x000142ac   Section      952  goommemorymonitorserver.o(.constdata)
    KFuncNameTerminator                      0x000142d4   Data           8  goommemorymonitorserver.o(.constdata)
    KFuncLeavePatternL                       0x000142dc   Data           8  goommemorymonitorserver.o(.constdata)
    __PRETTY_FUNCTION__@_ZN20CMemoryMonitorServer4NewLER14CMemoryMonitor_0 0x000142e4   Data          67  goommemorymonitorserver.o(.constdata)
    __PRETTY_FUNCTION__@_ZN20CMemoryMonitorServerD1Ev_0 0x00014327   Data          46  goommemorymonitorserver.o(.constdata)
    __PRETTY_FUNCTION__@_ZN20CMemoryMonitorServer7MonitorEv_0 0x00014355   Data          48  goommemorymonitorserver.o(.constdata)
    __PRETTY_FUNCTION__@_ZN20CMemoryMonitorServer17CloseAppsFinishedEii_0 0x00014385   Data          62  goommemorymonitorserver.o(.constdata)
    __PRETTY_FUNCTION__@_ZN20CMemoryMonitorServerC1ER14CMemoryMonitor_0 0x000143c3   Data          61  goommemorymonitorserver.o(.constdata)
    __PRETTY_FUNCTION__@_ZN20CMemoryMonitorServer10ConstructLEv_0 0x00014400   Data          40  goommemorymonitorserver.o(.constdata)
    __PRETTY_FUNCTION__@_ZNK20CMemoryMonitorServer11NewSessionLERK8TVersionRK9RMessage2_0 0x00014428   Data          88  goommemorymonitorserver.o(.constdata)
    __PRETTY_FUNCTION__@_ZN20CMemoryMonitorServer8RunErrorEi_0 0x00014480   Data          54  goommemorymonitorserver.o(.constdata)
    .constdata$1                             0x00014664   Data           0  goommemorymonitorsession.o(.constdata)
    KFuncNameTerminator                      0x00014664   Data           8  goommemorymonitorsession.o(.constdata)
    .constdata                               0x00014664   Section      636  goommemorymonitorsession.o(.constdata)
    KFuncLeavePatternL                       0x0001466c   Data           8  goommemorymonitorsession.o(.constdata)
    __PRETTY_FUNCTION__@_ZN21CMemoryMonitorSessionC1Ev_0 0x00014674   Data          47  goommemorymonitorsession.o(.constdata)
    __PRETTY_FUNCTION__@_ZN21CMemoryMonitorSession7CreateLEv_0 0x000146a3   Data          38  goommemorymonitorsession.o(.constdata)
    __PRETTY_FUNCTION__@_ZN21CMemoryMonitorSession17CloseAppsFinishedEii_0 0x000146c9   Data          63  goommemorymonitorsession.o(.constdata)
    __PRETTY_FUNCTION__@_ZN21CMemoryMonitorSessionD1Ev_0 0x00014708   Data          48  goommemorymonitorsession.o(.constdata)
    __PRETTY_FUNCTION__@_ZN21CMemoryMonitorSession6ServerEv_0 0x00014738   Data          54  goommemorymonitorsession.o(.constdata)
    __PRETTY_FUNCTION__@_ZN21CMemoryMonitorSession7MonitorEv_0 0x0001476e   Data          49  goommemorymonitorsession.o(.constdata)
    __PRETTY_FUNCTION__@_ZN21CMemoryMonitorSession8ServiceLERK9RMessage2_0 0x0001479f   Data          56  goommemorymonitorsession.o(.constdata)
    .constdata$1                             0x000148e0   Data           0  goommonitor.o(.constdata)
    KGraphicsMemoryMonitorServerName         0x000148e0   Data          40  goommonitor.o(.constdata)
    .constdata                               0x000148e0   Section      476  goommonitor.o(.constdata)
    KFuncNameTerminator                      0x00014908   Data           8  goommonitor.o(.constdata)
    KFuncLeavePatternL                       0x00014910   Data           8  goommonitor.o(.constdata)
    KGOOMWatcherThreadName                   0x00014918   Data          20  goommonitor.o(.constdata)
    __PRETTY_FUNCTION__@_Z25GOOMWatcherThreadFunctionPv_0 0x0001492c   Data          45  goommonitor.o(.constdata)
    __PRETTY_FUNCTION__@_Z24CreateGOOMWatcherThreadLv_0 0x00014959   Data          32  goommonitor.o(.constdata)
    __PRETTY_FUNCTION__@_Z11PanicClientRK12RMessagePtr223TGOomMonitorClientPanic_0 0x00014979   Data          64  goommonitor.o(.constdata)
    .constdata$1                             0x00014abc   Data           0  goommonitorplugin.o(.constdata)
    KFuncNameTerminator                      0x00014abc   Data           8  goommonitorplugin.o(.constdata)
    .constdata                               0x00014abc   Section      776  goommonitorplugin.o(.constdata)
    KFuncLeavePatternL                       0x00014ac4   Data           8  goommonitorplugin.o(.constdata)
    __PRETTY_FUNCTION__@_Z20SetGMemoryMonitorTlsP14CMemoryMonitor_0 0x00014acc   Data          44  goommonitorplugin.o(.constdata)
    __PRETTY_FUNCTION__@_Z16MemoryMonitorTlsv_0 0x00014af8   Data          35  goommonitorplugin.o(.constdata)
    __PRETTY_FUNCTION__@_Z22GOomMonitorPluginPanic23TGOomMonitorPluginPanic_0 0x00014b1b   Data          53  goommonitorplugin.o(.constdata)
    KCat@_Z22GOomMonitorPluginPanic23TGOomMonitorPluginPanic_1 0x00014b50   Data          40  goommonitorplugin.o(.constdata)
    __PRETTY_FUNCTION__@_ZN22CGOomMonitorPluginBaseC2Ev_0 0x00014b78   Data          49  goommonitorplugin.o(.constdata)
    __PRETTY_FUNCTION__@_ZN22CGOomMonitorPluginBaseD2Ev_0 0x00014ba9   Data          50  goommonitorplugin.o(.constdata)
    __PRETTY_FUNCTION__@_ZN22CGOomMonitorPluginBase10ConstructLEv_0 0x00014bdb   Data          42  goommonitorplugin.o(.constdata)
    __PRETTY_FUNCTION__@_ZN22CGOomMonitorPluginBase9FsSessionEv_0 0x00014c05   Data          41  goommonitorplugin.o(.constdata)
    __PRETTY_FUNCTION__@_ZN22CGOomMonitorPluginBase9WsSessionEv_0 0x00014c2e   Data          48  goommonitorplugin.o(.constdata)
    __PRETTY_FUNCTION__@_ZN22CGOomMonitorPluginBase18ExtensionInterfaceE4TUidRPv_0 0x00014c5e   Data          63  goommonitorplugin.o(.constdata)
    .constdata$1                             0x00014dc4   Data           0  goommonitorsession.o(.constdata)
    KGraphicsMemoryMonitorServerName         0x00014dc4   Data          40  goommonitorsession.o(.constdata)
    .constdata                               0x00014dc4   Section     1003  goommonitorsession.o(.constdata)
    KFuncNameTerminator                      0x00014dec   Data           8  goommonitorsession.o(.constdata)
    KFuncLeavePatternL                       0x00014df4   Data           8  goommonitorsession.o(.constdata)
    __PRETTY_FUNCTION__@_ZN19RGOomMonitorSession7ConnectEv_0 0x00014dfc   Data          42  goommonitorsession.o(.constdata)
    __PRETTY_FUNCTION__@_ZN19RGOomMonitorSession11IsConnectedEv_0 0x00014e26   Data          39  goommonitorsession.o(.constdata)
    __PRETTY_FUNCTION__@_ZN19RGOomMonitorSession17RequestFreeMemoryEi_0 0x00014e4d   Data          62  goommonitorsession.o(.constdata)
    __PRETTY_FUNCTION__@_ZN19RGOomMonitorSession17RequestFreeMemoryEiR14TRequestStatus_0 0x00014e8b   Data          74  goommonitorsession.o(.constdata)
    __PRETTY_FUNCTION__@_ZN19RGOomMonitorSession18RequestOptionalRamEiiiRi_0 0x00014ed5   Data         101  goommonitorsession.o(.constdata)
    __PRETTY_FUNCTION__@_ZN19RGOomMonitorSession18RequestOptionalRamEiiiR14TRequestStatus_0 0x00014f3a   Data          99  goommonitorsession.o(.constdata)
    __PRETTY_FUNCTION__@_ZN19RGOomMonitorSession23CancelRequestFreeMemoryEv_0 0x00014f9d   Data          52  goommonitorsession.o(.constdata)
    __PRETTY_FUNCTION__@_ZN19RGOomMonitorSession19ThisAppIsNotExitingEi_0 0x00014fd1   Data          58  goommonitorsession.o(.constdata)
    __PRETTY_FUNCTION__@_ZN19RGOomMonitorSession15SetGOomPriorityENS_13TGOomPriorityE_0 0x0001500b   Data          78  goommonitorsession.o(.constdata)
    __PRETTY_FUNCTION__@_ZN19RGOomMonitorSession23ApplicationAboutToStartERK4TUid_0 0x00015059   Data          64  goommonitorsession.o(.constdata)
    __PRETTY_FUNCTION__@_ZN19RGOomMonitorSession22UsesAbsoluteMemTargetsEi_0 0x00015099   Data          54  goommonitorsession.o(.constdata)
    __PRETTY_FUNCTION__@_ZN19RGOomMonitorSession7ConnectER14TRequestStatus_0 0x000150cf   Data          58  goommonitorsession.o(.constdata)
    __PRETTY_FUNCTION__@_ZN19RGOomMonitorSession15AppAboutToStartER14TRequestStatusRK4TUid_0 0x00015109   Data          74  goommonitorsession.o(.constdata)
    .constdata$1                             0x000151b0   Data           0  goompanic.o(.constdata)
    KCat@_Z16GOomMonitorPanic17TGOomMonitorPanic_0 0x000151b0   Data          28  goompanic.o(.constdata)
    .constdata                               0x000151b0   Section       56  goompanic.o(.constdata)
    KParserCat@_Z21GOomConfigParserPanici_0  0x000151cc   Data          28  goompanic.o(.constdata)
    .constdata$1                             0x000151e8   Data           0  goompluginwaiter.o(.constdata)
    KFuncNameTerminator                      0x000151e8   Data           8  goompluginwaiter.o(.constdata)
    .constdata                               0x000151e8   Section      311  goompluginwaiter.o(.constdata)
    KFuncLeavePatternL                       0x000151f0   Data           8  goompluginwaiter.o(.constdata)
    __PRETTY_FUNCTION__@_ZN17CGOomPluginWaiter4NewLEiR14CGOomRunPlugin_0 0x000151f8   Data          73  goompluginwaiter.o(.constdata)
    __PRETTY_FUNCTION__@_ZN17CGOomPluginWaiter5StartEv_0 0x00015241   Data          32  goompluginwaiter.o(.constdata)
    __PRETTY_FUNCTION__@_ZN17CGOomPluginWaiter4RunLEv_0 0x00015261   Data          31  goompluginwaiter.o(.constdata)
    __PRETTY_FUNCTION__@_ZN17CGOomPluginWaiterC1EiR14CGOomRunPlugin_0 0x00015280   Data          67  goompluginwaiter.o(.constdata)
    .constdata$1                             0x00015320   Data           0  goomrunplugin.o(.constdata)
    KFuncNameTerminator                      0x00015320   Data           8  goomrunplugin.o(.constdata)
    .constdata                               0x00015320   Section      768  goomrunplugin.o(.constdata)
    KFuncLeavePatternL                       0x00015328   Data           8  goomrunplugin.o(.constdata)
    __PRETTY_FUNCTION__@_ZN14CGOomRunPlugin4NewLEjR20CGOomRunPluginConfigR19MGOomActionObserverR18CGOomMonitorPlugin_0 0x00015330   Data         120  goomrunplugin.o(.constdata)
    __PRETTY_FUNCTION__@_ZN14CGOomRunPluginD1Ev_0 0x000153a8   Data          34  goomrunplugin.o(.constdata)
    __PRETTY_FUNCTION__@_ZN14CGOomRunPlugin10FreeMemoryEi_0 0x000153ca   Data          44  goomrunplugin.o(.constdata)
    __PRETTY_FUNCTION__@_ZN14CGOomRunPlugin10MemoryGoodEv_0 0x000153f6   Data          34  goomrunplugin.o(.constdata)
    __PRETTY_FUNCTION__@_ZN14CGOomRunPlugin10ConstructLER20CGOomRunPluginConfig_0 0x00015418   Data          56  goomrunplugin.o(.constdata)
    __PRETTY_FUNCTION__@_ZN14CGOomRunPluginC1EjR20CGOomRunPluginConfigR19MGOomActionObserverR18CGOomMonitorPlugin_0 0x00015450   Data         114  goomrunplugin.o(.constdata)
    .constdata$1                             0x00015620   Data           0  goomrunpluginconfig.o(.constdata)
    KFuncNameTerminator                      0x00015620   Data           8  goomrunpluginconfig.o(.constdata)
    .constdata                               0x00015620   Section      399  goomrunpluginconfig.o(.constdata)
    KFuncLeavePatternL                       0x00015628   Data           8  goomrunpluginconfig.o(.constdata)
    __PRETTY_FUNCTION__@_ZN20CGOomRunPluginConfig4NewLEj15TGOomPluginType_0 0x00015630   Data          80  goomrunpluginconfig.o(.constdata)
    __PRETTY_FUNCTION__@_ZN20CGOomRunPluginConfig23CalculatePluginPriorityERK20CGOomWindowGroupList_0 0x00015680   Data          89  goomrunpluginconfig.o(.constdata)
    __PRETTY_FUNCTION__@_ZN20CGOomRunPluginConfigD1Ev_0 0x000156d9   Data          46  goomrunpluginconfig.o(.constdata)
    __PRETTY_FUNCTION__@_ZN20CGOomRunPluginConfigC1Ej15TGOomPluginType_0 0x00015707   Data          74  goomrunpluginconfig.o(.constdata)
    .constdata$1                             0x000157b0   Data           0  goomwindowgrouplist.o(.constdata)
    KFuncNameTerminator                      0x000157b0   Data           8  goomwindowgrouplist.o(.constdata)
    .constdata                               0x000157b0   Section     2388  goomwindowgrouplist.o(.constdata)
    KFuncLeavePatternL                       0x000157b8   Data           8  goomwindowgrouplist.o(.constdata)
    KDummyWgName                             0x000157c0   Data          12  goomwindowgrouplist.o(.constdata)
    __PRETTY_FUNCTION__@_ZN20CGOomWindowGroupList4NewLER10RWsSession_0 0x000157cc   Data          63  goomwindowgrouplist.o(.constdata)
    __PRETTY_FUNCTION__@_ZN20CGOomWindowGroupList8RefreshLEv_0 0x0001580b   Data          38  goomwindowgrouplist.o(.constdata)
    __PRETTY_FUNCTION__@_ZN20CGOomWindowGroupList7RefreshEv_0 0x00015831   Data          37  goomwindowgrouplist.o(.constdata)
    __PRETTY_FUNCTION__@_ZNK20CGOomWindowGroupList5AppIdEii_0 0x00015856   Data          64  goomwindowgrouplist.o(.constdata)
    __PRETTY_FUNCTION__@_ZNK20CGOomWindowGroupList8IdleTimeEi_0 0x00015896   Data          70  goomwindowgrouplist.o(.constdata)
    __PRETTY_FUNCTION__@_ZN20CGOomWindowGroupListD1Ev_0 0x000158dc   Data          46  goomwindowgrouplist.o(.constdata)
    __PRETTY_FUNCTION__@_ZN20CGOomWindowGroupList15SetPriorityBusyEi_0 0x0001590a   Data          55  goomwindowgrouplist.o(.constdata)
    __PRETTY_FUNCTION__@_ZN20CGOomWindowGroupList17SetPriorityNormalEi_0 0x00015941   Data          57  goomwindowgrouplist.o(.constdata)
    __PRETTY_FUNCTION__@_ZN20CGOomWindowGroupList15SetPriorityHighEi_0 0x0001597a   Data          55  goomwindowgrouplist.o(.constdata)
    __PRETTY_FUNCTION__@_ZN20CGOomWindowGroupList21IsDynamicHighPriorityEi_0 0x000159b1   Data          60  goomwindowgrouplist.o(.constdata)
    __PRETTY_FUNCTION__@_ZNK20CGOomWindowGroupList17GetIndexFromAppIdEj_0 0x000159ed   Data          71  goomwindowgrouplist.o(.constdata)
    __PRETTY_FUNCTION__@_ZN20CGOomWindowGroupList23CollapseWindowGroupTreeEv_0 0x00015a34   Data          53  goomwindowgrouplist.o(.constdata)
    __PRETTY_FUNCTION__@_ZN20CGOomWindowGroupList33RemovePropertiesForClosedWindowsLEv_0 0x00015a69   Data          63  goomwindowgrouplist.o(.constdata)
    __PRETTY_FUNCTION__@_ZN20CGOomWindowGroupListC1ER10RWsSession_0 0x00015aa8   Data          57  goomwindowgrouplist.o(.constdata)
    __PRETTY_FUNCTION__@_ZN20CGOomWindowGroupList10ConstructLEv_0 0x00015ae1   Data          40  goomwindowgrouplist.o(.constdata)
    __PRETTY_FUNCTION__@_ZN20CGOomWindowGroupList26TGOomWindowGroupPropertiesC1Ev_0 0x00015b09   Data          79  goomwindowgrouplist.o(.constdata)
    .constdata$1                             0x00016104   Data           0  goomwserveventreceiver.o(.constdata)
    KFuncNameTerminator                      0x00016104   Data           8  goomwserveventreceiver.o(.constdata)
    .constdata                               0x00016104   Section      371  goomwserveventreceiver.o(.constdata)
    KFuncLeavePatternL                       0x0001610c   Data           8  goomwserveventreceiver.o(.constdata)
    KUidFastSwap                             0x00016114   Data           4  goomwserveventreceiver.o(.constdata)
    __PRETTY_FUNCTION__@_ZN19CWservEventReceiverC1ER14CMemoryMonitorR10RWsSession_0 0x00016118   Data          73  goomwserveventreceiver.o(.constdata)
    __PRETTY_FUNCTION__@_ZN19CWservEventReceiverD1Ev_0 0x00016161   Data          44  goomwserveventreceiver.o(.constdata)
    __PRETTY_FUNCTION__@_ZN19CWservEventReceiver10ConstructLEv_0 0x0001618d   Data          39  goomwserveventreceiver.o(.constdata)
    __PRETTY_FUNCTION__@_ZN19CWservEventReceiver5QueueEv_0 0x000161b4   Data          34  goomwserveventreceiver.o(.constdata)
    __PRETTY_FUNCTION__@_ZN19CWservEventReceiver8DoCancelEv_0 0x000161d6   Data          37  goomwserveventreceiver.o(.constdata)
    __PRETTY_FUNCTION__@_ZN19CWservEventReceiver4RunLEv_0 0x000161fb   Data          33  goomwserveventreceiver.o(.constdata)
    .constdata__ZTI11CGOomAction             0x00016278   Section       12  goomaction.o(.constdata__ZTI11CGOomAction)
    .constdata__ZTI11CGOomConfig             0x00016284   Section       12  goomconfig.o(.constdata__ZTI11CGOomConfig)
    .constdata__ZTI11CGOomLogger             0x00016290   Section       12  goomlog.o(.constdata__ZTI11CGOomLogger)
    .constdata__ZTI13CGOomCloseApp           0x0001629c   Section       12  goomcloseapp.o(.constdata__ZTI13CGOomCloseApp)
    .constdata__ZTI14CGOomRunPlugin          0x000162a8   Section       12  goomrunplugin.o(.constdata__ZTI14CGOomRunPlugin)
    .constdata__ZTI14CMemoryMonitor          0x000162b4   Section       12  goommemorymonitor.o(.constdata__ZTI14CMemoryMonitor)
    .constdata__ZTI15CGOomActionList         0x000162c0   Section       32  goomactionlist.o(.constdata__ZTI15CGOomActionList)
    .constdata__ZTI15CGOomPluginListI18CGOomMonitorPluginE 0x000162e0   Section       12  goomactionlist.o(.constdata__ZTI15CGOomPluginListI18CGOomMonitorPluginE)
    .constdata__ZTI15MGOomRuleConfig         0x000162ec   Section        8  goomIdletimerule.o(.constdata__ZTI15MGOomRuleConfig)
    .constdata__ZTI16CSimpleScheduler        0x000162f4   Section       12  goommonitor.o(.constdata__ZTI16CSimpleScheduler)
    .constdata__ZTI17CGOomActionConfig       0x00016300   Section       12  goomactionconfig.o(.constdata__ZTI17CGOomActionConfig)
    .constdata__ZTI17CGOomConfigParser       0x0001630c   Section       32  goomconfigparser.o(.constdata__ZTI17CGOomConfigParser)
    .constdata__ZTI17CGOomGlobalConfig       0x0001632c   Section       12  goomglobalconfig.o(.constdata__ZTI17CGOomGlobalConfig)
    .constdata__ZTI17CGOomIdleTimeRule       0x00016338   Section       32  goomIdletimerule.o(.constdata__ZTI17CGOomIdleTimeRule)
    .constdata__ZTI17CGOomPluginWaiter       0x00016358   Section       12  goompluginwaiter.o(.constdata__ZTI17CGOomPluginWaiter)
    .constdata__ZTI18CGOomAppCloseTimer      0x00016364   Section       12  goomappclosetimer.o(.constdata__ZTI18CGOomAppCloseTimer)
    .constdata__ZTI19CGOomCloseAppConfig     0x00016370   Section       12  goomcloseappconfig.o(.constdata__ZTI19CGOomCloseAppConfig)
    .constdata__ZTI19CGOomForegroundRule     0x0001637c   Section       32  goomforegroundrule.o(.constdata__ZTI19CGOomForegroundRule)
    .constdata__ZTI19CWservEventReceiver     0x0001639c   Section       12  goomwserveventreceiver.o(.constdata__ZTI19CWservEventReceiver)
    .constdata__ZTI19MGOomActionObserver     0x000163a8   Section        8  goomactionlist.o(.constdata__ZTI19MGOomActionObserver)
    .constdata__ZTI20CGOomAppCloseWatcher    0x000163b0   Section       12  goomappclosewatcher.o(.constdata__ZTI20CGOomAppCloseWatcher)
    .constdata__ZTI20CGOomRunPluginConfig    0x000163bc   Section       12  goomrunpluginconfig.o(.constdata__ZTI20CGOomRunPluginConfig)
    .constdata__ZTI20CGOomWindowGroupList    0x000163c8   Section       12  goomwindowgrouplist.o(.constdata__ZTI20CGOomWindowGroupList)
    .constdata__ZTI20CMemoryMonitorServer    0x000163d4   Section       12  goommemorymonitorserver.o(.constdata__ZTI20CMemoryMonitorServer)
    .constdata__ZTI21CAppGOomMonitorPlugin   0x000163e0   Section       12  goommonitorplugin.o(.constdata__ZTI21CAppGOomMonitorPlugin)
    .constdata__ZTI21CGoomThresholdCrossed   0x000163ec   Section       12  goommemorymonitor.o(.constdata__ZTI21CGoomThresholdCrossed)
    .constdata__ZTI21CMemoryMonitorSession   0x000163f8   Section       12  goommemorymonitorsession.o(.constdata__ZTI21CMemoryMonitorSession)
    .constdata__ZTI22CGOomApplicationConfig  0x00016404   Section       12  goomapplicationconfig.o(.constdata__ZTI22CGOomApplicationConfig)
    .constdata__ZTI22CGOomMonitorPluginBase  0x00016410   Section       12  goommonitorplugin.o(.constdata__ZTI22CGOomMonitorPluginBase)
    .constdata__ZTIN3Xml15MContentHandlerE   0x0001641c   Section        8  goomconfigparser.o(.constdata__ZTIN3Xml15MContentHandlerE)
    .constdata__ZTS11CGOomAction             0x00016424   Section       14  goomaction.o(.constdata__ZTS11CGOomAction)
    .constdata__ZTS11CGOomConfig             0x00016432   Section       14  goomconfig.o(.constdata__ZTS11CGOomConfig)
    .constdata__ZTS11CGOomLogger             0x00016440   Section       14  goomlog.o(.constdata__ZTS11CGOomLogger)
    .constdata__ZTS13CGOomCloseApp           0x0001644e   Section       16  goomcloseapp.o(.constdata__ZTS13CGOomCloseApp)
    .constdata__ZTS14CGOomRunPlugin          0x0001645e   Section       17  goomrunplugin.o(.constdata__ZTS14CGOomRunPlugin)
    .constdata__ZTS14CMemoryMonitor          0x0001646f   Section       17  goommemorymonitor.o(.constdata__ZTS14CMemoryMonitor)
    .constdata__ZTS15CGOomActionList         0x00016480   Section       18  goomactionlist.o(.constdata__ZTS15CGOomActionList)
    .constdata__ZTS15CGOomPluginListI18CGOomMonitorPluginE 0x00016492   Section       40  goomactionlist.o(.constdata__ZTS15CGOomPluginListI18CGOomMonitorPluginE)
    .constdata__ZTS15MGOomRuleConfig         0x000164ba   Section       18  goomIdletimerule.o(.constdata__ZTS15MGOomRuleConfig)
    .constdata__ZTS16CSimpleScheduler        0x000164cc   Section       19  goommonitor.o(.constdata__ZTS16CSimpleScheduler)
    .constdata__ZTS17CGOomActionConfig       0x000164df   Section       20  goomactionconfig.o(.constdata__ZTS17CGOomActionConfig)
    .constdata__ZTS17CGOomConfigParser       0x000164f3   Section       20  goomconfigparser.o(.constdata__ZTS17CGOomConfigParser)
    .constdata__ZTS17CGOomGlobalConfig       0x00016507   Section       20  goomglobalconfig.o(.constdata__ZTS17CGOomGlobalConfig)
    .constdata__ZTS17CGOomIdleTimeRule       0x0001651b   Section       20  goomIdletimerule.o(.constdata__ZTS17CGOomIdleTimeRule)
    .constdata__ZTS17CGOomPluginWaiter       0x0001652f   Section       20  goompluginwaiter.o(.constdata__ZTS17CGOomPluginWaiter)
    .constdata__ZTS18CGOomAppCloseTimer      0x00016543   Section       21  goomappclosetimer.o(.constdata__ZTS18CGOomAppCloseTimer)
    .constdata__ZTS19CGOomCloseAppConfig     0x00016558   Section       22  goomcloseappconfig.o(.constdata__ZTS19CGOomCloseAppConfig)
    .constdata__ZTS19CGOomForegroundRule     0x0001656e   Section       22  goomforegroundrule.o(.constdata__ZTS19CGOomForegroundRule)
    .constdata__ZTS19CWservEventReceiver     0x00016584   Section       22  goomwserveventreceiver.o(.constdata__ZTS19CWservEventReceiver)
    .constdata__ZTS19MGOomActionObserver     0x0001659a   Section       22  goomactionlist.o(.constdata__ZTS19MGOomActionObserver)
    .constdata__ZTS20CGOomAppCloseWatcher    0x000165b0   Section       23  goomappclosewatcher.o(.constdata__ZTS20CGOomAppCloseWatcher)
    .constdata__ZTS20CGOomRunPluginConfig    0x000165c7   Section       23  goomrunpluginconfig.o(.constdata__ZTS20CGOomRunPluginConfig)
    .constdata__ZTS20CGOomWindowGroupList    0x000165de   Section       23  goomwindowgrouplist.o(.constdata__ZTS20CGOomWindowGroupList)
    .constdata__ZTS20CMemoryMonitorServer    0x000165f5   Section       23  goommemorymonitorserver.o(.constdata__ZTS20CMemoryMonitorServer)
    .constdata__ZTS21CAppGOomMonitorPlugin   0x0001660c   Section       24  goommonitorplugin.o(.constdata__ZTS21CAppGOomMonitorPlugin)
    .constdata__ZTS21CGoomThresholdCrossed   0x00016624   Section       24  goommemorymonitor.o(.constdata__ZTS21CGoomThresholdCrossed)
    .constdata__ZTS21CMemoryMonitorSession   0x0001663c   Section       24  goommemorymonitorsession.o(.constdata__ZTS21CMemoryMonitorSession)
    .constdata__ZTS22CGOomApplicationConfig  0x00016654   Section       25  goomapplicationconfig.o(.constdata__ZTS22CGOomApplicationConfig)
    .constdata__ZTS22CGOomMonitorPluginBase  0x0001666d   Section       25  goommonitorplugin.o(.constdata__ZTS22CGOomMonitorPluginBase)
    .constdata__ZTSN3Xml15MContentHandlerE   0x00016686   Section       24  goomconfigparser.o(.constdata__ZTSN3Xml15MContentHandlerE)
    .constdata__ZTV11CGOomAction             0x000166a0   Section       28  goomaction.o(.constdata__ZTV11CGOomAction)
    .constdata__ZTV11CGOomConfig             0x000166bc   Section       20  goomconfig.o(.constdata__ZTV11CGOomConfig)
    .constdata__ZTV11CGOomLogger             0x000166d0   Section       32  goomlog.o(.constdata__ZTV11CGOomLogger)
    .constdata__ZTV13CGOomCloseApp           0x000166f0   Section       28  goomcloseapp.o(.constdata__ZTV13CGOomCloseApp)
    .constdata__ZTV14CGOomRunPlugin          0x0001670c   Section       28  goomrunplugin.o(.constdata__ZTV14CGOomRunPlugin)
    .constdata__ZTV14CMemoryMonitor          0x00016728   Section       20  goommemorymonitor.o(.constdata__ZTV14CMemoryMonitor)
    .constdata__ZTV15CGOomActionList         0x0001673c   Section       44  goomactionlist.o(.constdata__ZTV15CGOomActionList)
    .constdata__ZTV15CGOomPluginListI18CGOomMonitorPluginE 0x00016768   Section       20  goomactionlist.o(.constdata__ZTV15CGOomPluginListI18CGOomMonitorPluginE)
    .constdata__ZTV15MGOomRuleConfig         0x0001677c   Section       16  goomIdletimerule.o(.constdata__ZTV15MGOomRuleConfig)
    .constdata__ZTV16CSimpleScheduler        0x0001678c   Section       44  goommonitor.o(.constdata__ZTV16CSimpleScheduler)
    .constdata__ZTV17CGOomActionConfig       0x000167b8   Section       20  goomactionconfig.o(.constdata__ZTV17CGOomActionConfig)
    .constdata__ZTV17CGOomConfigParser       0x000167cc   Section      124  goomconfigparser.o(.constdata__ZTV17CGOomConfigParser)
    .constdata__ZTV17CGOomGlobalConfig       0x00016848   Section       20  goomglobalconfig.o(.constdata__ZTV17CGOomGlobalConfig)
    .constdata__ZTV17CGOomIdleTimeRule       0x0001685c   Section       44  goomIdletimerule.o(.constdata__ZTV17CGOomIdleTimeRule)
    .constdata__ZTV17CGOomPluginWaiter       0x00016888   Section       32  goompluginwaiter.o(.constdata__ZTV17CGOomPluginWaiter)
    .constdata__ZTV18CGOomAppCloseTimer      0x000168a8   Section       32  goomappclosetimer.o(.constdata__ZTV18CGOomAppCloseTimer)
    .constdata__ZTV19CGOomCloseAppConfig     0x000168c8   Section       20  goomcloseappconfig.o(.constdata__ZTV19CGOomCloseAppConfig)
    .constdata__ZTV19CGOomForegroundRule     0x000168dc   Section       44  goomforegroundrule.o(.constdata__ZTV19CGOomForegroundRule)
    .constdata__ZTV19CWservEventReceiver     0x00016908   Section       32  goomwserveventreceiver.o(.constdata__ZTV19CWservEventReceiver)
    .constdata__ZTV19MGOomActionObserver     0x00016928   Section       16  goomactionlist.o(.constdata__ZTV19MGOomActionObserver)
    .constdata__ZTV20CGOomAppCloseWatcher    0x00016938   Section       32  goomappclosewatcher.o(.constdata__ZTV20CGOomAppCloseWatcher)
    .constdata__ZTV20CGOomRunPluginConfig    0x00016958   Section       20  goomrunpluginconfig.o(.constdata__ZTV20CGOomRunPluginConfig)
    .constdata__ZTV20CGOomWindowGroupList    0x0001696c   Section       20  goomwindowgrouplist.o(.constdata__ZTV20CGOomWindowGroupList)
    .constdata__ZTV20CMemoryMonitorServer    0x00016980   Section       40  goommemorymonitorserver.o(.constdata__ZTV20CMemoryMonitorServer)
    .constdata__ZTV21CAppGOomMonitorPlugin   0x000169a8   Section       32  goommonitorplugin.o(.constdata__ZTV21CAppGOomMonitorPlugin)
    .constdata__ZTV21CGoomThresholdCrossed   0x000169c8   Section       32  goommemorymonitor.o(.constdata__ZTV21CGoomThresholdCrossed)
    .constdata__ZTV21CMemoryMonitorSession   0x000169e8   Section       40  goommemorymonitorsession.o(.constdata__ZTV21CMemoryMonitorSession)
    .constdata__ZTV22CGOomApplicationConfig  0x00016a10   Section       20  goomapplicationconfig.o(.constdata__ZTV22CGOomApplicationConfig)
    .constdata__ZTV22CGOomMonitorPluginBase  0x00016a24   Section       32  goommonitorplugin.o(.constdata__ZTV22CGOomMonitorPluginBase)
    .constdata__ZTVN3Xml15MContentHandlerE   0x00016a44   Section       56  goomconfigparser.o(.constdata__ZTVN3Xml15MContentHandlerE)
    .constdata__ZZN21CGoomThresholdCrossed10ThreadNameEvE19__PRETTY_FUNCTION__ 0x00016a7c   Section       51  goommemorymonitor.o(.constdata__ZZN21CGoomThresholdCrossed10ThreadNameEvE19__PRETTY_FUNCTION__)
    .constdata__ZZN21CGoomThresholdCrossed12SetThresholdEiE19__PRETTY_FUNCTION__ 0x00016aaf   Section       53  goommemorymonitor.o(.constdata__ZZN21CGoomThresholdCrossed12SetThresholdEiE19__PRETTY_FUNCTION__)
    .constdata__ZZN21CGoomThresholdCrossed15ResetThresholdsEvE19__PRETTY_FUNCTION__ 0x00016ae4   Section       46  goommemorymonitor.o(.constdata__ZZN21CGoomThresholdCrossed15ResetThresholdsEvE19__PRETTY_FUNCTION__)
    .constdata__ZZN21CGoomThresholdCrossed18StartRequestEventsEvE19__PRETTY_FUNCTION__ 0x00016b12   Section       49  goommemorymonitor.o(.constdata__ZZN21CGoomThresholdCrossed18StartRequestEventsEvE19__PRETTY_FUNCTION__)
    .constdata__ZZN21CGoomThresholdCrossed20RequestNotificationsEiE19__PRETTY_FUNCTION__ 0x00016b43   Section       54  goommemorymonitor.o(.constdata__ZZN21CGoomThresholdCrossed20RequestNotificationsEiE19__PRETTY_FUNCTION__)
    .constdata__ZZN21CGoomThresholdCrossed4RunLEvE19__PRETTY_FUNCTION__ 0x00016b79   Section       35  goommemorymonitor.o(.constdata__ZZN21CGoomThresholdCrossed4RunLEvE19__PRETTY_FUNCTION__)
    .constdata__ZZN21CGoomThresholdCrossed6CancelEvE19__PRETTY_FUNCTION__ 0x00016b9c   Section       37  goommemorymonitor.o(.constdata__ZZN21CGoomThresholdCrossed6CancelEvE19__PRETTY_FUNCTION__)
    .constdata__ZZN21CGoomThresholdCrossed7TriggerEiE19__PRETTY_FUNCTION__ 0x00016bc1   Section       48  goommemorymonitor.o(.constdata__ZZN21CGoomThresholdCrossed7TriggerEiE19__PRETTY_FUNCTION__)
    .constdata__ZZN21CGoomThresholdCrossed8DoCancelEvE19__PRETTY_FUNCTION__ 0x00016bf1   Section       39  goommemorymonitor.o(.constdata__ZZN21CGoomThresholdCrossed8DoCancelEvE19__PRETTY_FUNCTION__)
    .constdata__ZZN21CGoomThresholdCrossedC1ER14CMemoryMonitorjiE19__PRETTY_FUNCTION__ 0x00016c18   Section       89  goommemorymonitor.o(.constdata__ZZN21CGoomThresholdCrossedC1ER14CMemoryMonitorjiE19__PRETTY_FUNCTION__)
    .constdata__ZZN21CGoomThresholdCrossedD1EvE19__PRETTY_FUNCTION__ 0x00016c71   Section       48  goommemorymonitor.o(.constdata__ZZN21CGoomThresholdCrossedD1EvE19__PRETTY_FUNCTION__)
    .constdata___ARM__ZN21CGoomThresholdCrossed18StartRequestEventsEv_anon0 0x00016ca4   Section       20  goommemorymonitor.o(.constdata___ARM__ZN21CGoomThresholdCrossed18StartRequestEventsEv_anon0)
    __ARM_d__ZN15CGOomPluginListI18CGOomMonitorPluginE10ConstructLEi$21 0x00016cb8   Data           0  goomactionlist.o(__ARM_d__ZN15CGOomPluginListI18CGOomMonitorPluginE10ConstructLEi)
    __PRETTY_FUNCTION__@_ZN15CGOomPluginListI18CGOomMonitorPluginE10ConstructLEi_0 0x00016cb8   Data          78  goomactionlist.o(__ARM_d__ZN15CGOomPluginListI18CGOomMonitorPluginE10ConstructLEi)
    __ARM_d__ZN15CGOomPluginListI18CGOomMonitorPluginE10ConstructLEi 0x00016cb8   Section       78  goomactionlist.o(__ARM_d__ZN15CGOomPluginListI18CGOomMonitorPluginE10ConstructLEi)
    __ARM_d__ZN15CGOomPluginListI18CGOomMonitorPluginE4NewLEi$12 0x00016d06   Data           0  goomactionlist.o(__ARM_d__ZN15CGOomPluginListI18CGOomMonitorPluginE4NewLEi)
    __PRETTY_FUNCTION__@_ZN15CGOomPluginListI18CGOomMonitorPluginE4NewLEi_0 0x00016d06   Data          87  goomactionlist.o(__ARM_d__ZN15CGOomPluginListI18CGOomMonitorPluginE4NewLEi)
    __ARM_d__ZN15CGOomPluginListI18CGOomMonitorPluginE4NewLEi 0x00016d06   Section       87  goomactionlist.o(__ARM_d__ZN15CGOomPluginListI18CGOomMonitorPluginE4NewLEi)
    __ARM_d__ZN15CGOomPluginListI18CGOomMonitorPluginE7TPluginC1Ev$24 0x00016d5d   Data           0  goomactionlist.o(__ARM_d__ZN15CGOomPluginListI18CGOomMonitorPluginE7TPluginC1Ev)
    __PRETTY_FUNCTION__@_ZN15CGOomPluginListI18CGOomMonitorPluginE7TPluginC1Ev_0 0x00016d5d   Data          69  goomactionlist.o(__ARM_d__ZN15CGOomPluginListI18CGOomMonitorPluginE7TPluginC1Ev)
    __ARM_d__ZN15CGOomPluginListI18CGOomMonitorPluginE7TPluginC1Ev 0x00016d5d   Section       69  goomactionlist.o(__ARM_d__ZN15CGOomPluginListI18CGOomMonitorPluginE7TPluginC1Ev)
    __ARM_d__ZN15CGOomPluginListI18CGOomMonitorPluginEC1Ev$18 0x00016da2   Data           0  goomactionlist.o(__ARM_d__ZN15CGOomPluginListI18CGOomMonitorPluginEC1Ev)
    __PRETTY_FUNCTION__@_ZN15CGOomPluginListI18CGOomMonitorPluginEC1Ev_0 0x00016da2   Data          68  goomactionlist.o(__ARM_d__ZN15CGOomPluginListI18CGOomMonitorPluginEC1Ev)
    __ARM_d__ZN15CGOomPluginListI18CGOomMonitorPluginEC1Ev 0x00016da2   Section       68  goomactionlist.o(__ARM_d__ZN15CGOomPluginListI18CGOomMonitorPluginEC1Ev)
    __ARM_d__ZN15CGOomPluginListI18CGOomMonitorPluginED1Ev$15 0x00016de6   Data           0  goomactionlist.o(__ARM_d__ZN15CGOomPluginListI18CGOomMonitorPluginED1Ev)
    __PRETTY_FUNCTION__@_ZN15CGOomPluginListI18CGOomMonitorPluginED1Ev_0 0x00016de6   Data          69  goomactionlist.o(__ARM_d__ZN15CGOomPluginListI18CGOomMonitorPluginED1Ev)
    __ARM_d__ZN15CGOomPluginListI18CGOomMonitorPluginED1Ev 0x00016de6   Section       69  goomactionlist.o(__ARM_d__ZN15CGOomPluginListI18CGOomMonitorPluginED1Ev)
    .ARM.exidx                               0x00016e2c   Section        8  ucppinit.o(.ARM.exidx)

    Global Symbols

    Symbol Name                              Value     Ov Type        Size  Object(Section)

    BuildAttributes$$THUMB_ISAv2$ARM_ISAv5$M$PE$A:L22$X:L11$S22$IEEE1$IW$USESV6$~STKCKD$USESV7$~SHL$OSPACE$ROPI$IEEEJ$EBA8$UX$FPIC$INDIRECT$REQ8$PRES8$EABIv2 0x00000000   Number         0  anon$$obj.o ABSOLUTE
    apgrfx{000a0000}[10003a3c].dll           0x00000000   Data           0  anon$$obj.o ABSOLUTE
    bafl{000a0000}[10003a0f].dll             0x00000000   Data           0  anon$$obj.o ABSOLUTE
    cone{000a0000}[10003a41].dll             0x00000000   Data           0  anon$$obj.o ABSOLUTE
    drtaeabi{000a0000}.dll                   0x00000000   Data           0  anon$$obj.o ABSOLUTE
    drtrvct2_2{000a0000}.dll                 0x00000000   Data           0  anon$$obj.o ABSOLUTE
    ecom{000a0000}[10009d8e].dll             0x00000000   Data           0  anon$$obj.o ABSOLUTE
    efsrv{000a0000}[100039e4].dll            0x00000000   Data           0  anon$$obj.o ABSOLUTE
    euser{000a0000}[100039e5].dll            0x00000000   Data           0  anon$$obj.o ABSOLUTE
    goommonitor{000a0000}[10282dbf].dll      0x00000000   Data           0  anon$$obj.o ABSOLUTE
    libEGL{000a0000}.dll                     0x00000000   Data           0  anon$$obj.o ABSOLUTE
    libc{00010000}[10207369].dll             0x00000000   Data           0  anon$$obj.o ABSOLUTE
    scppnwdl{000a0000}.dll                   0x00000000   Data           0  anon$$obj.o ABSOLUTE
    ws32{000a0000}[10003b21].dll             0x00000000   Data           0  anon$$obj.o ABSOLUTE
    xmlframework{000a0000}[101fadcc].dll     0x00000000   Data           0  anon$$obj.o ABSOLUTE
    SHT$$INIT_ARRAY$$Base                     - Undefined Weak Reference
    SHT$$INIT_ARRAY$$Limit                    - Undefined Weak Reference
    RArrayBase::Close()                       - Undefined Reference
    _ZN10RArrayBase5CloseEv@euser{000a0000}[100039e5].dll  - Undefined Reference
    RArrayBase::Reset()                       - Undefined Reference
    _ZN10RArrayBase5ResetEv@euser{000a0000}[100039e5].dll  - Undefined Reference
    RArrayBase::Append(const void*)           - Undefined Reference
    _ZN10RArrayBase6AppendEPKv@euser{000a0000}[100039e5].dll  - Undefined Reference
    RArrayBase::Remove(int)                   - Undefined Reference
    _ZN10RArrayBase6RemoveEi@euser{000a0000}[100039e5].dll  - Undefined Reference
    RArrayBase::DoReserve(int)                - Undefined Reference
    _ZN10RArrayBase9DoReserveEi@euser{000a0000}[100039e5].dll  - Undefined Reference
    RArrayBase::InsertIsq(const void*, int(*)(const void*, const void*), int)  - Undefined Reference
    _ZN10RArrayBase9InsertIsqEPKvPFiS1_S1_Ei@euser{000a0000}[100039e5].dll  - Undefined Reference
    RArrayBase::RArrayBase(int)               - Undefined Reference
    _ZN10RArrayBaseC1Ei@euser{000a0000}[100039e5].dll  - Undefined Reference
    RWsSession::EventReady(TRequestStatus*)   - Undefined Reference
    _ZN10RWsSession10EventReadyEP14TRequestStatus@ws32{000a0000}[10003b21].dll  - Undefined Reference
    RWsSession::ComputeMode(RWsSession::TComputeMode)  - Undefined Reference
    _ZN10RWsSession11ComputeModeENS_12TComputeModeE@ws32{000a0000}[10003b21].dll  - Undefined Reference
    RWsSession::EventReadyCancel()            - Undefined Reference
    _ZN10RWsSession16EventReadyCancelEv@ws32{000a0000}[10003b21].dll  - Undefined Reference
    RWsSession::SendEventToWindowGroup(int, const TWsEvent&)  - Undefined Reference
    _ZN10RWsSession22SendEventToWindowGroupEiRK8TWsEvent@ws32{000a0000}[10003b21].dll  - Undefined Reference
    RWsSession::Close()                       - Undefined Reference
    _ZN10RWsSession5CloseEv@ws32{000a0000}[10003b21].dll  - Undefined Reference
    RWsSession::Connect()                     - Undefined Reference
    _ZN10RWsSession7ConnectEv@ws32{000a0000}[10003b21].dll  - Undefined Reference
    RWsSession::RWsSession()                  - Undefined Reference
    _ZN10RWsSessionC1Ev@ws32{000a0000}[10003b21].dll  - Undefined Reference
    TBufBase16::TBufBase16(int)               - Undefined Reference
    _ZN10TBufBase16C1Ei@euser{000a0000}[100039e5].dll  - Undefined Reference
    DefaultHash::Integer(const int&)          - Undefined Reference
    _ZN11DefaultHash7IntegerERKi@euser{000a0000}[100039e5].dll  - Undefined Reference
    RHandleBase::Close()                      - Undefined Reference
    _ZN11RHandleBase5CloseEv@euser{000a0000}[100039e5].dll  - Undefined Reference
    CTrapCleanup::New()                       - Undefined Reference
    _ZN12CTrapCleanup3NewEv@euser{000a0000}[100039e5].dll  - Undefined Reference
    CleanupStack::PopAndDestroy(int)          - Undefined Reference
    _ZN12CleanupStack13PopAndDestroyEi@euser{000a0000}[100039e5].dll  - Undefined Reference
    CleanupStack::PopAndDestroy()             - Undefined Reference
    _ZN12CleanupStack13PopAndDestroyEv@euser{000a0000}[100039e5].dll  - Undefined Reference
    CleanupStack::Pop()                       - Undefined Reference
    _ZN12CleanupStack3PopEv@euser{000a0000}[100039e5].dll  - Undefined Reference
    CleanupStack::Check(void*)                - Undefined Reference
    _ZN12CleanupStack5CheckEPv@euser{000a0000}[100039e5].dll  - Undefined Reference
    CleanupStack::PushL(TCleanupItem)         - Undefined Reference
    _ZN12CleanupStack5PushLE12TCleanupItem@euser{000a0000}[100039e5].dll  - Undefined Reference
    CleanupStack::PushL(CBase*)               - Undefined Reference
    _ZN12CleanupStack5PushLEP5CBase@euser{000a0000}[100039e5].dll  - Undefined Reference
    REComSession::ListImplementationsL(TUid, RPointerArray<CImplementationInformation>&)  - Undefined Reference
    _ZN12REComSession20ListImplementationsLE4TUidR13RPointerArrayI26CImplementationInformationE@ecom{000a0000}[10009d8e].dll  - Undefined Reference
    REComSession::CreateImplementationL(TUid, TUid&, void*)  - Undefined Reference
    _ZN12REComSession21CreateImplementationLE4TUidRS0_Pv@ecom{000a0000}[10009d8e].dll  - Undefined Reference
    REComSession::DestroyedImplementation(TUid)  - Undefined Reference
    _ZN12REComSession23DestroyedImplementationE4TUid@ecom{000a0000}[10009d8e].dll  - Undefined Reference
    RSessionBase::CreateSession(const TDesC16&, const TVersion&, int, TIpcSessionType, const TSecurityPolicy*, TRequestStatus*)  - Undefined Reference
    _ZN12RSessionBase13CreateSessionERK7TDesC16RK8TVersioni15TIpcSessionTypePK15TSecurityPolicyP14TRequestStatus@euser{000a0000}[100039e5].dll  - Undefined Reference
    RWindowGroup::AutoForeground(int)         - Undefined Reference
    _ZN12RWindowGroup14AutoForegroundEi@ws32{000a0000}[10003b21].dll  - Undefined Reference
    RWindowGroup::EnableReceiptOfFocus(int)   - Undefined Reference
    _ZN12RWindowGroup20EnableReceiptOfFocusEi@ws32{000a0000}[10003b21].dll  - Undefined Reference
    RWindowGroup::Construct(unsigned long, int)  - Undefined Reference
    _ZN12RWindowGroup9ConstructEmi@ws32{000a0000}[10003b21].dll  - Undefined Reference
    RWindowGroup::RWindowGroup(RWsSession&)   - Undefined Reference
    _ZN12RWindowGroupC1ER10RWsSession@ws32{000a0000}[10003b21].dll  - Undefined Reference
    RHashTableBase::ValueInsertL(const void*, int, const void*, int, int)  - Undefined Reference
    _ZN14RHashTableBase12ValueInsertLEPKviS1_ii@euser{000a0000}[100039e5].dll  - Undefined Reference
    RHashTableBase::Close()                   - Undefined Reference
    _ZN14RHashTableBase5CloseEv@euser{000a0000}[100039e5].dll  - Undefined Reference
    RHashTableBase::ReserveL(int)             - Undefined Reference
    _ZN14RHashTableBase8ReserveLEi@euser{000a0000}[100039e5].dll  - Undefined Reference
    RHashTableBase::RHashTableBase(unsigned long(*)(const void*), int(*)(const void*, const void*), int, int)  - Undefined Reference
    _ZN14RHashTableBaseC1EPFmPKvEPFiS1_S1_Eii@euser{000a0000}[100039e5].dll  - Undefined Reference
    DefaultIdentity::Integer(const int&, const int&)  - Undefined Reference
    _ZN15DefaultIdentity7IntegerERKiS1_@euser{000a0000}[100039e5].dll  - Undefined Reference
    RWindowTreeNode::SetOrdinalPosition(int, int)  - Undefined Reference
    _ZN15RWindowTreeNode18SetOrdinalPositionEii@ws32{000a0000}[10003b21].dll  - Undefined Reference
    RWindowTreeNode::EnableFocusChangeEvents()  - Undefined Reference
    _ZN15RWindowTreeNode23EnableFocusChangeEventsEv@ws32{000a0000}[10003b21].dll  - Undefined Reference
    RWindowTreeNode::Close()                  - Undefined Reference
    _ZN15RWindowTreeNode5CloseEv@ws32{000a0000}[10003b21].dll  - Undefined Reference
    TDblQueIterBase::SetToFirst()             - Undefined Reference
    _ZN15TDblQueIterBase10SetToFirstEv@euser{000a0000}[100039e5].dll  - Undefined Reference
    TDblQueIterBase::DoPostInc()              - Undefined Reference
    _ZN15TDblQueIterBase9DoPostIncEv@euser{000a0000}[100039e5].dll  - Undefined Reference
    CActiveScheduler::Extension_(unsigned, void*&, void*)  - Undefined Reference
    _ZN16CActiveScheduler10Extension_EjRPvS0_@euser{000a0000}[100039e5].dll  - Undefined Reference
    CActiveScheduler::OnStarting()            - Undefined Reference
    _ZN16CActiveScheduler10OnStartingEv@euser{000a0000}[100039e5].dll  - Undefined Reference
    CActiveScheduler::OnStopping()            - Undefined Reference
    _ZN16CActiveScheduler10OnStoppingEv@euser{000a0000}[100039e5].dll  - Undefined Reference
    CActiveScheduler::Reserved_1()            - Undefined Reference
    _ZN16CActiveScheduler10Reserved_1Ev@euser{000a0000}[100039e5].dll  - Undefined Reference
    CActiveScheduler::Reserved_2()            - Undefined Reference
    _ZN16CActiveScheduler10Reserved_2Ev@euser{000a0000}[100039e5].dll  - Undefined Reference
    CActiveScheduler::WaitForAnyRequest()     - Undefined Reference
    _ZN16CActiveScheduler17WaitForAnyRequestEv@euser{000a0000}[100039e5].dll  - Undefined Reference
    CActiveScheduler::Add(CActive*)           - Undefined Reference
    _ZN16CActiveScheduler3AddEP7CActive@euser{000a0000}[100039e5].dll  - Undefined Reference
    CActiveScheduler::Start()                 - Undefined Reference
    _ZN16CActiveScheduler5StartEv@euser{000a0000}[100039e5].dll  - Undefined Reference
    CActiveScheduler::Install(CActiveScheduler*)  - Undefined Reference
    _ZN16CActiveScheduler7InstallEPS_@euser{000a0000}[100039e5].dll  - Undefined Reference
    CActiveScheduler::CActiveScheduler()      - Undefined Reference
    _ZN16CActiveSchedulerC1Ev@euser{000a0000}[100039e5].dll  - Undefined Reference
    CActiveScheduler::~CActiveScheduler()     - Undefined Reference
    _ZN16CActiveSchedulerD1Ev@euser{000a0000}[100039e5].dll  - Undefined Reference
    RCriticalSection::CreateLocal(TOwnerType)  - Undefined Reference
    _ZN16RCriticalSection11CreateLocalE10TOwnerType@euser{000a0000}[100039e5].dll  - Undefined Reference
    RCriticalSection::Wait()                  - Undefined Reference
    _ZN16RCriticalSection4WaitEv@euser{000a0000}[100039e5].dll  - Undefined Reference
    RCriticalSection::Close()                 - Undefined Reference
    _ZN16RCriticalSection5CloseEv@euser{000a0000}[100039e5].dll  - Undefined Reference
    RCriticalSection::Signal()                - Undefined Reference
    _ZN16RCriticalSection6SignalEv@euser{000a0000}[100039e5].dll  - Undefined Reference
    RCriticalSection::RCriticalSection()      - Undefined Reference
    _ZN16RCriticalSectionC1Ev@euser{000a0000}[100039e5].dll  - Undefined Reference
    RPointerArrayBase::Close()                - Undefined Reference
    _ZN17RPointerArrayBase5CloseEv@euser{000a0000}[100039e5].dll  - Undefined Reference
    RPointerArrayBase::Reset()                - Undefined Reference
    _ZN17RPointerArrayBase5ResetEv@euser{000a0000}[100039e5].dll  - Undefined Reference
    RPointerArrayBase::Append(const void*)    - Undefined Reference
    _ZN17RPointerArrayBase6AppendEPKv@euser{000a0000}[100039e5].dll  - Undefined Reference
    RPointerArrayBase::RPointerArrayBase()    - Undefined Reference
    _ZN17RPointerArrayBaseC1Ev@euser{000a0000}[100039e5].dll  - Undefined Reference
    THashTableIterBase::RemoveCurrent()       - Undefined Reference
    _ZN18THashTableIterBase13RemoveCurrentEv@euser{000a0000}[100039e5].dll  - Undefined Reference
    THashTableIterBase::Next(int)             - Undefined Reference
    _ZN18THashTableIterBase4NextEi@euser{000a0000}[100039e5].dll  - Undefined Reference
    THashTableIterBase::THashTableIterBase(const RHashTableBase&)  - Undefined Reference
    _ZN18THashTableIterBaseC1ERK14RHashTableBase@euser{000a0000}[100039e5].dll  - Undefined Reference
    CApaWindowGroupName::FindByAppUid(TUid, RWsSession&, int&)  - Undefined Reference
    _ZN19CApaWindowGroupName12FindByAppUidE4TUidR10RWsSessionRi@apgrfx{000a0000}[10003a3c].dll  - Undefined Reference
    CApaWindowGroupName::SetWindowGroupName(HBufC16*)  - Undefined Reference
    _ZN19CApaWindowGroupName18SetWindowGroupNameEP7HBufC16@apgrfx{000a0000}[10003a3c].dll  - Undefined Reference
    CApaWindowGroupName::NewL(const RWsSession&)  - Undefined Reference
    _ZN19CApaWindowGroupName4NewLERK10RWsSession@apgrfx{000a0000}[10003a3c].dll  - Undefined Reference
    CApaWindowGroupName::NewLC(const RWsSession&, int)  - Undefined Reference
    _ZN19CApaWindowGroupName5NewLCERK10RWsSessioni@apgrfx{000a0000}[10003a3c].dll  - Undefined Reference
    RFs::GetSystemDriveChar()                 - Undefined Reference
    _ZN3RFs18GetSystemDriveCharEv@efsrv{000a0000}[100039e4].dll  - Undefined Reference
    RFs::Close()                              - Undefined Reference
    _ZN3RFs5CloseEv@efsrv{000a0000}[100039e4].dll  - Undefined Reference
    RFs::Connect(int)                         - Undefined Reference
    _ZN3RFs7ConnectEi@efsrv{000a0000}[100039e4].dll  - Undefined Reference
    Xml::CParser::NewLC(const TDesC8&, Xml::MContentHandler&)  - Undefined Reference
    _ZN3Xml7CParser5NewLCERK6TDesC8RNS_15MContentHandlerE@xmlframework{000a0000}[101fadcc].dll  - Undefined Reference
    Xml::CParser::ParseL(const TDesC8&)       - Undefined Reference
    _ZN3Xml7CParser6ParseLERK6TDesC8@xmlframework{000a0000}[101fadcc].dll  - Undefined Reference
    User::NTickCount()                        - Undefined Reference
    _ZN4User10NTickCountEv@euser{000a0000}[100039e5].dll  - Undefined Reference
    User::LeaveIfError(int)                   - Undefined Reference
    _ZN4User12LeaveIfErrorEi@euser{000a0000}[100039e5].dll  - Undefined Reference
    User::RenameThread(const TDesC16&)        - Undefined Reference
    _ZN4User12RenameThreadERK7TDesC16@euser{000a0000}[100039e5].dll  - Undefined Reference
    User::RequestComplete(TRequestStatus*&, int)  - Undefined Reference
    _ZN4User15RequestCompleteERP14TRequestStatusi@euser{000a0000}[100039e5].dll  - Undefined Reference
    User::MarkCleanupStack()                  - Undefined Reference
    _ZN4User16MarkCleanupStackEv@euser{000a0000}[100039e5].dll  - Undefined Reference
    User::UnMarkCleanupStack(TTrapHandler*)   - Undefined Reference
    _ZN4User18UnMarkCleanupStackEP12TTrapHandler@euser{000a0000}[100039e5].dll  - Undefined Reference
    User::Free(void*)                         - Undefined Reference
    _ZN4User4FreeEPv@euser{000a0000}[100039e5].dll  - Undefined Reference
    User::After(TTimeIntervalMicroSeconds32)  - Undefined Reference
    _ZN4User5AfterE27TTimeIntervalMicroSeconds32@euser{000a0000}[100039e5].dll  - Undefined Reference
    User::Alloc(int)                          - Undefined Reference
    _ZN4User5AllocEi@euser{000a0000}[100039e5].dll  - Undefined Reference
    User::Leave(int)                          - Undefined Reference
    _ZN4User5LeaveEi@euser{000a0000}[100039e5].dll  - Undefined Reference
    User::Panic(const TDesC16&, int)          - Undefined Reference
    _ZN4User5PanicERK7TDesC16i@euser{000a0000}[100039e5].dll  - Undefined Reference
    User::AllocZ(int)                         - Undefined Reference
    _ZN4User6AllocZEi@euser{000a0000}[100039e5].dll  - Undefined Reference
    User::AllocZL(int)                        - Undefined Reference
    _ZN4User7AllocZLEi@euser{000a0000}[100039e5].dll  - Undefined Reference
    User::Invariant()                         - Undefined Reference
    _ZN4User9InvariantEv@euser{000a0000}[100039e5].dll  - Undefined Reference
    CBase::Extension_(unsigned, void*&, void*)  - Undefined Reference
    _ZN5CBase10Extension_EjRPvS0_@euser{000a0000}[100039e5].dll  - Undefined Reference
    CBase::~CBase()                           - Undefined Reference
    _ZN5CBaseD1Ev@euser{000a0000}[100039e5].dll  - Undefined Reference
    RFile::Open(RFs&, const TDesC16&, unsigned)  - Undefined Reference
    _ZN5RFile4OpenER3RFsRK7TDesC16j@efsrv{000a0000}[100039e4].dll  - Undefined Reference
    RFile::Close()                            - Undefined Reference
    _ZN5RFile5CloseEv@efsrv{000a0000}[100039e4].dll  - Undefined Reference
    RFile::Write(const TDesC8&)               - Undefined Reference
    _ZN5RFile5WriteERK6TDesC8@efsrv{000a0000}[100039e4].dll  - Undefined Reference
    RFile::Create(RFs&, const TDesC16&, unsigned)  - Undefined Reference
    _ZN5RFile6CreateER3RFsRK7TDesC16j@efsrv{000a0000}[100039e4].dll  - Undefined Reference
    TDes8::AppendFormat(TRefByValue<const TDesC8>, ...)  - Undefined Reference
    _ZN5TDes812AppendFormatE11TRefByValueIK6TDesC8Ez@euser{000a0000}[100039e5].dll  - Undefined Reference
    TDes8::Copy(const TDesC8&)                - Undefined Reference
    _ZN5TDes84CopyERK6TDesC8@euser{000a0000}[100039e5].dll  - Undefined Reference
    TDes8::Copy(const TDesC16&)               - Undefined Reference
    _ZN5TDes84CopyERK7TDesC16@euser{000a0000}[100039e5].dll  - Undefined Reference
    TDes8::Zero()                             - Undefined Reference
    _ZN5TDes84ZeroEv@euser{000a0000}[100039e5].dll  - Undefined Reference
    TDes8::Append(const TDesC8&)              - Undefined Reference
    _ZN5TDes86AppendERK6TDesC8@euser{000a0000}[100039e5].dll  - Undefined Reference
    TLex8::Val(unsigned long&, TRadix)        - Undefined Reference
    _ZN5TLex83ValERm6TRadix@euser{000a0000}[100039e5].dll  - Undefined Reference
    TLex8::Assign(const TDesC8&)              - Undefined Reference
    _ZN5TLex86AssignERK6TDesC8@euser{000a0000}[100039e5].dll  - Undefined Reference
    TTime::UniversalTime()                    - Undefined Reference
    _ZN5TTime13UniversalTimeEv@euser{000a0000}[100039e5].dll  - Undefined Reference
    TTime::HomeTime()                         - Undefined Reference
    _ZN5TTime8HomeTimeEv@euser{000a0000}[100039e5].dll  - Undefined Reference
    CTimer::ConstructL()                      - Undefined Reference
    _ZN6CTimer10ConstructLEv@euser{000a0000}[100039e5].dll  - Undefined Reference
    CTimer::After(TTimeIntervalMicroSeconds32)  - Undefined Reference
    _ZN6CTimer5AfterE27TTimeIntervalMicroSeconds32@euser{000a0000}[100039e5].dll  - Undefined Reference
    CTimer::HighRes(TTimeIntervalMicroSeconds32)  - Undefined Reference
    _ZN6CTimer7HighResE27TTimeIntervalMicroSeconds32@euser{000a0000}[100039e5].dll  - Undefined Reference
    CTimer::DoCancel()                        - Undefined Reference
    _ZN6CTimer8DoCancelEv@euser{000a0000}[100039e5].dll  - Undefined Reference
    CTimer::CTimer__sub_object(int)           - Undefined Reference
    _ZN6CTimerC2Ei@euser{000a0000}[100039e5].dll  - Undefined Reference
    CTimer::~CTimer__sub_object()             - Undefined Reference
    _ZN6CTimerD2Ev@euser{000a0000}[100039e5].dll  - Undefined Reference
    RDebug::Print(TRefByValue<const TDesC16>, ...)  - Undefined Reference
    _ZN6RDebug5PrintE11TRefByValueIK7TDesC16Ez@euser{000a0000}[100039e5].dll  - Undefined Reference
    RDebug::Printf(const char*, ...)          - Undefined Reference
    _ZN6RDebug6PrintfEPKcz@euser{000a0000}[100039e5].dll  - Undefined Reference
    TDes16::Copy(const TDesC8&)               - Undefined Reference
    _ZN6TDes164CopyERK6TDesC8@euser{000a0000}[100039e5].dll  - Undefined Reference
    TDes16::Append(TChar)                     - Undefined Reference
    _ZN6TDes166AppendE5TChar@euser{000a0000}[100039e5].dll  - Undefined Reference
    TDes16::Append(const TDesC16&)            - Undefined Reference
    _ZN6TDes166AppendERK7TDesC16@euser{000a0000}[100039e5].dll  - Undefined Reference
    TDes16::Replace(int, int, const TDesC16&)  - Undefined Reference
    _ZN6TDes167ReplaceEiiRK7TDesC16@euser{000a0000}[100039e5].dll  - Undefined Reference
    TDes16::AppendNum(long long)              - Undefined Reference
    _ZN6TDes169AppendNumEx@euser{000a0000}[100039e5].dll  - Undefined Reference
    TPtrC8::TPtrC8(const unsigned char*)      - Undefined Reference
    _ZN6TPtrC8C1EPKh@euser{000a0000}[100039e5].dll  - Undefined Reference
    TPtrC8::TPtrC8(const TDesC8&)             - Undefined Reference
    _ZN6TPtrC8C1ERK6TDesC8@euser{000a0000}[100039e5].dll  - Undefined Reference
    TPtrC8::TPtrC8()                          - Undefined Reference
    _ZN6TPtrC8C1Ev@euser{000a0000}[100039e5].dll  - Undefined Reference
    CActive::Extension_(unsigned, void*&, void*)  - Undefined Reference
    _ZN7CActive10Extension_EjRPvS0_@euser{000a0000}[100039e5].dll  - Undefined Reference
    CActive::Cancel()                         - Undefined Reference
    _ZN7CActive6CancelEv@euser{000a0000}[100039e5].dll  - Undefined Reference
    CActive::RunError(int)                    - Undefined Reference
    _ZN7CActive8RunErrorEi@euser{000a0000}[100039e5].dll  - Undefined Reference
    CActive::SetActive()                      - Undefined Reference
    _ZN7CActive9SetActiveEv@euser{000a0000}[100039e5].dll  - Undefined Reference
    CActive::CActive__sub_object(int)         - Undefined Reference
    _ZN7CActiveC2Ei@euser{000a0000}[100039e5].dll  - Undefined Reference
    CActive::~CActive__sub_object()           - Undefined Reference
    _ZN7CActiveD2Ev@euser{000a0000}[100039e5].dll  - Undefined Reference
    CCoeEnv::Static()                         - Undefined Reference
    _ZN7CCoeEnv6StaticEv@cone{000a0000}[10003a41].dll  - Undefined Reference
    HBufC16::Des()                            - Undefined Reference
    _ZN7HBufC163DesEv@euser{000a0000}[100039e5].dll  - Undefined Reference
    HBufC16::NewL(int)                        - Undefined Reference
    _ZN7HBufC164NewLEi@euser{000a0000}[100039e5].dll  - Undefined Reference
    HBufC16::operator =(const TDesC16&)       - Undefined Reference
    _ZN7HBufC16aSERK7TDesC16@euser{000a0000}[100039e5].dll  - Undefined Reference
    RThread::Open(TThreadId, TOwnerType)      - Undefined Reference
    _ZN7RThread4OpenE9TThreadId10TOwnerType@euser{000a0000}[100039e5].dll  - Undefined Reference
    RThread::Create(const TDesC16&, int(*)(void*), int, RAllocator*, void*, TOwnerType)  - Undefined Reference
    _ZN7RThread6CreateERK7TDesC16PFiPvEiP10RAllocatorS3_10TOwnerType@euser{000a0000}[100039e5].dll  - Undefined Reference
    TPtrC16::TPtrC16(const unsigned short*)   - Undefined Reference
    _ZN7TPtrC16C1EPKt@euser{000a0000}[100039e5].dll  - Undefined Reference
    UserHal::MemoryInfo(TDes8&)               - Undefined Reference
    _ZN7UserHal10MemoryInfoER5TDes8@euser{000a0000}[100039e5].dll  - Undefined Reference
    UserSvr::DllFreeTls(int)                  - Undefined Reference
    _ZN7UserSvr10DllFreeTlsEi@euser{000a0000}[100039e5].dll  - Undefined Reference
    UserSvr::DllTls(int, int)                 - Undefined Reference
    _ZN7UserSvr6DllTlsEii@euser{000a0000}[100039e5].dll  - Undefined Reference
    UserSvr::DllSetTls(int, int, void*)       - Undefined Reference
    _ZN7UserSvr9DllSetTlsEiiPv@euser{000a0000}[100039e5].dll  - Undefined Reference
    CFileMan::Copy(const TDesC16&, const TDesC16&, unsigned)  - Undefined Reference
    _ZN8CFileMan4CopyERK7TDesC16S2_j@efsrv{000a0000}[100039e4].dll  - Undefined Reference
    CFileMan::NewL(RFs&)                      - Undefined Reference
    _ZN8CFileMan4NewLER3RFs@efsrv{000a0000}[100039e4].dll  - Undefined Reference
    CServer2::Extension_(unsigned, void*&, void*)  - Undefined Reference
    _ZN8CServer210Extension_EjRPvS0_@euser{000a0000}[100039e5].dll  - Undefined Reference
    CServer2::RunL()                          - Undefined Reference
    _ZN8CServer24RunLEv@euser{000a0000}[100039e5].dll  - Undefined Reference
    CServer2::StartL(const TDesC16&)          - Undefined Reference
    _ZN8CServer26StartLERK7TDesC16@euser{000a0000}[100039e5].dll  - Undefined Reference
    CServer2::ReStart()                       - Undefined Reference
    _ZN8CServer27ReStartEv@euser{000a0000}[100039e5].dll  - Undefined Reference
    CServer2::DoCancel()                      - Undefined Reference
    _ZN8CServer28DoCancelEv@euser{000a0000}[100039e5].dll  - Undefined Reference
    CServer2::DoConnect(const RMessage2&)     - Undefined Reference
    _ZN8CServer29DoConnectERK9RMessage2@euser{000a0000}[100039e5].dll  - Undefined Reference
    CServer2::CServer2__sub_object(int, CServer2::TServerType)  - Undefined Reference
    _ZN8CServer2C2EiNS_11TServerTypeE@euser{000a0000}[100039e5].dll  - Undefined Reference
    CServer2::~CServer2__sub_object()         - Undefined Reference
    _ZN8CServer2D2Ev@euser{000a0000}[100039e5].dll  - Undefined Reference
    RProcess::Open(TProcessId, TOwnerType)    - Undefined Reference
    _ZN8RProcess4OpenE10TProcessId10TOwnerType@euser{000a0000}[100039e5].dll  - Undefined Reference
    TApaTask::EndTask()                       - Undefined Reference
    _ZN8TApaTask7EndTaskEv@apgrfx{000a0000}[10003a3c].dll  - Undefined Reference
    TApaTask::SetWgId(int)                    - Undefined Reference
    _ZN8TApaTask7SetWgIdEi@apgrfx{000a0000}[10003a3c].dll  - Undefined Reference
    TApaTask::KillTask()                      - Undefined Reference
    _ZN8TApaTask8KillTaskEv@apgrfx{000a0000}[10003a3c].dll  - Undefined Reference
    TApaTask::TApaTask(RWsSession&)           - Undefined Reference
    _ZN8TApaTaskC1ER10RWsSession@apgrfx{000a0000}[10003a3c].dll  - Undefined Reference
    TVersion::TVersion(int, int, int)         - Undefined Reference
    _ZN8TVersionC1Eiii@euser{000a0000}[100039e5].dll  - Undefined Reference
    CSession2::Disconnect(const RMessage2&)   - Undefined Reference
    _ZN9CSession210DisconnectERK9RMessage2@euser{000a0000}[100039e5].dll  - Undefined Reference
    CSession2::Extension_(unsigned, void*&, void*)  - Undefined Reference
    _ZN9CSession210Extension_EjRPvS0_@euser{000a0000}[100039e5].dll  - Undefined Reference
    CSession2::ServiceError(const RMessage2&, int)  - Undefined Reference
    _ZN9CSession212ServiceErrorERK9RMessage2i@euser{000a0000}[100039e5].dll  - Undefined Reference
    CSession2::CountResources()               - Undefined Reference
    _ZN9CSession214CountResourcesEv@euser{000a0000}[100039e5].dll  - Undefined Reference
    CSession2::CSession2__sub_object()        - Undefined Reference
    _ZN9CSession2C2Ev@euser{000a0000}[100039e5].dll  - Undefined Reference
    CSession2::~CSession2__sub_object()       - Undefined Reference
    _ZN9CSession2D2Ev@euser{000a0000}[100039e5].dll  - Undefined Reference
    TBufBase8::TBufBase8(int)                 - Undefined Reference
    _ZN9TBufBase8C1Ei@euser{000a0000}[100039e5].dll  - Undefined Reference
    TBufBase8::TBufBase8(int, int)            - Undefined Reference
    _ZN9TBufBase8C1Eii@euser{000a0000}[100039e5].dll  - Undefined Reference
    RArrayBase::At(int) const                 - Undefined Reference
    _ZNK10RArrayBase2AtEi@euser{000a0000}[100039e5].dll  - Undefined Reference
    RArrayBase::Count() const                 - Undefined Reference
    _ZNK10RArrayBase5CountEv@euser{000a0000}[100039e5].dll  - Undefined Reference
    RWsSession::NumWindowGroups(int) const    - Undefined Reference
    _ZNK10RWsSession15NumWindowGroupsEi@ws32{000a0000}[10003b21].dll  - Undefined Reference
    RWsSession::WindowGroupList(int, RArray<RWsSession::TWindowGroupChainInfo>*) const  - Undefined Reference
    _ZNK10RWsSession15WindowGroupListEiP6RArrayINS_21TWindowGroupChainInfoEE@ws32{000a0000}[10003b21].dll  - Undefined Reference
    RWsSession::GetFocusWindowGroup() const   - Undefined Reference
    _ZNK10RWsSession19GetFocusWindowGroupEv@ws32{000a0000}[10003b21].dll  - Undefined Reference
    RWsSession::GetWindowGroupNameFromIdentifier(int, TDes16&) const  - Undefined Reference
    _ZNK10RWsSession32GetWindowGroupNameFromIdentifierEiR6TDes16@ws32{000a0000}[10003b21].dll  - Undefined Reference
    RWsSession::GetEvent(TWsEvent&) const     - Undefined Reference
    _ZNK10RWsSession8GetEventER8TWsEvent@ws32{000a0000}[10003b21].dll  - Undefined Reference
    RStringBase::DesC() const                 - Undefined Reference
    _ZNK11RStringBase4DesCEv@bafl{000a0000}[10003a0f].dll  - Undefined Reference
    RMessagePtr2::Panic(const TDesC16&, int) const  - Undefined Reference
    _ZNK12RMessagePtr25PanicERK7TDesC16i@euser{000a0000}[100039e5].dll  - Undefined Reference
    RMessagePtr2::Client(RThread&, TOwnerType) const  - Undefined Reference
    _ZNK12RMessagePtr26ClientER7RThread10TOwnerType@euser{000a0000}[100039e5].dll  - Undefined Reference
    RMessagePtr2::Complete(int) const         - Undefined Reference
    _ZNK12RMessagePtr28CompleteEi@euser{000a0000}[100039e5].dll  - Undefined Reference
    RSessionBase::DoSendReceive(int, const TIpcArgs*) const  - Undefined Reference
    _ZNK12RSessionBase13DoSendReceiveEiPK8TIpcArgs@euser{000a0000}[100039e5].dll  - Undefined Reference
    RSessionBase::DoSendReceive(int, const TIpcArgs*, TRequestStatus&) const  - Undefined Reference
    _ZNK12RSessionBase13DoSendReceiveEiPK8TIpcArgsR14TRequestStatus@euser{000a0000}[100039e5].dll  - Undefined Reference
    RWindowGroup::Identifier() const          - Undefined Reference
    _ZNK12RWindowGroup10IdentifierEv@ws32{000a0000}[10003b21].dll  - Undefined Reference
    RHashTableBase::Find(const void*, int) const  - Undefined Reference
    _ZNK14RHashTableBase4FindEPKvi@euser{000a0000}[100039e5].dll  - Undefined Reference
    XLeaveException::GetReason() const        - Undefined Reference
    _ZNK15XLeaveException9GetReasonEv@euser{000a0000}[100039e5].dll  - Undefined Reference
    RPointerArrayBase::At(int) const          - Undefined Reference
    _ZNK17RPointerArrayBase2AtEi@euser{000a0000}[100039e5].dll  - Undefined Reference
    RPointerArrayBase::Count() const          - Undefined Reference
    _ZNK17RPointerArrayBase5CountEv@euser{000a0000}[100039e5].dll  - Undefined Reference
    THashTableIterBase::Current(int) const    - Undefined Reference
    _ZNK18THashTableIterBase7CurrentEi@euser{000a0000}[100039e5].dll  - Undefined Reference
    CApaWindowGroupName::AppUid() const       - Undefined Reference
    _ZNK19CApaWindowGroupName6AppUidEv@apgrfx{000a0000}[10003a3c].dll  - Undefined Reference
    CApaWindowGroupName::Hidden() const       - Undefined Reference
    _ZNK19CApaWindowGroupName6HiddenEv@apgrfx{000a0000}[10003a3c].dll  - Undefined Reference
    CApaWindowGroupName::IsBusy() const       - Undefined Reference
    _ZNK19CApaWindowGroupName6IsBusyEv@apgrfx{000a0000}[10003a3c].dll  - Undefined Reference
    CApaWindowGroupName::IsSystem() const     - Undefined Reference
    _ZNK19CApaWindowGroupName8IsSystemEv@apgrfx{000a0000}[10003a3c].dll  - Undefined Reference
    Xml::RAttribute::Value() const            - Undefined Reference
    _ZNK3Xml10RAttribute5ValueEv@xmlframework{000a0000}[101fadcc].dll  - Undefined Reference
    Xml::RAttribute::Attribute() const        - Undefined Reference
    _ZNK3Xml10RAttribute9AttributeEv@xmlframework{000a0000}[101fadcc].dll  - Undefined Reference
    Xml::RTagInfo::LocalName() const          - Undefined Reference
    _ZNK3Xml8RTagInfo9LocalNameEv@xmlframework{000a0000}[101fadcc].dll  - Undefined Reference
    TUid::operator !=(const TUid&) const      - Undefined Reference
    _ZNK4TUidneERKS_@euser{000a0000}[100039e5].dll  - Undefined Reference
    RFile::Read(TDes8&) const                 - Undefined Reference
    _ZNK5RFile4ReadER5TDes8@efsrv{000a0000}[100039e4].dll  - Undefined Reference
    RFile::Seek(TSeek, int&) const            - Undefined Reference
    _ZNK5RFile4SeekE5TSeekRi@efsrv{000a0000}[100039e4].dll  - Undefined Reference
    TTime::MicroSecondsFrom(TTime) const      - Undefined Reference
    _ZNK5TTime16MicroSecondsFromES_@euser{000a0000}[100039e5].dll  - Undefined Reference
    TTime::FormatL(TDes16&, const TDesC16&) const  - Undefined Reference
    _ZNK5TTime7FormatLER6TDes16RK7TDesC16@euser{000a0000}[100039e5].dll  - Undefined Reference
    TDesC8::Find(const TDesC8&) const         - Undefined Reference
    _ZNK6TDesC84FindERKS_@euser{000a0000}[100039e5].dll  - Undefined Reference
    TDesC8::Left(int) const                   - Undefined Reference
    _ZNK6TDesC84LeftEi@euser{000a0000}[100039e5].dll  - Undefined Reference
    TDesC8::Right(int) const                  - Undefined Reference
    _ZNK6TDesC85RightEi@euser{000a0000}[100039e5].dll  - Undefined Reference
    TDesC8::Compare(const TDesC8&) const      - Undefined Reference
    _ZNK6TDesC87CompareERKS_@euser{000a0000}[100039e5].dll  - Undefined Reference
    RThread::LogonCancel(TRequestStatus&) const  - Undefined Reference
    _ZNK7RThread11LogonCancelER14TRequestStatus@euser{000a0000}[100039e5].dll  - Undefined Reference
    RThread::SetPriority(TThreadPriority) const  - Undefined Reference
    _ZNK7RThread11SetPriorityE15TThreadPriority@euser{000a0000}[100039e5].dll  - Undefined Reference
    RThread::ProcessPriority() const          - Undefined Reference
    _ZNK7RThread15ProcessPriorityEv@euser{000a0000}[100039e5].dll  - Undefined Reference
    RThread::RequestComplete(TRequestStatus*&, int) const  - Undefined Reference
    _ZNK7RThread15RequestCompleteERP14TRequestStatusi@euser{000a0000}[100039e5].dll  - Undefined Reference
    RThread::SetProcessPriority(TProcessPriority) const  - Undefined Reference
    _ZNK7RThread18SetProcessPriorityE16TProcessPriority@euser{000a0000}[100039e5].dll  - Undefined Reference
    RThread::Id() const                       - Undefined Reference
    _ZNK7RThread2IdEv@euser{000a0000}[100039e5].dll  - Undefined Reference
    RThread::Logon(TRequestStatus&) const     - Undefined Reference
    _ZNK7RThread5LogonER14TRequestStatus@euser{000a0000}[100039e5].dll  - Undefined Reference
    RThread::Resume() const                   - Undefined Reference
    _ZNK7RThread6ResumeEv@euser{000a0000}[100039e5].dll  - Undefined Reference
    RThread::SecureId() const                 - Undefined Reference
    _ZNK7RThread8SecureIdEv@euser{000a0000}[100039e5].dll  - Undefined Reference
    RProcess::SecureId() const                - Undefined Reference
    _ZNK8RProcess8SecureIdEv@euser{000a0000}[100039e5].dll  - Undefined Reference
    TApaTask::ThreadId() const                - Undefined Reference
    _ZNK8TApaTask8ThreadIdEv@apgrfx{000a0000}[10003a3c].dll  - Undefined Reference
    typeinfo for XLeaveException              - Undefined Reference
    _ZTI15XLeaveException@drtaeabi{000a0000}.dll  - Undefined Reference
    typeinfo for CActiveScheduler             - Undefined Reference
    _ZTI16CActiveScheduler@euser{000a0000}[100039e5].dll  - Undefined Reference
    typeinfo for CBase                        - Undefined Reference
    _ZTI5CBase@euser{000a0000}[100039e5].dll  - Undefined Reference
    typeinfo for CTimer                       - Undefined Reference
    _ZTI6CTimer@euser{000a0000}[100039e5].dll  - Undefined Reference
    typeinfo for CActive                      - Undefined Reference
    _ZTI7CActive@euser{000a0000}[100039e5].dll  - Undefined Reference
    typeinfo for CServer2                     - Undefined Reference
    _ZTI8CServer2@euser{000a0000}[100039e5].dll  - Undefined Reference
    typeinfo for CSession2                    - Undefined Reference
    _ZTI9CSession2@euser{000a0000}[100039e5].dll  - Undefined Reference
    vtable for CBase                          - Undefined Reference
    _ZTV5CBase@euser{000a0000}[100039e5].dll  - Undefined Reference
    vtable for __cxxabiv1::__class_type_info  - Undefined Reference
    _ZTVN10__cxxabiv117__class_type_infoE@drtaeabi{000a0000}.dll  - Undefined Reference
    vtable for __cxxabiv1::__si_class_type_info  - Undefined Reference
    _ZTVN10__cxxabiv120__si_class_type_infoE@drtaeabi{000a0000}.dll  - Undefined Reference
    vtable for __cxxabiv1::__vmi_class_type_info  - Undefined Reference
    _ZTVN10__cxxabiv121__vmi_class_type_infoE@drtaeabi{000a0000}.dll  - Undefined Reference
    operator delete (void*)                   - Undefined Reference
    _ZdlPv@scppnwdl{000a0000}.dll             - Undefined Reference
    __ARM_ll_cmple                            - Undefined Reference
    __ARM_ll_cmple@drtrvct2_2{000a0000}.dll   - Undefined Reference
    __aeabi_memclr4                           - Undefined Reference
    __aeabi_memclr4@drtaeabi{000a0000}.dll    - Undefined Reference
    __aeabi_memcpy4                           - Undefined Reference
    __aeabi_memcpy4@drtaeabi{000a0000}.dll    - Undefined Reference
    __aeabi_uidivmod                          - Undefined Reference
    __aeabi_uidivmod@drtaeabi{000a0000}.dll   - Undefined Reference
    __aeabi_unwind_cpp_pr0                    - Undefined Reference
    __aeabi_unwind_cpp_pr0@drtaeabi{000a0000}.dll  - Undefined Reference
    __aeabi_unwind_cpp_pr1                    - Undefined Reference
    __aeabi_unwind_cpp_pr1@drtaeabi{000a0000}.dll  - Undefined Reference
    __cxa_begin_catch                         - Undefined Reference
    __cxa_begin_catch@drtaeabi{000a0000}.dll  - Undefined Reference
    __cxa_call_unexpected                     - Undefined Reference
    __cxa_call_unexpected@drtaeabi{000a0000}.dll  - Undefined Reference
    __cxa_end_catch                           - Undefined Reference
    __cxa_end_catch@drtaeabi{000a0000}.dll    - Undefined Reference
    __cxa_end_cleanup                         - Undefined Reference
    __cxa_end_cleanup@drtaeabi{000a0000}.dll  - Undefined Reference
    __cxa_pure_virtual                        - Undefined Reference
    __cxa_pure_virtual@drtaeabi{000a0000}.dll  - Undefined Reference
    eglGetDisplay                             - Undefined Reference
    eglGetDisplay@libEGL{000a0000}.dll        - Undefined Reference
    eglGetProcAddress                         - Undefined Reference
    eglGetProcAddress@libEGL{000a0000}.dll    - Undefined Reference
    eglInitialize                             - Undefined Reference
    eglInitialize@libEGL{000a0000}.dll        - Undefined Reference
    eglQueryString                            - Undefined Reference
    eglQueryString@libEGL{000a0000}.dll       - Undefined Reference
    eglTerminate                              - Undefined Reference
    eglTerminate@libEGL{000a0000}.dll         - Undefined Reference
    memclr                                    - Undefined Reference
    memclr@euser{000a0000}[100039e5].dll      - Undefined Reference
    run_static_dtors                          - Undefined Weak Reference
    strcspn                                   - Undefined Reference
    strcspn@libc{00010000}[10207369].dll      - Undefined Reference
    strlen                                    - Undefined Reference
    strlen@libc{00010000}[10207369].dll       - Undefined Reference
    strncmp                                   - Undefined Reference
    strncmp@libc{00010000}[10207369].dll      - Undefined Reference
    Image$$ER_RO$$Base                       0x00008000   Number         0  anon$$obj.o(linker$$defined$$symbols)
    _E32Dll                                  0x00008000   ARM Code      40  uc_dll_.o(.emb_text)
    Symbian$$CPP$$Exception$$Descriptor      0x00008014   Data           0  uc_dll_.o(.emb_text)
    __cpp_initialize__aeabi_                 0x00008028   ARM Code      52  ucppinit.o(.emb_text)
    std::nothrow                             0x0000805c   ARM Code       0  ucppinit.o(.emb_text)
    __PLT                                    0x0000805c   ARM Code       0  anon$$obj.o(.plt)
    CGOomIdleTimeRule::CGOomIdleTimeRule(TTimeIntervalSeconds, int) 0x000086fd   Thumb Code    52  goomIdletimerule.o(.text)
    CGOomIdleTimeRule::CGOomIdleTimeRule__sub_object(TTimeIntervalSeconds, int) 0x000086fd   Thumb Code     0  goomIdletimerule.o(.text)
    CGOomIdleTimeRule::NewL(TTimeIntervalSeconds, int) 0x00008731   Thumb Code    52  goomIdletimerule.o(.text)
    CGOomIdleTimeRule::RuleIsApplicable(const CGOomWindowGroupList&, int) const 0x00008765   Thumb Code    74  goomIdletimerule.o(.text)
    thunk{-4} to CGOomIdleTimeRule::RuleIsApplicable(const CGOomWindowGroupList&, int) const 0x000087af   Thumb Code    22  goomIdletimerule.o(.text)
    CGOomIdleTimeRule::~CGOomIdleTimeRule()  0x000087c5   Thumb Code    42  goomIdletimerule.o(.text)
    CGOomIdleTimeRule::~CGOomIdleTimeRule__sub_object() 0x000087c5   Thumb Code     0  goomIdletimerule.o(.text)
    CGOomIdleTimeRule::~CGOomIdleTimeRule__deallocating() 0x000087ef   Thumb Code    22  goomIdletimerule.o(.text)
    CGOomAction::~CGOomAction()              0x00008859   Thumb Code     0  goomaction.o(.text)
    CGOomAction::~CGOomAction__sub_object()  0x00008859   Thumb Code    38  goomaction.o(.text)
    CGOomAction::~CGOomAction__deallocating() 0x0000887f   Thumb Code    22  goomaction.o(.text)
    CGOomAction::MemoryFreed(int)            0x00008895   Thumb Code    42  goomaction.o(.text)
    CGOomAction::CGOomAction__sub_object(MGOomActionObserver&) 0x000088bf   Thumb Code    40  goomaction.o(.text)
    CGOomActionConfig::AddRuleL(MGOomRuleConfig*) 0x00008935   Thumb Code    46  goomactionconfig.o(.text)
    CGOomActionConfig::~CGOomActionConfig()  0x00008963   Thumb Code    56  goomactionconfig.o(.text)
    CGOomActionConfig::~CGOomActionConfig__sub_object() 0x00008963   Thumb Code     0  goomactionconfig.o(.text)
    CGOomActionConfig::~CGOomActionConfig__deallocating() 0x0000899b   Thumb Code    22  goomactionconfig.o(.text)
    CGOomActionConfig::Priority(const CGOomWindowGroupList&, int) const 0x000089b1   Thumb Code   146  goomactionconfig.o(.text)
    CGOomActionConfig::ConstructL()          0x00008a43   Thumb Code    26  goomactionconfig.o(.text)
    CGOomActionConfig::CGOomActionConfig(long) 0x00008a5d   Thumb Code    56  goomactionconfig.o(.text)
    CGOomActionConfig::CGOomActionConfig__sub_object(long) 0x00008a5d   Thumb Code     0  goomactionconfig.o(.text)
    CGOomActionList::ConstructL(CGOomConfig&) 0x00008ae5   Thumb Code   212  goomactionlist.o(.text)
    CGOomActionList::CGOomActionList(CMemoryMonitor&, CMemoryMonitorServer&, RWsSession&) 0x00008bb9   Thumb Code   112  goomactionlist.o(.text)
    CGOomActionList::CGOomActionList__sub_object(CMemoryMonitor&, CMemoryMonitorServer&, RWsSession&) 0x00008bb9   Thumb Code     0  goomactionlist.o(.text)
    CGOomActionList::NewL(CMemoryMonitor&, CMemoryMonitorServer&, RWsSession&, CGOomConfig&) 0x00008c29   Thumb Code    68  goomactionlist.o(.text)
    CGOomActionList::~CGOomActionList()      0x00008c6d   Thumb Code   100  goomactionlist.o(.text)
    CGOomActionList::~CGOomActionList__sub_object() 0x00008c6d   Thumb Code     0  goomactionlist.o(.text)
    CGOomActionList::~CGOomActionList__deallocating() 0x00008cd1   Thumb Code    22  goomactionlist.o(.text)
    CGOomActionList::ComparePriorities(const TActionRef&, const TActionRef&) 0x00008ce7   Thumb Code   466  goomactionlist.o(.text)
    CGOomActionList::BuildActionListL(CGOomWindowGroupList&, CGOomConfig&) 0x00008eb9   Thumb Code   750  goomactionlist.o(.text)
    CGOomActionList::MemoryGood()            0x000091a7   Thumb Code   108  goomactionlist.o(.text)
    CGOomActionList::FreeMemoryAboveTarget(int&) 0x00009213   Thumb Code   102  goomactionlist.o(.text)
    CGOomActionList::FreeMemory(int)         0x00009279   Thumb Code   504  goomactionlist.o(.text)
    CGOomActionList::AppNotExiting(int)      0x00009471   Thumb Code   116  goomactionlist.o(.text)
    CGOomActionList::StateChanged()          0x000094e5   Thumb Code   340  goomactionlist.o(.text)
    thunk{-4} to CGOomActionList::StateChanged() 0x00009639   Thumb Code    14  goomactionlist.o(.text)
    TActionRef::TActionRef(TActionRef::TActionType, int, TGOomSyncMode, int, CGOomRunPlugin&, unsigned) 0x00009647   Thumb Code    20  goomactionref.o(.text)
    TActionRef::TActionRef__sub_object(TActionRef::TActionType, int, TGOomSyncMode, int, CGOomRunPlugin&, unsigned) 0x00009647   Thumb Code     0  goomactionref.o(.text)
    TActionRef::TActionRef(TActionRef::TActionType, int, TGOomSyncMode, int, int, unsigned) 0x0000965b   Thumb Code    24  goomactionref.o(.text)
    TActionRef::TActionRef__sub_object(TActionRef::TActionType, int, TGOomSyncMode, int, int, unsigned) 0x0000965b   Thumb Code     0  goomactionref.o(.text)
    TActionRef::Type() const                 0x00009673   Thumb Code     6  goomactionref.o(.text)
    TActionRef::Priority() const             0x00009679   Thumb Code     6  goomactionref.o(.text)
    TActionRef::SyncMode() const             0x0000967f   Thumb Code     6  goomactionref.o(.text)
    TActionRef::RamEstimate() const          0x00009685   Thumb Code     6  goomactionref.o(.text)
    TActionRef::WgId() const                 0x0000968b   Thumb Code     6  goomactionref.o(.text)
    TActionRef::WgIndex() const              0x00009691   Thumb Code     6  goomactionref.o(.text)
    TActionRef::RunPlugin()                  0x00009697   Thumb Code     6  goomactionref.o(.text)
    CGOomAppCloseTimer::CGOomAppCloseTimer(CGOomCloseApp&) 0x000096dd   Thumb Code    52  goomappclosetimer.o(.text)
    CGOomAppCloseTimer::CGOomAppCloseTimer__sub_object(CGOomCloseApp&) 0x000096dd   Thumb Code     0  goomappclosetimer.o(.text)
    CGOomAppCloseTimer::NewL(CGOomCloseApp&) 0x00009711   Thumb Code    74  goomappclosetimer.o(.text)
    CGOomAppCloseTimer::RunL()               0x0000975b   Thumb Code    32  goomappclosetimer.o(.text)
    CGOomAppCloseWatcher::CGOomAppCloseWatcher(CGOomCloseApp&) 0x000097c5   Thumb Code    68  goomappclosewatcher.o(.text)
    CGOomAppCloseWatcher::CGOomAppCloseWatcher__sub_object(CGOomCloseApp&) 0x000097c5   Thumb Code     0  goomappclosewatcher.o(.text)
    CGOomAppCloseWatcher::~CGOomAppCloseWatcher() 0x00009809   Thumb Code    44  goomappclosewatcher.o(.text)
    CGOomAppCloseWatcher::~CGOomAppCloseWatcher__sub_object() 0x00009809   Thumb Code     0  goomappclosewatcher.o(.text)
    CGOomAppCloseWatcher::~CGOomAppCloseWatcher__deallocating() 0x00009835   Thumb Code    22  goomappclosewatcher.o(.text)
    CGOomAppCloseWatcher::Start(const TApaTask&) 0x0000984b   Thumb Code   132  goomappclosewatcher.o(.text)
    CGOomAppCloseWatcher::DoCancel()         0x000098cf   Thumb Code    54  goomappclosewatcher.o(.text)
    CGOomAppCloseWatcher::RunL()             0x00009905   Thumb Code    76  goomappclosewatcher.o(.text)
    CGOomApplicationConfig::ConstructL()     0x000099a1   Thumb Code    34  goomapplicationconfig.o(.text)
    CGOomApplicationConfig::CGOomApplicationConfig(unsigned) 0x000099c3   Thumb Code    40  goomapplicationconfig.o(.text)
    CGOomApplicationConfig::CGOomApplicationConfig__sub_object(unsigned) 0x000099c3   Thumb Code     0  goomapplicationconfig.o(.text)
    CGOomApplicationConfig::NewL(unsigned)   0x000099eb   Thumb Code    72  goomapplicationconfig.o(.text)
    CGOomApplicationConfig::AddRuleL(MGOomRuleConfig*) 0x00009a33   Thumb Code    46  goomapplicationconfig.o(.text)
    CGOomApplicationConfig::~CGOomApplicationConfig() 0x00009a61   Thumb Code    54  goomapplicationconfig.o(.text)
    CGOomApplicationConfig::~CGOomApplicationConfig__sub_object() 0x00009a61   Thumb Code     0  goomapplicationconfig.o(.text)
    CGOomApplicationConfig::~CGOomApplicationConfig__deallocating() 0x00009a97   Thumb Code    22  goomapplicationconfig.o(.text)
    CGOomCloseApp::ConstructL()              0x00009afd   Thumb Code    54  goomcloseapp.o(.text)
    CGOomCloseApp::CGOomCloseApp(MGOomActionObserver&, RWsSession&) 0x00009b33   Thumb Code    60  goomcloseapp.o(.text)
    CGOomCloseApp::CGOomCloseApp__sub_object(MGOomActionObserver&, RWsSession&) 0x00009b33   Thumb Code     0  goomcloseapp.o(.text)
    CGOomCloseApp::NewL(MGOomActionObserver&, RWsSession&) 0x00009b6f   Thumb Code    74  goomcloseapp.o(.text)
    CGOomCloseApp::FreeMemory(int)           0x00009bb9   Thumb Code   100  goomcloseapp.o(.text)
    CGOomCloseApp::~CGOomCloseApp()          0x00009c1d   Thumb Code    94  goomcloseapp.o(.text)
    CGOomCloseApp::~CGOomCloseApp__sub_object() 0x00009c1d   Thumb Code     0  goomcloseapp.o(.text)
    CGOomCloseApp::~CGOomCloseApp__deallocating() 0x00009c7b   Thumb Code    22  goomcloseapp.o(.text)
    CGOomCloseApp::CloseAppEvent()           0x00009c91   Thumb Code    62  goomcloseapp.o(.text)
    CGOomCloseApp::Reconfigure(const TActionRef&) 0x00009ccf   Thumb Code    36  goomcloseapp.o(.text)
    CGOomCloseApp::KillTask()                0x00009cf3   Thumb Code    54  goomcloseapp.o(.text)
    CGOomCloseAppConfig::CGOomCloseAppConfig(long) 0x00009d79   Thumb Code    44  goomcloseappconfig.o(.text)
    CGOomCloseAppConfig::CGOomCloseAppConfig__sub_object(long) 0x00009d79   Thumb Code     0  goomcloseappconfig.o(.text)
    CGOomCloseAppConfig::NewL(long)          0x00009da5   Thumb Code    74  goomcloseappconfig.o(.text)
    CGOomCloseAppConfig::~CGOomCloseAppConfig() 0x00009def   Thumb Code    38  goomcloseappconfig.o(.text)
    CGOomCloseAppConfig::~CGOomCloseAppConfig__sub_object() 0x00009def   Thumb Code     0  goomcloseappconfig.o(.text)
    CGOomCloseAppConfig::~CGOomCloseAppConfig__deallocating() 0x00009e15   Thumb Code    22  goomcloseappconfig.o(.text)
    CGOomConfig::ConstructL()                0x00009e75   Thumb Code    26  goomconfig.o(.text)
    CGOomConfig::NewL()                      0x00009e8f   Thumb Code    68  goomconfig.o(.text)
    CGOomConfig::SetAppCloseConfigL(CGOomCloseAppConfig*) 0x00009ed3   Thumb Code    90  goomconfig.o(.text)
    CGOomConfig::AddPluginConfigL(CGOomRunPluginConfig*) 0x00009f2d   Thumb Code    88  goomconfig.o(.text)
    CGOomConfig::AddApplicationRuleL(unsigned, MGOomRuleConfig*) 0x00009f85   Thumb Code    62  goomconfig.o(.text)
    CGOomConfig::AddPluginRuleL(unsigned, MGOomRuleConfig*) 0x00009fc3   Thumb Code    64  goomconfig.o(.text)
    CGOomConfig::AddApplicationConfigL(CGOomApplicationConfig*) 0x0000a003   Thumb Code    68  goomconfig.o(.text)
    CGOomConfig::GetApplicationConfig(long)  0x0000a047   Thumb Code    70  goomconfig.o(.text)
    CGOomConfig::GetPluginConfig(long)       0x0000a08d   Thumb Code    74  goomconfig.o(.text)
    CGOomConfig::~CGOomConfig()              0x0000a0d7   Thumb Code   192  goomconfig.o(.text)
    CGOomConfig::~CGOomConfig__sub_object()  0x0000a0d7   Thumb Code     0  goomconfig.o(.text)
    CGOomConfig::~CGOomConfig__deallocating() 0x0000a197   Thumb Code    22  goomconfig.o(.text)
    CGOomConfigParser::CGOomConfigParser(CGOomConfig&, RFs&) 0x0000a1f9   Thumb Code    28  goomconfigparser.o(.text)
    CGOomConfigParser::CGOomConfigParser__sub_object(CGOomConfig&, RFs&) 0x0000a1f9   Thumb Code     0  goomconfigparser.o(.text)
    CGOomConfigParser::ParseL()              0x0000a215   Thumb Code   358  goomconfigparser.o(.text)
    CGOomConfigParser::OnStartDocumentL(const Xml::RDocumentParameters&, int) 0x0000a37b   Thumb Code    30  goomconfigparser.o(.text)
    thunk{-4} to CGOomConfigParser::OnStartDocumentL(const Xml::RDocumentParameters&, int) 0x0000a399   Thumb Code    22  goomconfigparser.o(.text)
    CGOomConfigParser::OnEndDocumentL(int)   0x0000a3af   Thumb Code    28  goomconfigparser.o(.text)
    thunk{-4} to CGOomConfigParser::OnEndDocumentL(int) 0x0000a3cb   Thumb Code    18  goomconfigparser.o(.text)
    CGOomConfigParser::ConfigError(int)      0x0000a3dd   Thumb Code    14  goomconfigparser.o(.text)
    CGOomConfigParser::GetValueFromAttributeList(const RArray<Xml::RAttribute>&, const TDesC8&, TPtrC8&) 0x0000a3eb   Thumb Code   154  goomconfigparser.o(.text)
    CGOomConfigParser::GetValueFromDecimalAttributeList(const RArray<Xml::RAttribute>&, const TDesC8&, unsigned&) 0x0000a485   Thumb Code   100  goomconfigparser.o(.text)
    CGOomConfigParser::GetValueFromHexAttributeList(const RArray<Xml::RAttribute>&, const TDesC8&, unsigned&) 0x0000a4e9   Thumb Code   232  goomconfigparser.o(.text)
    CGOomConfigParser::SetPluginForegroundAppPriorityL(const RArray<Xml::RAttribute>&) 0x0000a5d1   Thumb Code   226  goomconfigparser.o(.text)
    CGOomConfigParser::CheckState(CGOomConfigParser::TGOomParsingState, CGOomConfigParser::TGOomParsingState, int) 0x0000a6b3   Thumb Code    32  goomconfigparser.o(.text)
    CGOomConfigParser::GetValueFromDecimalAttributeList(const RArray<Xml::RAttribute>&, const TDesC8&, int&) 0x0000a6d3   Thumb Code    32  goomconfigparser.o(.text)
    CGOomConfigParser::SetPluginIdlePriorityL(const RArray<Xml::RAttribute>&) 0x0000a6f3   Thumb Code   156  goomconfigparser.o(.text)
    CGOomConfigParser::CheckState(CGOomConfigParser::TGOomParsingState, int) 0x0000a78f   Thumb Code    24  goomconfigparser.o(.text)
    CGOomConfigParser::SetPluginSyncMode(const RArray<Xml::RAttribute>&, CGOomRunPluginConfig&) 0x0000a7a7   Thumb Code   148  goomconfigparser.o(.text)
    CGOomConfigParser::SetAppPluginConfigL(const RArray<Xml::RAttribute>&) 0x0000a83b   Thumb Code   270  goomconfigparser.o(.text)
    CGOomConfigParser::SetSystemPluginConfigL(const RArray<Xml::RAttribute>&) 0x0000a949   Thumb Code   222  goomconfigparser.o(.text)
    CGOomConfigParser::SetForegroundAppPriorityL(const RArray<Xml::RAttribute>&) 0x0000aa27   Thumb Code   154  goomconfigparser.o(.text)
    CGOomConfigParser::SetAppCloseIdlePriorityConfigL(const RArray<Xml::RAttribute>&) 0x0000aac1   Thumb Code   156  goomconfigparser.o(.text)
    CGOomConfigParser::SetCloseAppConfigL(const RArray<Xml::RAttribute>&) 0x0000ab5d   Thumb Code   354  goomconfigparser.o(.text)
    CGOomConfigParser::SetAppConfigL(const RArray<Xml::RAttribute>&) 0x0000acbf   Thumb Code   294  goomconfigparser.o(.text)
    CGOomConfigParser::SetForceCheckConfigL(const RArray<Xml::RAttribute>&) 0x0000ade5   Thumb Code    86  goomconfigparser.o(.text)
    CGOomConfigParser::ChangeState(CGOomConfigParser::TGOomParsingState) 0x0000ae3b   Thumb Code     4  goomconfigparser.o(.text)
    CGOomConfigParser::SetGlobalSettings(const RArray<Xml::RAttribute>&) 0x0000ae3f   Thumb Code   222  goomconfigparser.o(.text)
    CGOomConfigParser::StartElementL(const TDesC8&, const RArray<Xml::RAttribute>&) 0x0000af1d   Thumb Code   598  goomconfigparser.o(.text)
    CGOomConfigParser::OnStartElementL(const Xml::RTagInfo&, const RArray<Xml::RAttribute>&, int) 0x0000b173   Thumb Code    58  goomconfigparser.o(.text)
    thunk{-4} to CGOomConfigParser::OnStartElementL(const Xml::RTagInfo&, const RArray<Xml::RAttribute>&, int) 0x0000b1ad   Thumb Code    26  goomconfigparser.o(.text)
    CGOomConfigParser::OnEndElementL(const Xml::RTagInfo&, int) 0x0000b1c7   Thumb Code     2  goomconfigparser.o(.text)
    thunk{-4} to CGOomConfigParser::OnEndElementL(const Xml::RTagInfo&, int) 0x0000b1c9   Thumb Code    22  goomconfigparser.o(.text)
    CGOomConfigParser::OnContentL(const TDesC8&, int) 0x0000b1df   Thumb Code     2  goomconfigparser.o(.text)
    thunk{-4} to CGOomConfigParser::OnContentL(const TDesC8&, int) 0x0000b1e1   Thumb Code    22  goomconfigparser.o(.text)
    CGOomConfigParser::OnStartPrefixMappingL(const RString&, const RString&, int) 0x0000b1f7   Thumb Code     2  goomconfigparser.o(.text)
    thunk{-4} to CGOomConfigParser::OnStartPrefixMappingL(const RString&, const RString&, int) 0x0000b1f9   Thumb Code    26  goomconfigparser.o(.text)
    CGOomConfigParser::OnEndPrefixMappingL(const RString&, int) 0x0000b213   Thumb Code     2  goomconfigparser.o(.text)
    thunk{-4} to CGOomConfigParser::OnEndPrefixMappingL(const RString&, int) 0x0000b215   Thumb Code    22  goomconfigparser.o(.text)
    CGOomConfigParser::OnIgnorableWhiteSpaceL(const TDesC8&, int) 0x0000b22b   Thumb Code     2  goomconfigparser.o(.text)
    thunk{-4} to CGOomConfigParser::OnIgnorableWhiteSpaceL(const TDesC8&, int) 0x0000b22d   Thumb Code    22  goomconfigparser.o(.text)
    CGOomConfigParser::OnSkippedEntityL(const RString&, int) 0x0000b243   Thumb Code     2  goomconfigparser.o(.text)
    thunk{-4} to CGOomConfigParser::OnSkippedEntityL(const RString&, int) 0x0000b245   Thumb Code    22  goomconfigparser.o(.text)
    CGOomConfigParser::OnProcessingInstructionL(const TDesC8&, const TDesC8&, int) 0x0000b25b   Thumb Code     2  goomconfigparser.o(.text)
    thunk{-4} to CGOomConfigParser::OnProcessingInstructionL(const TDesC8&, const TDesC8&, int) 0x0000b25d   Thumb Code    26  goomconfigparser.o(.text)
    CGOomConfigParser::OnError(int)          0x0000b277   Thumb Code     2  goomconfigparser.o(.text)
    thunk{-4} to CGOomConfigParser::OnError(int) 0x0000b279   Thumb Code    18  goomconfigparser.o(.text)
    CGOomConfigParser::GetExtendedInterface(long) 0x0000b28b   Thumb Code     6  goomconfigparser.o(.text)
    thunk{-4} to CGOomConfigParser::GetExtendedInterface(long) 0x0000b291   Thumb Code    18  goomconfigparser.o(.text)
    CGOomForegroundRule::CGOomForegroundRule(int, int) 0x0000b2e5   Thumb Code    52  goomforegroundrule.o(.text)
    CGOomForegroundRule::CGOomForegroundRule__sub_object(int, int) 0x0000b2e5   Thumb Code     0  goomforegroundrule.o(.text)
    CGOomForegroundRule::RuleIsApplicable(const CGOomWindowGroupList&, int) const 0x0000b319   Thumb Code    72  goomforegroundrule.o(.text)
    thunk{-4} to CGOomForegroundRule::RuleIsApplicable(const CGOomWindowGroupList&, int) const 0x0000b361   Thumb Code    22  goomforegroundrule.o(.text)
    CGOomGlobalConfig::~CGOomGlobalConfig()  0x0000b3c9   Thumb Code    48  goomglobalconfig.o(.text)
    CGOomGlobalConfig::~CGOomGlobalConfig__sub_object() 0x0000b3c9   Thumb Code     0  goomglobalconfig.o(.text)
    CGOomGlobalConfig::~CGOomGlobalConfig__deallocating() 0x0000b3f9   Thumb Code    22  goomglobalconfig.o(.text)
    CGOomLogger::ConstructL()                0x0000b419   Thumb Code   216  goomlog.o(.text)
    CGOomLogger::CGOomLogger(RWsSession&, RFs&) 0x0000b4f1   Thumb Code   106  goomlog.o(.text)
    CGOomLogger::CGOomLogger__sub_object(RWsSession&, RFs&) 0x0000b4f1   Thumb Code     0  goomlog.o(.text)
    CGOomLogger::NewL(RWsSession&, RFs&)     0x0000b55b   Thumb Code    58  goomlog.o(.text)
    CGOomLogger::LogFreeMemory()             0x0000b595   Thumb Code    76  goomlog.o(.text)
    CGOomLogger::Write(const TDesC8&)        0x0000b5e1   Thumb Code    46  goomlog.o(.text)
    CGOomLogger::GetUidFromWindowGroupId(int) 0x0000b60f   Thumb Code    72  goomlog.o(.text)
    CGOomLogger::ColapseWindowGroupTree()    0x0000b657   Thumb Code   182  goomlog.o(.text)
    CGOomLogger::LogApplicationIds()         0x0000b70d   Thumb Code   248  goomlog.o(.text)
    CGOomLogger::StartL()                    0x0000b805   Thumb Code   144  goomlog.o(.text)
    CGOomLogger::RunL()                      0x0000b895   Thumb Code   132  goomlog.o(.text)
    CGOomLogger::DoCancel()                  0x0000b919   Thumb Code    42  goomlog.o(.text)
    CGOomLogger::~CGOomLogger()              0x0000b943   Thumb Code    42  goomlog.o(.text)
    CGOomLogger::~CGOomLogger__sub_object()  0x0000b943   Thumb Code     0  goomlog.o(.text)
    CGOomLogger::~CGOomLogger__deallocating() 0x0000b96d   Thumb Code    22  goomlog.o(.text)
    EGLSynchObjThreadStartFunction(void*)    0x0000b9d9   Thumb Code    76  goommemorymonitor.o(.text)
    CreateThresholdCrossedThreadL(CMemoryMonitor&, unsigned, int) 0x0000ba25   Thumb Code   118  goommemorymonitor.o(.text)
    CMemoryMonitor::GetFreeMemory()          0x0000ba9b   Thumb Code   348  goommemorymonitor.o(.text)
    CMemoryMonitor::GlobalConfig()           0x0000bbf7   Thumb Code    16  goommemorymonitor.o(.text)
    CMemoryMonitor::RefreshThresholds(int)   0x0000bc07   Thumb Code   606  goommemorymonitor.o(.text)
    CMemoryMonitor::ConstructL()             0x0000be65   Thumb Code   394  goommemorymonitor.o(.text)
    CMemoryMonitor::CMemoryMonitor()         0x0000bfef   Thumb Code    66  goommemorymonitor.o(.text)
    CMemoryMonitor::CMemoryMonitor__sub_object() 0x0000bfef   Thumb Code     0  goommemorymonitor.o(.text)
    CMemoryMonitor::NewL()                   0x0000c031   Thumb Code    68  goommemorymonitor.o(.text)
    CMemoryMonitor::~CMemoryMonitor()        0x0000c075   Thumb Code   192  goommemorymonitor.o(.text)
    CMemoryMonitor::~CMemoryMonitor__sub_object() 0x0000c075   Thumb Code     0  goommemorymonitor.o(.text)
    CMemoryMonitor::~CMemoryMonitor__deallocating() 0x0000c135   Thumb Code    22  goommemorymonitor.o(.text)
    CMemoryMonitor::ResetTargets()           0x0000c14b   Thumb Code    36  goommemorymonitor.o(.text)
    CMemoryMonitor::FreeGraphicsMemoryAboveThresholdL(int&) 0x0000c16f   Thumb Code   150  goommemorymonitor.o(.text)
    CMemoryMonitor::StartFreeSomeRamL(int, int) 0x0000c205   Thumb Code   152  goommemorymonitor.o(.text)
    CMemoryMonitor::StartFreeSomeRamL(int)   0x0000c29d   Thumb Code    36  goommemorymonitor.o(.text)
    CMemoryMonitor::FreeMemThresholdCrossedL(int, int) 0x0000c2c1   Thumb Code   164  goommemorymonitor.o(.text)
    CMemoryMonitor::AppNotExiting(int)       0x0000c365   Thumb Code    36  goommemorymonitor.o(.text)
    CMemoryMonitor::FreeOptionalRamL(int, int, int) 0x0000c389   Thumb Code    78  goommemorymonitor.o(.text)
    CMemoryMonitor::RequestFreeMemoryL(int, int) 0x0000c3d7   Thumb Code    52  goommemorymonitor.o(.text)
    CMemoryMonitor::HandleFocusedWgChangeL(int) 0x0000c40b   Thumb Code    72  goommemorymonitor.o(.text)
    CMemoryMonitor::SetPriorityBusy(int)     0x0000c453   Thumb Code    36  goommemorymonitor.o(.text)
    CMemoryMonitor::SetPriorityNormal(int)   0x0000c477   Thumb Code    34  goommemorymonitor.o(.text)
    CMemoryMonitor::SetPriorityHigh(int)     0x0000c499   Thumb Code    16  goommemorymonitor.o(.text)
    CMemoryMonitor::DoPostponedMemoryGood()  0x0000c4a9   Thumb Code    74  goommemorymonitor.o(.text)
    CMemoryMonitorServer::ConstructL()       0x0000c559   Thumb Code    84  goommemorymonitorserver.o(.text)
    CMemoryMonitorServer::CMemoryMonitorServer(CMemoryMonitor&) 0x0000c5ad   Thumb Code    48  goommemorymonitorserver.o(.text)
    CMemoryMonitorServer::CMemoryMonitorServer__sub_object(CMemoryMonitor&) 0x0000c5ad   Thumb Code     0  goommemorymonitorserver.o(.text)
    CMemoryMonitorServer::NewL(CMemoryMonitor&) 0x0000c5dd   Thumb Code   116  goommemorymonitorserver.o(.text)
    CMemoryMonitorServer::~CMemoryMonitorServer() 0x0000c651   Thumb Code    38  goommemorymonitorserver.o(.text)
    CMemoryMonitorServer::~CMemoryMonitorServer__sub_object() 0x0000c651   Thumb Code     0  goommemorymonitorserver.o(.text)
    CMemoryMonitorServer::~CMemoryMonitorServer__deallocating() 0x0000c677   Thumb Code    22  goommemorymonitorserver.o(.text)
    CMemoryMonitorServer::Monitor()          0x0000c68d   Thumb Code    30  goommemorymonitorserver.o(.text)
    CMemoryMonitorServer::CloseAppsFinished(int, int) 0x0000c6ab   Thumb Code    66  goommemorymonitorserver.o(.text)
    CMemoryMonitorServer::NewSessionL(const TVersion&, const RMessage2&) const 0x0000c6ed   Thumb Code    48  goommemorymonitorserver.o(.text)
    CMemoryMonitorServer::RunError(int)      0x0000c71d   Thumb Code    50  goommemorymonitorserver.o(.text)
    CMemoryMonitorSession::CMemoryMonitorSession() 0x0000c7a1   Thumb Code    50  goommemorymonitorsession.o(.text)
    CMemoryMonitorSession::CMemoryMonitorSession__sub_object() 0x0000c7a1   Thumb Code     0  goommemorymonitorsession.o(.text)
    CMemoryMonitorSession::CreateL()         0x0000c7d3   Thumb Code    26  goommemorymonitorsession.o(.text)
    CMemoryMonitorSession::Server()          0x0000c7ed   Thumb Code    34  goommemorymonitorsession.o(.text)
    CMemoryMonitorSession::CloseAppsFinished(int, int) 0x0000c80f   Thumb Code   128  goommemorymonitorsession.o(.text)
    CMemoryMonitorSession::~CMemoryMonitorSession() 0x0000c88f   Thumb Code    74  goommemorymonitorsession.o(.text)
    CMemoryMonitorSession::~CMemoryMonitorSession__sub_object() 0x0000c88f   Thumb Code     0  goommemorymonitorsession.o(.text)
    CMemoryMonitorSession::~CMemoryMonitorSession__deallocating() 0x0000c8d9   Thumb Code    22  goommemorymonitorsession.o(.text)
    CMemoryMonitorSession::Monitor()         0x0000c8ef   Thumb Code    42  goommemorymonitorsession.o(.text)
    CMemoryMonitorSession::ServiceL(const RMessage2&) 0x0000c919   Thumb Code   686  goommemorymonitorsession.o(.text)
    GOOMWatcherThreadFunction(void*)         0x0000cc0d   Thumb Code   282  goommonitor.o(.text)
    CreateGOOMWatcherThreadL()               0x0000cd27   Thumb Code   134  goommonitor.o(.text)
    PanicClient(const RMessagePtr2&, TGOomMonitorClientPanic) 0x0000cdad   Thumb Code    50  goommonitor.o(.text)
    SetGMemoryMonitorTls(CMemoryMonitor*)    0x0000cea5   Thumb Code    30  goommonitorplugin.o(.text)
    MemoryMonitorTls()                       0x0000cec3   Thumb Code    32  goommonitorplugin.o(.text)
    GOomMonitorPluginPanic(TGOomMonitorPluginPanic) 0x0000cee3   Thumb Code    44  goommonitorplugin.o(.text)
    CGOomMonitorPluginBase::CGOomMonitorPluginBase__sub_object() 0x0000cf0f   Thumb Code    92  goommonitorplugin.o(.text)
    CGOomMonitorPluginBase::~CGOomMonitorPluginBase() 0x0000cf6b   Thumb Code     0  goommonitorplugin.o(.text)
    CGOomMonitorPluginBase::~CGOomMonitorPluginBase__sub_object() 0x0000cf6b   Thumb Code    38  goommonitorplugin.o(.text)
    CGOomMonitorPluginBase::~CGOomMonitorPluginBase__deallocating() 0x0000cf91   Thumb Code    22  goommonitorplugin.o(.text)
    CGOomMonitorPluginBase::ConstructL()     0x0000cfa7   Thumb Code    26  goommonitorplugin.o(.text)
    CGOomMonitorPluginBase::FsSession()      0x0000cfc1   Thumb Code    32  goommonitorplugin.o(.text)
    CGOomMonitorPluginBase::WsSession()      0x0000cfe1   Thumb Code    34  goommonitorplugin.o(.text)
    CGOomMonitorPluginBase::ExtensionInterface(TUid, void*&) 0x0000d003   Thumb Code    28  goommonitorplugin.o(.text)
    CAppGOomMonitorPlugin::CAppGOomMonitorPlugin(TUid) 0x0000d01f   Thumb Code    24  goommonitorplugin.o(.text)
    CAppGOomMonitorPlugin::CAppGOomMonitorPlugin__sub_object(TUid) 0x0000d01f   Thumb Code     0  goommonitorplugin.o(.text)
    CAppGOomMonitorPlugin::NewL(TUid)        0x0000d037   Thumb Code    26  goommonitorplugin.o(.text)
    CAppGOomMonitorPlugin::SendMessageToApp(int) 0x0000d051   Thumb Code   124  goommonitorplugin.o(.text)
    CAppGOomMonitorPlugin::FreeRam(int)      0x0000d0cd   Thumb Code    16  goommonitorplugin.o(.text)
    CAppGOomMonitorPlugin::MemoryGood()      0x0000d0dd   Thumb Code    16  goommonitorplugin.o(.text)
    RGOomMonitorSession::Connect()           0x0000d14d   Thumb Code    86  goommonitorsession.o(.text)
    RGOomMonitorSession::IsConnected()       0x0000d1a3   Thumb Code    34  goommonitorsession.o(.text)
    RGOomMonitorSession::RequestFreeMemory(int) 0x0000d1c5   Thumb Code    88  goommonitorsession.o(.text)
    RGOomMonitorSession::RequestFreeMemory(int, TRequestStatus&) 0x0000d21d   Thumb Code    94  goommonitorsession.o(.text)
    RGOomMonitorSession::RequestOptionalRam(int, int, int, int&) 0x0000d27b   Thumb Code   120  goommonitorsession.o(.text)
    RGOomMonitorSession::RequestOptionalRam(int, int, int, TRequestStatus&) 0x0000d2f3   Thumb Code   102  goommonitorsession.o(.text)
    RGOomMonitorSession::CancelRequestFreeMemory() 0x0000d359   Thumb Code    58  goommonitorsession.o(.text)
    RGOomMonitorSession::ThisAppIsNotExiting(int) 0x0000d393   Thumb Code    64  goommonitorsession.o(.text)
    RGOomMonitorSession::SetGOomPriority(RGOomMonitorSession::TGOomPriority) 0x0000d3d3   Thumb Code   158  goommonitorsession.o(.text)
    RGOomMonitorSession::ApplicationAboutToStart(const TUid&) 0x0000d471   Thumb Code    66  goommonitorsession.o(.text)
    RGOomMonitorSession::UsesAbsoluteMemTargets(int) 0x0000d4b3   Thumb Code    78  goommonitorsession.o(.text)
    RGOomMonitorSession::Connect(TRequestStatus&) 0x0000d501   Thumb Code    86  goommonitorsession.o(.text)
    RGOomMonitorSession::AppAboutToStart(TRequestStatus&, const TUid&) 0x0000d557   Thumb Code    70  goommonitorsession.o(.text)
    GOomMonitorPanic(TGOomMonitorPanic)      0x0000d5a5   Thumb Code    22  goompanic.o(.text)
    GOomConfigParserPanic(int)               0x0000d5bb   Thumb Code    24  goompanic.o(.text)
    CGOomPluginWaiter::CGOomPluginWaiter(int, CGOomRunPlugin&) 0x0000d619   Thumb Code    56  goompluginwaiter.o(.text)
    CGOomPluginWaiter::CGOomPluginWaiter__sub_object(int, CGOomRunPlugin&) 0x0000d619   Thumb Code     0  goompluginwaiter.o(.text)
    CGOomPluginWaiter::NewL(int, CGOomRunPlugin&) 0x0000d651   Thumb Code    76  goompluginwaiter.o(.text)
    CGOomPluginWaiter::Start()               0x0000d69d   Thumb Code    50  goompluginwaiter.o(.text)
    CGOomPluginWaiter::RunL()                0x0000d6cf   Thumb Code    36  goompluginwaiter.o(.text)
    CGOomRunPlugin::ConstructL(CGOomRunPluginConfig&) 0x0000d73d   Thumb Code    58  goomrunplugin.o(.text)
    CGOomRunPlugin::CGOomRunPlugin(unsigned, CGOomRunPluginConfig&, MGOomActionObserver&, CGOomMonitorPlugin&) 0x0000d777   Thumb Code    62  goomrunplugin.o(.text)
    CGOomRunPlugin::CGOomRunPlugin__sub_object(unsigned, CGOomRunPluginConfig&, MGOomActionObserver&, CGOomMonitorPlugin&) 0x0000d777   Thumb Code     0  goomrunplugin.o(.text)
    CGOomRunPlugin::NewL(unsigned, CGOomRunPluginConfig&, MGOomActionObserver&, CGOomMonitorPlugin&) 0x0000d7b5   Thumb Code    78  goomrunplugin.o(.text)
    CGOomRunPlugin::~CGOomRunPlugin()        0x0000d803   Thumb Code    54  goomrunplugin.o(.text)
    CGOomRunPlugin::~CGOomRunPlugin__sub_object() 0x0000d803   Thumb Code     0  goomrunplugin.o(.text)
    CGOomRunPlugin::~CGOomRunPlugin__deallocating() 0x0000d839   Thumb Code    22  goomrunplugin.o(.text)
    CGOomRunPlugin::FreeMemory(int)          0x0000d84f   Thumb Code   134  goomrunplugin.o(.text)
    CGOomRunPlugin::MemoryGood()             0x0000d8d5   Thumb Code    46  goomrunplugin.o(.text)
    CGOomRunPluginConfig::CGOomRunPluginConfig(unsigned, TGOomPluginType) 0x0000d951   Thumb Code    54  goomrunpluginconfig.o(.text)
    CGOomRunPluginConfig::CGOomRunPluginConfig__sub_object(unsigned, TGOomPluginType) 0x0000d951   Thumb Code     0  goomrunpluginconfig.o(.text)
    CGOomRunPluginConfig::NewL(unsigned, TGOomPluginType) 0x0000d987   Thumb Code    52  goomrunpluginconfig.o(.text)
    CGOomRunPluginConfig::CalculatePluginPriority(const CGOomWindowGroupList&) 0x0000d9bb   Thumb Code    52  goomrunpluginconfig.o(.text)
    CGOomRunPluginConfig::~CGOomRunPluginConfig() 0x0000d9ef   Thumb Code    38  goomrunpluginconfig.o(.text)
    CGOomRunPluginConfig::~CGOomRunPluginConfig__sub_object() 0x0000d9ef   Thumb Code     0  goomrunpluginconfig.o(.text)
    CGOomRunPluginConfig::~CGOomRunPluginConfig__deallocating() 0x0000da15   Thumb Code    22  goomrunpluginconfig.o(.text)
    CGOomWindowGroupList::ConstructL()       0x0000da79   Thumb Code   108  goomwindowgrouplist.o(.text)
    CGOomWindowGroupList::CGOomWindowGroupList(RWsSession&) 0x0000dae5   Thumb Code   154  goomwindowgrouplist.o(.text)
    CGOomWindowGroupList::CGOomWindowGroupList__sub_object(RWsSession&) 0x0000dae5   Thumb Code     0  goomwindowgrouplist.o(.text)
    CGOomWindowGroupList::NewL(RWsSession&)  0x0000db7f   Thumb Code    74  goomwindowgrouplist.o(.text)
    CGOomWindowGroupList::TGOomWindowGroupProperties::TGOomWindowGroupProperties() 0x0000dbc9   Thumb Code    34  goomwindowgrouplist.o(.text)
    CGOomWindowGroupList::TGOomWindowGroupProperties::TGOomWindowGroupProperties__sub_object() 0x0000dbc9   Thumb Code     0  goomwindowgrouplist.o(.text)
    CGOomWindowGroupList::AppId(int, int) const 0x0000dbeb   Thumb Code   314  goomwindowgrouplist.o(.text)
    CGOomWindowGroupList::RemovePropertiesForClosedWindowsL() 0x0000dd25   Thumb Code   256  goomwindowgrouplist.o(.text)
    CGOomWindowGroupList::CollapseWindowGroupTree() 0x0000de25   Thumb Code   186  goomwindowgrouplist.o(.text)
    CGOomWindowGroupList::RefreshL()         0x0000dedf   Thumb Code  1050  goomwindowgrouplist.o(.text)
    CGOomWindowGroupList::Refresh()          0x0000e2f9   Thumb Code   104  goomwindowgrouplist.o(.text)
    CGOomWindowGroupList::IdleTime(int) const 0x0000e361   Thumb Code   136  goomwindowgrouplist.o(.text)
    CGOomWindowGroupList::~CGOomWindowGroupList() 0x0000e3e9   Thumb Code    90  goomwindowgrouplist.o(.text)
    CGOomWindowGroupList::~CGOomWindowGroupList__sub_object() 0x0000e3e9   Thumb Code     0  goomwindowgrouplist.o(.text)
    CGOomWindowGroupList::~CGOomWindowGroupList__deallocating() 0x0000e443   Thumb Code    22  goomwindowgrouplist.o(.text)
    CGOomWindowGroupList::FindParentIdL(int) 0x0000e459   Thumb Code   170  goomwindowgrouplist.o(.text)
    CGOomWindowGroupList::SetPriorityBusy(int) 0x0000e503   Thumb Code   118  goomwindowgrouplist.o(.text)
    CGOomWindowGroupList::SetPriorityNormal(int) 0x0000e579   Thumb Code   116  goomwindowgrouplist.o(.text)
    CGOomWindowGroupList::SetPriorityHigh(int) 0x0000e5ed   Thumb Code   118  goomwindowgrouplist.o(.text)
    CGOomWindowGroupList::IsBusy(int)        0x0000e663   Thumb Code    86  goomwindowgrouplist.o(.text)
    CGOomWindowGroupList::IsDynamicHighPriority(int) 0x0000e6b9   Thumb Code    96  goomwindowgrouplist.o(.text)
    CGOomWindowGroupList::WgName() const     0x0000e719   Thumb Code     8  goomwindowgrouplist.o(.text)
    CGOomWindowGroupList::GetIndexFromAppId(unsigned) const 0x0000e721   Thumb Code    80  goomwindowgrouplist.o(.text)
    CWservEventReceiver::CWservEventReceiver(CMemoryMonitor&, RWsSession&) 0x0000e7b5   Thumb Code    68  goomwserveventreceiver.o(.text)
    CWservEventReceiver::CWservEventReceiver__sub_object(CMemoryMonitor&, RWsSession&) 0x0000e7b5   Thumb Code     0  goomwserveventreceiver.o(.text)
    CWservEventReceiver::~CWservEventReceiver() 0x0000e7f9   Thumb Code    52  goomwserveventreceiver.o(.text)
    CWservEventReceiver::~CWservEventReceiver__sub_object() 0x0000e7f9   Thumb Code     0  goomwserveventreceiver.o(.text)
    CWservEventReceiver::~CWservEventReceiver__deallocating() 0x0000e82d   Thumb Code    22  goomwserveventreceiver.o(.text)
    CWservEventReceiver::Queue()             0x0000e843   Thumb Code    40  goomwserveventreceiver.o(.text)
    CWservEventReceiver::ConstructL()        0x0000e86b   Thumb Code    90  goomwserveventreceiver.o(.text)
    CWservEventReceiver::DoCancel()          0x0000e8c5   Thumb Code    32  goomwserveventreceiver.o(.text)
    CWservEventReceiver::RunL()              0x0000e8e5   Thumb Code   178  goomwserveventreceiver.o(.text)
    __ARM_switch8                            0x0000e9b0   ARM Code      24  switch8.o(.text)
    __rt_switch8                             0x0000e9b0   ARM Code       0  switch8.o(.text)
    _E32Dll_Body                             0x0000e9c8   ARM Code      76  uc_dll.o(.text)
    Dll::SetTls(void*)                       0x0000ea19   Thumb Code    16  up_dll_tls.o(.text)
    Dll::Tls()                               0x0000ea29   Thumb Code    12  up_dll_tls.o(.text)
    Dll::FreeTls()                           0x0000ea35   Thumb Code    10  up_dll_tls.o(.text)
    __DLL_Export_Table__                     0x0000ea44   ARM Code       4  dllexp.o(.text)
    CGOomConfig::CGOomConfig()               0x0000f0c9   Thumb Code   158  goomconfig.o(i._ZN11CGOomConfigC1Ev)
    CGOomConfig::CGOomConfig__sub_object()   0x0000f0c9   Thumb Code     0  goomconfig.o(i._ZN11CGOomConfigC1Ev)
    CleanupStack::Pop(void*)                 0x0000f191   Thumb Code    16  goomconfigparser.o(i._ZN12CleanupStack3PopEPv)
    CGOomCloseApp::IsRunning()               0x0000f1a1   Thumb Code     6  goomcloseapp.o(i._ZN13CGOomCloseApp9IsRunningEv)
    CGOomRunPlugin::IsRunning()              0x0000f1a7   Thumb Code    12  goomrunplugin.o(i._ZN14CGOomRunPlugin9IsRunningEv)
    CMemoryMonitor::NeedToPostponeMemGood()  0x0000f1b3   Thumb Code    16  goommemorymonitor.o(i._ZN14CMemoryMonitor21NeedToPostponeMemGoodEv)
    CMemoryMonitor::SessionInCriticalAllocation(int) 0x0000f1c3   Thumb Code    48  goommemorymonitorsession.o(i._ZN14CMemoryMonitor27SessionInCriticalAllocationEi)
    CGOomActionList::ClientId()              0x0000f1f3   Thumb Code     8  goomactionlist.o(i._ZN15CGOomActionList8ClientIdEv)
    CGOomPluginList<CGOomMonitorPlugin>::~CGOomPluginList__deallocating() 0x0000f1fb   Thumb Code    22  goomactionlist.o(i._ZN15CGOomPluginListI18CGOomMonitorPluginED0Ev)
    CSimpleScheduler::~CSimpleScheduler__deallocating() 0x0000f211   Thumb Code    24  goommonitor.o(i._ZN16CSimpleSchedulerD0Ev)
    CSimpleScheduler::~CSimpleScheduler()    0x0000f229   Thumb Code    14  goommonitor.o(i._ZN16CSimpleSchedulerD1Ev)
    CSimpleScheduler::~CSimpleScheduler__sub_object() 0x0000f229   Thumb Code     0  goommonitor.o(i._ZN16CSimpleSchedulerD1Ev)
    CGOomConfigParser::~CGOomConfigParser__deallocating() 0x0000f237   Thumb Code    24  goomconfigparser.o(i._ZN17CGOomConfigParserD0Ev)
    CGOomConfigParser::~CGOomConfigParser()  0x0000f24f   Thumb Code    14  goomconfigparser.o(i._ZN17CGOomConfigParserD1Ev)
    CGOomConfigParser::~CGOomConfigParser__sub_object() 0x0000f24f   Thumb Code     0  goomconfigparser.o(i._ZN17CGOomConfigParserD1Ev)
    CGOomPluginWaiter::~CGOomPluginWaiter__deallocating() 0x0000f25d   Thumb Code    24  goompluginwaiter.o(i._ZN17CGOomPluginWaiterD0Ev)
    CGOomPluginWaiter::~CGOomPluginWaiter()  0x0000f275   Thumb Code    14  goompluginwaiter.o(i._ZN17CGOomPluginWaiterD1Ev)
    CGOomPluginWaiter::~CGOomPluginWaiter__sub_object() 0x0000f275   Thumb Code     0  goompluginwaiter.o(i._ZN17CGOomPluginWaiterD1Ev)
    CGOomAppCloseTimer::~CGOomAppCloseTimer__deallocating() 0x0000f283   Thumb Code    24  goomappclosetimer.o(i._ZN18CGOomAppCloseTimerD0Ev)
    CGOomAppCloseTimer::~CGOomAppCloseTimer() 0x0000f29b   Thumb Code    14  goomappclosetimer.o(i._ZN18CGOomAppCloseTimerD1Ev)
    CGOomAppCloseTimer::~CGOomAppCloseTimer__sub_object() 0x0000f29b   Thumb Code     0  goomappclosetimer.o(i._ZN18CGOomAppCloseTimerD1Ev)
    CGOomForegroundRule::~CGOomForegroundRule__deallocating() 0x0000f2a9   Thumb Code    24  goomforegroundrule.o(i._ZN19CGOomForegroundRuleD0Ev)
    CGOomForegroundRule::~CGOomForegroundRule() 0x0000f2c1   Thumb Code    14  goomforegroundrule.o(i._ZN19CGOomForegroundRuleD1Ev)
    CGOomForegroundRule::~CGOomForegroundRule__sub_object() 0x0000f2c1   Thumb Code     0  goomforegroundrule.o(i._ZN19CGOomForegroundRuleD1Ev)
    CAppGOomMonitorPlugin::~CAppGOomMonitorPlugin__deallocating() 0x0000f2cf   Thumb Code    24  goommonitorplugin.o(i._ZN21CAppGOomMonitorPluginD0Ev)
    CAppGOomMonitorPlugin::~CAppGOomMonitorPlugin() 0x0000f2e7   Thumb Code    14  goommonitorplugin.o(i._ZN21CAppGOomMonitorPluginD1Ev)
    CAppGOomMonitorPlugin::~CAppGOomMonitorPlugin__sub_object() 0x0000f2e7   Thumb Code     0  goommonitorplugin.o(i._ZN21CAppGOomMonitorPluginD1Ev)
    CGoomThresholdCrossed::ThreadName()      0x0000f2f5   Thumb Code    30  goommemorymonitor.o(i._ZN21CGoomThresholdCrossed10ThreadNameEv)
    CGoomThresholdCrossed::SetThreshold(int) 0x0000f319   Thumb Code    40  goommemorymonitor.o(i._ZN21CGoomThresholdCrossed12SetThresholdEi)
    CGoomThresholdCrossed::ResetThresholds() 0x0000f351   Thumb Code    44  goommemorymonitor.o(i._ZN21CGoomThresholdCrossed15ResetThresholdsEv)
    CGoomThresholdCrossed::StartRequestEvents() 0x0000f38d   Thumb Code   238  goommemorymonitor.o(i._ZN21CGoomThresholdCrossed18StartRequestEventsEv)
    CGoomThresholdCrossed::RequestNotifications(int) 0x0000f4dd   Thumb Code    88  goommemorymonitor.o(i._ZN21CGoomThresholdCrossed20RequestNotificationsEi)
    CGoomThresholdCrossed::RunL()            0x0000f549   Thumb Code   118  goommemorymonitor.o(i._ZN21CGoomThresholdCrossed4RunLEv)
    CGoomThresholdCrossed::Stop()            0x0000f5d3   Thumb Code    30  goommemorymonitor.o(i._ZN21CGoomThresholdCrossed4StopEv)
    CGoomThresholdCrossed::Trigger(int)      0x0000f5f1   Thumb Code   154  goommemorymonitor.o(i._ZN21CGoomThresholdCrossed7TriggerEi)
    CGoomThresholdCrossed::Continue()        0x0000f6a7   Thumb Code    24  goommemorymonitor.o(i._ZN21CGoomThresholdCrossed8ContinueEv)
    CGoomThresholdCrossed::DoCancel()        0x0000f6c1   Thumb Code    34  goommemorymonitor.o(i._ZN21CGoomThresholdCrossed8DoCancelEv)
    CGoomThresholdCrossed::CGoomThresholdCrossed(CMemoryMonitor&, unsigned, int) 0x0000f6f5   Thumb Code   222  goommemorymonitor.o(i._ZN21CGoomThresholdCrossedC1ER14CMemoryMonitorji)
    CGoomThresholdCrossed::CGoomThresholdCrossed__sub_object(CMemoryMonitor&, unsigned, int) 0x0000f6f5   Thumb Code     0  goommemorymonitor.o(i._ZN21CGoomThresholdCrossedC1ER14CMemoryMonitorji)
    CGoomThresholdCrossed::~CGoomThresholdCrossed__deallocating() 0x0000f7f5   Thumb Code    22  goommemorymonitor.o(i._ZN21CGoomThresholdCrossedD0Ev)
    CGoomThresholdCrossed::~CGoomThresholdCrossed() 0x0000f80d   Thumb Code    86  goommemorymonitor.o(i._ZN21CGoomThresholdCrossedD1Ev)
    CGoomThresholdCrossed::~CGoomThresholdCrossed__sub_object() 0x0000f80d   Thumb Code     0  goommemorymonitor.o(i._ZN21CGoomThresholdCrossedD1Ev)
    CBase::operator new(unsigned)            0x0000f88b   Thumb Code    16  goommonitor.o(i._ZN5CBasenwEj)
    TLex8::TLex8(const TDesC8&)              0x0000f89b   Thumb Code    30  goomconfigparser.o(i._ZN5TLex8C1ERK6TDesC8)
    TLex8::TLex8__sub_object(const TDesC8&)  0x0000f89b   Thumb Code     0  goomconfigparser.o(i._ZN5TLex8C1ERK6TDesC8)
    TFuncLog::Cleanup(void*)                 0x0000f8b9   Thumb Code    22  goomIdletimerule.o(i._ZN8TFuncLog7CleanupEPv)
    TFuncLog::TFuncLog(const char*)          0x0000f8e5   Thumb Code   210  goomIdletimerule.o(i._ZN8TFuncLogC1EPKc)
    TFuncLog::TFuncLog__sub_object(const char*) 0x0000f8e5   Thumb Code     0  goomIdletimerule.o(i._ZN8TFuncLogC1EPKc)
    TFuncLog::~TFuncLog()                    0x0000f9d9   Thumb Code    34  goomconfigparser.o(i._ZN8TFuncLogD1Ev)
    TFuncLog::~TFuncLog__sub_object()        0x0000f9d9   Thumb Code     0  goomconfigparser.o(i._ZN8TFuncLogD1Ev)
    RMessagePtr2::IsNull() const             0x0000fa01   Thumb Code    16  goommemorymonitorsession.o(i._ZNK12RMessagePtr26IsNullEv)
    RSessionBase::SendReceive(int, const TIpcArgs&) const 0x0000fa11   Thumb Code    20  goommonitorsession.o(i._ZNK12RSessionBase11SendReceiveEiRK8TIpcArgs)
    CSimpleScheduler::Error(int) const       0x0000fa25   Thumb Code     2  goommonitor.o(i._ZNK16CSimpleScheduler5ErrorEi)
    CGOomIdleTimeRule::Priority() const      0x0000fa27   Thumb Code     6  goomIdletimerule.o(i._ZNK17CGOomIdleTimeRule8PriorityEv)
    CGOomForegroundRule::Priority() const    0x0000fa2d   Thumb Code     6  goomforegroundrule.o(i._ZNK19CGOomForegroundRule8PriorityEv)
    CGOomWindowGroupList::Count() const      0x0000fa33   Thumb Code    14  goomactionlist.o(i._ZNK20CGOomWindowGroupList5CountEv)
    TDesC8::operator ==(const TDesC8&) const 0x0000fa41   Thumb Code    26  goomconfigparser.o(i._ZNK6TDesC8eqERKS_)
    thunk{-4} to CGOomActionList::ClientId() 0x0000fa5b   Thumb Code    12  goomactionlist.o(i._ZThn4_N15CGOomActionList8ClientIdEv)
    thunk{-4} to CGOomIdleTimeRule::Priority() const 0x0000fa67   Thumb Code     8  goomIdletimerule.o(i._ZThn4_NK17CGOomIdleTimeRule8PriorityEv)
    thunk{-4} to CGOomForegroundRule::Priority() const 0x0000fa6f   Thumb Code     8  goomforegroundrule.o(i._ZThn4_NK19CGOomForegroundRule8PriorityEv)
    operator delete (void*, void*)           0x0000fa77   Thumb Code     2  goomconfigparser.o(i._ZdlPvS_)
    operator new(unsigned, void*)            0x0000fa79   Thumb Code     6  goomIdletimerule.o(i._ZnwjPv)
    CleanupClose<RPointerArray<CImplementationInformation>>::Close(void*) 0x0000fa7f   Thumb Code    14  goomactionlist.o(t._ZN12CleanupCloseI13RPointerArrayI26CImplementationInformationEE5CloseEPv)
    CleanupClose<RFile>::Close(void*)        0x0000fa8d   Thumb Code    12  goomconfigparser.o(t._ZN12CleanupCloseI5RFileE5CloseEPv)
    RPointerArray<CGOomCloseApp>::ResetAndDestroy() 0x0000fa99   Thumb Code    64  goomactionlist.o(t._ZN13RPointerArrayI13CGOomCloseAppE15ResetAndDestroyEv)
    RPointerArray<CGOomRunPlugin>::ResetAndDestroy() 0x0000fad9   Thumb Code    64  goomactionlist.o(t._ZN13RPointerArrayI14CGOomRunPluginE15ResetAndDestroyEv)
    RPointerArray<MGOomRuleConfig>::ResetAndDestroy() 0x0000fb19   Thumb Code    54  goomactionconfig.o(t._ZN13RPointerArrayI15MGOomRuleConfigE15ResetAndDestroyEv)
    CGOomPluginList<CGOomMonitorPlugin>::ConstructL(int) 0x0000fb51   Thumb Code   200  goomactionlist.o(t._ZN15CGOomPluginListI18CGOomMonitorPluginE10ConstructLEi)
    CGOomPluginList<CGOomMonitorPlugin>::Uid(int) 0x0000fc2b   Thumb Code    18  goomactionlist.o(t._ZN15CGOomPluginListI18CGOomMonitorPluginE3UidEi)
    CGOomPluginList<CGOomMonitorPlugin>::NewL(int) 0x0000fc3d   Thumb Code    72  goomactionlist.o(t._ZN15CGOomPluginListI18CGOomMonitorPluginE4NewLEi)
    CGOomPluginList<CGOomMonitorPlugin>::Count() 0x0000fc93   Thumb Code    14  goomactionlist.o(t._ZN15CGOomPluginListI18CGOomMonitorPluginE5CountEv)
    CGOomPluginList<CGOomMonitorPlugin>::TPlugin::TPlugin() 0x0000fca1   Thumb Code    30  goomactionlist.o(t._ZN15CGOomPluginListI18CGOomMonitorPluginE7TPluginC1Ev)
    CGOomPluginList<CGOomMonitorPlugin>::TPlugin::TPlugin__sub_object() 0x0000fca1   Thumb Code     0  goomactionlist.o(t._ZN15CGOomPluginListI18CGOomMonitorPluginE7TPluginC1Ev)
    CGOomPluginList<CGOomMonitorPlugin>::CGOomPluginList() 0x0000fcc5   Thumb Code    48  goomactionlist.o(t._ZN15CGOomPluginListI18CGOomMonitorPluginEC1Ev)
    CGOomPluginList<CGOomMonitorPlugin>::CGOomPluginList__sub_object() 0x0000fcc5   Thumb Code     0  goomactionlist.o(t._ZN15CGOomPluginListI18CGOomMonitorPluginEC1Ev)
    CGOomPluginList<CGOomMonitorPlugin>::~CGOomPluginList() 0x0000fd0d   Thumb Code    86  goomactionlist.o(t._ZN15CGOomPluginListI18CGOomMonitorPluginED1Ev)
    CGOomPluginList<CGOomMonitorPlugin>::~CGOomPluginList__sub_object() 0x0000fd0d   Thumb Code     0  goomactionlist.o(t._ZN15CGOomPluginListI18CGOomMonitorPluginED1Ev)
    RArray<TActionRef>::operator [](int)     0x0000fd7d   Thumb Code    16  goomactionlist.o(t._ZN6RArrayI10TActionRefEixEi)
    RArray<RWsSession::TWindowGroupChainInfo>::ReserveL(int) 0x0000fd8d   Thumb Code    22  goomlog.o(t._ZN6RArrayIN10RWsSession21TWindowGroupChainInfoEE8ReserveLEi)
    RArray<RWsSession::TWindowGroupChainInfo>::RArray() 0x0000fda3   Thumb Code    16  goomwindowgrouplist.o(t._ZN6RArrayIN10RWsSession21TWindowGroupChainInfoEEC1Ev)
    RArray<RWsSession::TWindowGroupChainInfo>::RArray__sub_object() 0x0000fda3   Thumb Code     0  goomwindowgrouplist.o(t._ZN6RArrayIN10RWsSession21TWindowGroupChainInfoEEC1Ev)
    RArray<RWsSession::TWindowGroupChainInfo>::operator [](int) 0x0000fdb3   Thumb Code    16  goomlog.o(t._ZN6RArrayIN10RWsSession21TWindowGroupChainInfoEEixEi)
    RArray<CGOomPluginList<CGOomMonitorPlugin>::TPlugin>::operator [](int) 0x0000fdc3   Thumb Code    16  goomactionlist.o(t._ZN6RArrayIN15CGOomPluginListI18CGOomMonitorPluginE7TPluginEEixEi)
    RHashMap<int, CGOomWindowGroupList::TGOomWindowGroupProperties>::Find(const int&) 0x0000fdd3   Thumb Code    28  goomwindowgrouplist.o(t._ZN8RHashMapIiN20CGOomWindowGroupList26TGOomWindowGroupPropertiesEE4FindERKi)
    RHashMap<long, CGOomRunPluginConfig*>::Find(const long&) 0x0000fdef   Thumb Code    28  goomconfig.o(t._ZN8RHashMapIlP20CGOomRunPluginConfigE4FindERKl)
    RHashMap<long, CGOomApplicationConfig*>::Find(const long&) 0x0000fe0b   Thumb Code    28  goomconfig.o(t._ZN8RHashMapIlP22CGOomApplicationConfigE4FindERKl)
    RHashMap<long, CGOomApplicationConfig*>::InsertL(const long&, CGOomApplicationConfig*const &) 0x0000fe27   Thumb Code    34  goomconfig.o(t._ZN8RHashMapIlP22CGOomApplicationConfigE7InsertLERKlRKS1_)
    RArray<TActionRef>::Count() const        0x0000fe49   Thumb Code    12  goomactionlist.o(t._ZNK6RArrayI10TActionRefE5CountEv)
    RArray<RWsSession::TWindowGroupChainInfo>::Count() const 0x0000fe55   Thumb Code    12  goomwindowgrouplist.o(t._ZNK6RArrayIN10RWsSession21TWindowGroupChainInfoEE5CountEv)
    typeinfo for CGOomAction                 0x00016278   Data          12  goomaction.o(.constdata__ZTI11CGOomAction)
    typeinfo for CGOomConfig                 0x00016284   Data          12  goomconfig.o(.constdata__ZTI11CGOomConfig)
    typeinfo for CGOomLogger                 0x00016290   Data          12  goomlog.o(.constdata__ZTI11CGOomLogger)
    typeinfo for CGOomCloseApp               0x0001629c   Data          12  goomcloseapp.o(.constdata__ZTI13CGOomCloseApp)
    typeinfo for CGOomRunPlugin              0x000162a8   Data          12  goomrunplugin.o(.constdata__ZTI14CGOomRunPlugin)
    typeinfo for CMemoryMonitor              0x000162b4   Data          12  goommemorymonitor.o(.constdata__ZTI14CMemoryMonitor)
    typeinfo for CGOomActionList             0x000162c0   Data          32  goomactionlist.o(.constdata__ZTI15CGOomActionList)
    typeinfo for CGOomPluginList<CGOomMonitorPlugin> 0x000162e0   Data          12  goomactionlist.o(.constdata__ZTI15CGOomPluginListI18CGOomMonitorPluginE)
    typeinfo for MGOomRuleConfig             0x000162ec   Data           8  goomIdletimerule.o(.constdata__ZTI15MGOomRuleConfig)
    typeinfo for CSimpleScheduler            0x000162f4   Data          12  goommonitor.o(.constdata__ZTI16CSimpleScheduler)
    typeinfo for CGOomActionConfig           0x00016300   Data          12  goomactionconfig.o(.constdata__ZTI17CGOomActionConfig)
    typeinfo for CGOomConfigParser           0x0001630c   Data          32  goomconfigparser.o(.constdata__ZTI17CGOomConfigParser)
    typeinfo for CGOomGlobalConfig           0x0001632c   Data          12  goomglobalconfig.o(.constdata__ZTI17CGOomGlobalConfig)
    typeinfo for CGOomIdleTimeRule           0x00016338   Data          32  goomIdletimerule.o(.constdata__ZTI17CGOomIdleTimeRule)
    typeinfo for CGOomPluginWaiter           0x00016358   Data          12  goompluginwaiter.o(.constdata__ZTI17CGOomPluginWaiter)
    typeinfo for CGOomAppCloseTimer          0x00016364   Data          12  goomappclosetimer.o(.constdata__ZTI18CGOomAppCloseTimer)
    typeinfo for CGOomCloseAppConfig         0x00016370   Data          12  goomcloseappconfig.o(.constdata__ZTI19CGOomCloseAppConfig)
    typeinfo for CGOomForegroundRule         0x0001637c   Data          32  goomforegroundrule.o(.constdata__ZTI19CGOomForegroundRule)
    typeinfo for CWservEventReceiver         0x0001639c   Data          12  goomwserveventreceiver.o(.constdata__ZTI19CWservEventReceiver)
    typeinfo for MGOomActionObserver         0x000163a8   Data           8  goomactionlist.o(.constdata__ZTI19MGOomActionObserver)
    typeinfo for CGOomAppCloseWatcher        0x000163b0   Data          12  goomappclosewatcher.o(.constdata__ZTI20CGOomAppCloseWatcher)
    typeinfo for CGOomRunPluginConfig        0x000163bc   Data          12  goomrunpluginconfig.o(.constdata__ZTI20CGOomRunPluginConfig)
    typeinfo for CGOomWindowGroupList        0x000163c8   Data          12  goomwindowgrouplist.o(.constdata__ZTI20CGOomWindowGroupList)
    typeinfo for CMemoryMonitorServer        0x000163d4   Data          12  goommemorymonitorserver.o(.constdata__ZTI20CMemoryMonitorServer)
    typeinfo for CAppGOomMonitorPlugin       0x000163e0   Data          12  goommonitorplugin.o(.constdata__ZTI21CAppGOomMonitorPlugin)
    typeinfo for CGoomThresholdCrossed       0x000163ec   Data          12  goommemorymonitor.o(.constdata__ZTI21CGoomThresholdCrossed)
    typeinfo for CMemoryMonitorSession       0x000163f8   Data          12  goommemorymonitorsession.o(.constdata__ZTI21CMemoryMonitorSession)
    typeinfo for CGOomApplicationConfig      0x00016404   Data          12  goomapplicationconfig.o(.constdata__ZTI22CGOomApplicationConfig)
    typeinfo for CGOomMonitorPluginBase      0x00016410   Data          12  goommonitorplugin.o(.constdata__ZTI22CGOomMonitorPluginBase)
    typeinfo for Xml::MContentHandler        0x0001641c   Data           8  goomconfigparser.o(.constdata__ZTIN3Xml15MContentHandlerE)
    typeinfo name for CGOomAction            0x00016424   Data          14  goomaction.o(.constdata__ZTS11CGOomAction)
    typeinfo name for CGOomConfig            0x00016432   Data          14  goomconfig.o(.constdata__ZTS11CGOomConfig)
    typeinfo name for CGOomLogger            0x00016440   Data          14  goomlog.o(.constdata__ZTS11CGOomLogger)
    typeinfo name for CGOomCloseApp          0x0001644e   Data          16  goomcloseapp.o(.constdata__ZTS13CGOomCloseApp)
    typeinfo name for CGOomRunPlugin         0x0001645e   Data          17  goomrunplugin.o(.constdata__ZTS14CGOomRunPlugin)
    typeinfo name for CMemoryMonitor         0x0001646f   Data          17  goommemorymonitor.o(.constdata__ZTS14CMemoryMonitor)
    typeinfo name for CGOomActionList        0x00016480   Data          18  goomactionlist.o(.constdata__ZTS15CGOomActionList)
    typeinfo name for CGOomPluginList<CGOomMonitorPlugin> 0x00016492   Data          40  goomactionlist.o(.constdata__ZTS15CGOomPluginListI18CGOomMonitorPluginE)
    typeinfo name for MGOomRuleConfig        0x000164ba   Data          18  goomIdletimerule.o(.constdata__ZTS15MGOomRuleConfig)
    typeinfo name for CSimpleScheduler       0x000164cc   Data          19  goommonitor.o(.constdata__ZTS16CSimpleScheduler)
    typeinfo name for CGOomActionConfig      0x000164df   Data          20  goomactionconfig.o(.constdata__ZTS17CGOomActionConfig)
    typeinfo name for CGOomConfigParser      0x000164f3   Data          20  goomconfigparser.o(.constdata__ZTS17CGOomConfigParser)
    typeinfo name for CGOomGlobalConfig      0x00016507   Data          20  goomglobalconfig.o(.constdata__ZTS17CGOomGlobalConfig)
    typeinfo name for CGOomIdleTimeRule      0x0001651b   Data          20  goomIdletimerule.o(.constdata__ZTS17CGOomIdleTimeRule)
    typeinfo name for CGOomPluginWaiter      0x0001652f   Data          20  goompluginwaiter.o(.constdata__ZTS17CGOomPluginWaiter)
    typeinfo name for CGOomAppCloseTimer     0x00016543   Data          21  goomappclosetimer.o(.constdata__ZTS18CGOomAppCloseTimer)
    typeinfo name for CGOomCloseAppConfig    0x00016558   Data          22  goomcloseappconfig.o(.constdata__ZTS19CGOomCloseAppConfig)
    typeinfo name for CGOomForegroundRule    0x0001656e   Data          22  goomforegroundrule.o(.constdata__ZTS19CGOomForegroundRule)
    typeinfo name for CWservEventReceiver    0x00016584   Data          22  goomwserveventreceiver.o(.constdata__ZTS19CWservEventReceiver)
    typeinfo name for MGOomActionObserver    0x0001659a   Data          22  goomactionlist.o(.constdata__ZTS19MGOomActionObserver)
    typeinfo name for CGOomAppCloseWatcher   0x000165b0   Data          23  goomappclosewatcher.o(.constdata__ZTS20CGOomAppCloseWatcher)
    typeinfo name for CGOomRunPluginConfig   0x000165c7   Data          23  goomrunpluginconfig.o(.constdata__ZTS20CGOomRunPluginConfig)
    typeinfo name for CGOomWindowGroupList   0x000165de   Data          23  goomwindowgrouplist.o(.constdata__ZTS20CGOomWindowGroupList)
    typeinfo name for CMemoryMonitorServer   0x000165f5   Data          23  goommemorymonitorserver.o(.constdata__ZTS20CMemoryMonitorServer)
    typeinfo name for CAppGOomMonitorPlugin  0x0001660c   Data          24  goommonitorplugin.o(.constdata__ZTS21CAppGOomMonitorPlugin)
    typeinfo name for CGoomThresholdCrossed  0x00016624   Data          24  goommemorymonitor.o(.constdata__ZTS21CGoomThresholdCrossed)
    typeinfo name for CMemoryMonitorSession  0x0001663c   Data          24  goommemorymonitorsession.o(.constdata__ZTS21CMemoryMonitorSession)
    typeinfo name for CGOomApplicationConfig 0x00016654   Data          25  goomapplicationconfig.o(.constdata__ZTS22CGOomApplicationConfig)
    typeinfo name for CGOomMonitorPluginBase 0x0001666d   Data          25  goommonitorplugin.o(.constdata__ZTS22CGOomMonitorPluginBase)
    typeinfo name for Xml::MContentHandler   0x00016686   Data          24  goomconfigparser.o(.constdata__ZTSN3Xml15MContentHandlerE)
    vtable for CGOomAction                   0x000166a0   Data          28  goomaction.o(.constdata__ZTV11CGOomAction)
    vtable for CGOomConfig                   0x000166bc   Data          20  goomconfig.o(.constdata__ZTV11CGOomConfig)
    vtable for CGOomLogger                   0x000166d0   Data          32  goomlog.o(.constdata__ZTV11CGOomLogger)
    vtable for CGOomCloseApp                 0x000166f0   Data          28  goomcloseapp.o(.constdata__ZTV13CGOomCloseApp)
    vtable for CGOomRunPlugin                0x0001670c   Data          28  goomrunplugin.o(.constdata__ZTV14CGOomRunPlugin)
    vtable for CMemoryMonitor                0x00016728   Data          20  goommemorymonitor.o(.constdata__ZTV14CMemoryMonitor)
    vtable for CGOomActionList               0x0001673c   Data          44  goomactionlist.o(.constdata__ZTV15CGOomActionList)
    vtable for CGOomPluginList<CGOomMonitorPlugin> 0x00016768   Data          20  goomactionlist.o(.constdata__ZTV15CGOomPluginListI18CGOomMonitorPluginE)
    vtable for MGOomRuleConfig               0x0001677c   Data          16  goomIdletimerule.o(.constdata__ZTV15MGOomRuleConfig)
    vtable for CSimpleScheduler              0x0001678c   Data          44  goommonitor.o(.constdata__ZTV16CSimpleScheduler)
    vtable for CGOomActionConfig             0x000167b8   Data          20  goomactionconfig.o(.constdata__ZTV17CGOomActionConfig)
    vtable for CGOomConfigParser             0x000167cc   Data         124  goomconfigparser.o(.constdata__ZTV17CGOomConfigParser)
    vtable for CGOomGlobalConfig             0x00016848   Data          20  goomglobalconfig.o(.constdata__ZTV17CGOomGlobalConfig)
    vtable for CGOomIdleTimeRule             0x0001685c   Data          44  goomIdletimerule.o(.constdata__ZTV17CGOomIdleTimeRule)
    vtable for CGOomPluginWaiter             0x00016888   Data          32  goompluginwaiter.o(.constdata__ZTV17CGOomPluginWaiter)
    vtable for CGOomAppCloseTimer            0x000168a8   Data          32  goomappclosetimer.o(.constdata__ZTV18CGOomAppCloseTimer)
    vtable for CGOomCloseAppConfig           0x000168c8   Data          20  goomcloseappconfig.o(.constdata__ZTV19CGOomCloseAppConfig)
    vtable for CGOomForegroundRule           0x000168dc   Data          44  goomforegroundrule.o(.constdata__ZTV19CGOomForegroundRule)
    vtable for CWservEventReceiver           0x00016908   Data          32  goomwserveventreceiver.o(.constdata__ZTV19CWservEventReceiver)
    vtable for MGOomActionObserver           0x00016928   Data          16  goomactionlist.o(.constdata__ZTV19MGOomActionObserver)
    vtable for CGOomAppCloseWatcher          0x00016938   Data          32  goomappclosewatcher.o(.constdata__ZTV20CGOomAppCloseWatcher)
    vtable for CGOomRunPluginConfig          0x00016958   Data          20  goomrunpluginconfig.o(.constdata__ZTV20CGOomRunPluginConfig)
    vtable for CGOomWindowGroupList          0x0001696c   Data          20  goomwindowgrouplist.o(.constdata__ZTV20CGOomWindowGroupList)
    vtable for CMemoryMonitorServer          0x00016980   Data          40  goommemorymonitorserver.o(.constdata__ZTV20CMemoryMonitorServer)
    vtable for CAppGOomMonitorPlugin         0x000169a8   Data          32  goommonitorplugin.o(.constdata__ZTV21CAppGOomMonitorPlugin)
    vtable for CGoomThresholdCrossed         0x000169c8   Data          32  goommemorymonitor.o(.constdata__ZTV21CGoomThresholdCrossed)
    vtable for CMemoryMonitorSession         0x000169e8   Data          40  goommemorymonitorsession.o(.constdata__ZTV21CMemoryMonitorSession)
    vtable for CGOomApplicationConfig        0x00016a10   Data          20  goomapplicationconfig.o(.constdata__ZTV22CGOomApplicationConfig)
    vtable for CGOomMonitorPluginBase        0x00016a24   Data          32  goommonitorplugin.o(.constdata__ZTV22CGOomMonitorPluginBase)
    vtable for Xml::MContentHandler          0x00016a44   Data          56  goomconfigparser.o(.constdata__ZTVN3Xml15MContentHandlerE)
    CGoomThresholdCrossed::ThreadName()::__PRETTY_FUNCTION__ 0x00016a7c   Data          51  goommemorymonitor.o(.constdata__ZZN21CGoomThresholdCrossed10ThreadNameEvE19__PRETTY_FUNCTION__)
    CGoomThresholdCrossed::SetThreshold(int)::__PRETTY_FUNCTION__ 0x00016aaf   Data          53  goommemorymonitor.o(.constdata__ZZN21CGoomThresholdCrossed12SetThresholdEiE19__PRETTY_FUNCTION__)
    CGoomThresholdCrossed::ResetThresholds()::__PRETTY_FUNCTION__ 0x00016ae4   Data          46  goommemorymonitor.o(.constdata__ZZN21CGoomThresholdCrossed15ResetThresholdsEvE19__PRETTY_FUNCTION__)
    CGoomThresholdCrossed::StartRequestEvents()::__PRETTY_FUNCTION__ 0x00016b12   Data          49  goommemorymonitor.o(.constdata__ZZN21CGoomThresholdCrossed18StartRequestEventsEvE19__PRETTY_FUNCTION__)
    CGoomThresholdCrossed::RequestNotifications(int)::__PRETTY_FUNCTION__ 0x00016b43   Data          54  goommemorymonitor.o(.constdata__ZZN21CGoomThresholdCrossed20RequestNotificationsEiE19__PRETTY_FUNCTION__)
    CGoomThresholdCrossed::RunL()::__PRETTY_FUNCTION__ 0x00016b79   Data          35  goommemorymonitor.o(.constdata__ZZN21CGoomThresholdCrossed4RunLEvE19__PRETTY_FUNCTION__)
    CGoomThresholdCrossed::Cancel()::__PRETTY_FUNCTION__ 0x00016b9c   Data          37  goommemorymonitor.o(.constdata__ZZN21CGoomThresholdCrossed6CancelEvE19__PRETTY_FUNCTION__)
    CGoomThresholdCrossed::Trigger(int)::__PRETTY_FUNCTION__ 0x00016bc1   Data          48  goommemorymonitor.o(.constdata__ZZN21CGoomThresholdCrossed7TriggerEiE19__PRETTY_FUNCTION__)
    CGoomThresholdCrossed::DoCancel()::__PRETTY_FUNCTION__ 0x00016bf1   Data          39  goommemorymonitor.o(.constdata__ZZN21CGoomThresholdCrossed8DoCancelEvE19__PRETTY_FUNCTION__)
    CGoomThresholdCrossed::CGoomThresholdCrossed(CMemoryMonitor&, unsigned, int)::__PRETTY_FUNCTION__ 0x00016c18   Data          89  goommemorymonitor.o(.constdata__ZZN21CGoomThresholdCrossedC1ER14CMemoryMonitorjiE19__PRETTY_FUNCTION__)
    CGoomThresholdCrossed::~CGoomThresholdCrossed()::__PRETTY_FUNCTION__ 0x00016c71   Data          48  goommemorymonitor.o(.constdata__ZZN21CGoomThresholdCrossedD1EvE19__PRETTY_FUNCTION__)
    __ARM__ZN21CGoomThresholdCrossed18StartRequestEventsEv_anon0 0x00016ca4   Data          20  goommemorymonitor.o(.constdata___ARM__ZN21CGoomThresholdCrossed18StartRequestEventsEv_anon0)
    .ARM.exidx$$Base                         0x00016e2c   Number         0  ucppinit.o(.ARM.exidx)
    .ARM.exidx$$Limit                        0x00017804   Number         0  goomactionlist.o(.ARM.exidx)
    Image$$ER_RO$$Limit                      0x00017804   Number         0  anon$$obj.o(linker$$defined$$symbols)

